:100000000C945C210C948D210C948D210C948D21E9
:100010000C948D210C948D210C948D210C948D21A8
:100020000C948D210C948D210C948D210C948D2198
:100030000C948D210D94733E0C948D210C948D2184
:100040000C948D210C94CDDA0C948D210C948D217F
:100050000C948D210C948D210C9494D70D94293EF1
:100060000C948D210C94084D0C94FE4C0C948D2115
:100070000C948D210C948D210C948D210C948D2148
:100080000C948D210C948D210C948D210C948D2138
:100090000C948D210C948D210C948D210C948D2128
:1000A0000C948D210C948D210C948D210C948D2118
:1000B0000C948D210C948D210C948D210C948D2108
:1000C0000C948D210C948D210C948D210C948D21F8
:1000D0000C948D210C948D210C948D210C948D21E8
:1000E0000C948D21084AD73B3BCE016E84BCBFFDEA
:1000F000C12F3D6C74319ABD56833DDA3D00C77FF8
:1001000011BED9E4BB4C3E916BAAAABE0000008090
:100110003F05A84CCDB2D44EB93836A9020C50B91F
:10012000918688083CA6AAAA2ABE000000803F004B
:100130000C943B7D0C9492210D94AA370C9402B23E
:100140000C94AE840C949A7C0C94FCB10C94464DA7
:100150000C9458830C94DA7C0C9471880C949E4D0A
:100160000C9444830D9497380C9415CA0C947D7AA2
:100170000C94C6B10C94E98D0D9411380C94A24DD9
:100180000C9496C90C948A840C94E49B0D942838A2
:100190000C944C830D945F4A0C94E7CB0C942ACBBF
:1001A0000C94D07C0C9475B50C94BB780C948F2176
:1001B0000C94ED870C9427780C940FCB0C94F58756
:1001C0000C9409B30D9419380C940B840C9446804C
:1001D0000D94CA370C94937E0C94D57C0C9432CA3F
:1001E0000D946A380C9458840C94F3830C94F48620
:1001F0000C94E7870D9499370C94B1CC0C943FAADA
:100200000C944B7A0C9448830C9456880C94C44DEF
:100210000C949D7E0D94A4370C94C27C0C94D886CB
:100220000C945C830C943C830C94E4870C94C6C5BA
:100230000C948F7E0C94D37A0C948C7A0D94C637E0
:100240000C9475850C94757B0C94934D0C940C2236
:100250000C94DE8C0C94DEB10C94E0860C94E67A5F
:100260000C94E1870C94754D0C945DB50C94CF966D
:100270000C94AACA0C948FBE0C944D7B0D947E37BF
:100280000D94D0370C94997E0C94D6A00C945B7D81
:100290000C9426A70C9455780C94A37C0C94D286CD
:1002A0000C94F0870D9483370C9480220C94C0B189
:1002B0000C9468900D941E380C9452800C949D25DB
:1002C0000C94BA7B0C945F7D0C94E5840C94BACBAF
:1002D0000C9450830C94D8B10C94417D0C94079BE2
:1002E0000C94EAB50C94667B0D948D380D94A1376F
:1002F0000C9418850C94CCB10D943C380C94D17BA3
:100300000C9498220C94CC4D0C94559D0C94AE4DAD
:100310000D94414A0C9455A20C943A7B0C94EA87B4
:100320000C9471840C940EBF0C944C8F0D94BC37BC
:100330000C942C7D0C94CB7C0C9440830C94457EC7
:100340000C94844D0C940EA90C94B94D0C94A38478
:100350000C9490AE0C9438BF0D94CA160C9453B5FF
:100360000C94F6B10C946E9A0D9479380C94E4B117
:100370000D9456380C940A930C94567D0C942B9F34
:100380000C9474250C94C07A0C94F0B10C94917E6A
:100390000C9459980C94FF7A0D9483380C9412B2F3
:1003A0000D9495370C94187B0C94D2B10C94D08793
:1003B0000C94A77A0C9439990D94D4370C9443B9C2
:1003C0000D94A1380D9498160D946B160C94A64DAF
:1003D0000C94CCA00C94CD940C943F840C94537C3E
:1003E0000D94AB380C94277B0C944EB50D94EE49CC
:1003F0000C94FF250C94E9860C9453880C94A880E7
:100400000D94B8370C94C47C0D9460380C94AF7C78
:100410000C94EFBE0C94EAB10C94867E0C94CBCA7B
:100420000D9444380C94AD780C944A780C942F8534
:100430000C94127D0C94A8CB0C943E7D0C94C67C3D
:100440000C94B24D0C9436860C94DB870C94F78791
:100450000C941DBE0C9403840C949A4D0C94273973
:100460000C9418810C943CBE0C94AEBE0C94FD8789
:100470000C9454830C9419C70C94647A0C948C7B60
:100480000C9458B50C94C5C50D944C380C940D7F44
:100490000D94C1170C9433340C94A4800C949B7E5F
:1004A0000C9408B20C94F47D0C94A0800C94447DC0
:1004B0000C9494780C940B8B0C94CF990D94AE37CC
:1004C0000C9427A40C94AA4D0C94957E0C94DE8772
:1004D0000C94FA870D949D370C94C4840D94323893
:1004E0000C9424B60D94C2370C94367E0D94B43718
:1004F0000C94A37B0C9443C50C9460830C94977E5E
:100500004E414E494E495459494E46CDCCCC3D0AF8
:10051000D7233C17B7D13877CC2B329595E6241FDB
:10052000B14F0A000020410000C84200401C462094
:10053000BCBE4CCA1B0E5AAEC59D7400407A10F367
:100540005A00A0724E18090010A5D4E80000E87601
:1005500048170000E40B54020000CA9A3B00000058
:10056000E1F505000080969800000040420F000071
:1005700000A08601000000102700000000E8030032
:100580000000006400000000000A000000000001FC
:1005900000000000002C76D888DC674F0823DFC1FC
:1005A000DFAE59E1B1B796E5E3E453C63AE65199B7
:1005B0007696E8E6C28426EB898C9B62ED407C6FE0
:1005C000FCEFBC9C9F40F2BAA56FA5F490055A2A97
:1005D000F75C936B6CF9676DC11BFCE0E40D47FEA3
:1005E000F520E6B500D0ED902E0300943577050098
:1005F00080841E080000204E0A000000C80C33331F
:1006000033330F986E12831141EF8D2114893BE62D
:100610005516CFFEE6DB18D1844B381BF77C1D90B6
:100620001DA4BBE424203284725E228100C9F1241F
:10063000ECA1E53D27434F4D4D554E4943415449AB
:100640004F4E0044525952554E004552524F52534C
:1006500000494E464F004543484F004572726F7245
:100660002077726974696E6720746F204545505217
:100670004F4D210A0053544F505045442E200050F6
:1006800072696E7465722073746F70706564206433
:10069000756520746F206572726F72732E204669C3
:1006A0007820746865206572726F7220616E6420B4
:1006B000757365204D39393920746F2072657374F4
:1006C0006172742E202854656D7065726174757244
:1006D000652069732072657365742E2053657420DC
:1006E00069742061667465722072657374617274D6
:1006F000696E67290A004E6F20436865636B7375E6
:100700006D2077697468206C696E65206E756D6206
:1007100065722C204C617374204C696E653A200020
:100720004E6F20436865636B73756D2077697468DD
:10073000206C696E65206E756D6265722C204C614F
:100740007374204C696E653A2000636865636B734F
:10075000756D206D69736D617463682C204C6173D5
:1007600074204C696E653A20004C696E65204E75A8
:100770006D626572206973206E6F74204C617374B2
:10078000204C696E65204E756D6265722B312C2090
:100790004C617374204C696E653A20004D313130E4
:1007A0000053657269616C20737461747573206D98
:1007B00069736D617463680A00776169740A005334
:1007C000442072656164206572726F720A00486F1E
:1007D00074656E642049646C652054696D656F753D
:1007E0007400486F74656E642049646C65205469B8
:1007F0006D656F75740A002121204B494C4C2063B4
:100800006175736564206279204B494C4C20627598
:1008100074746F6E2F70696E0A002121204B494C51
:100820004C2063617573656420627920746F6F205A
:100830006D75636820696E6163746976652074699B
:100840006D65202D2063757272656E7420636F6D07
:100850006D616E643A20007061757365004D3630CD
:1008600030002066696C616D656E745F72756E6FC5
:100870007574200066696C616D656E745F72756E6B
:100880006F757420540046696C616D656E745275A5
:100890006E6F75742054004D656469612052656DFA
:1008A0006F766564004D6564696120496E73657299
:1008B000746564004D313030305300627573793A9D
:1008C0002070617573656420666F7220696E707543
:1008D000740A00627573793A2070617573656420DB
:1008E000666F7220757365720A00627573793A20BB
:1008F00070726F63657373696E670A00506C65612F
:100900007365205265736574005052494E544552C8
:100910002048414C5445440025533A20255300704B
:100920006F7765726F6666004B494C4C45442E20CC
:10093000005072696E7465722068616C7465642E13
:10094000206B696C6C28292063616C6C6564210ADA
:10095000006563686F3A004572726F723A000A4D23
:100960006561737572656420706F696E74733A0A9D
:1009700000387838206D6573682E205A206F6666BF
:100980007365743A20005072696E74696E67204F07
:10099000626A656374002553202569002F2F616307
:1009A00074696F6E3A0073746172740070726F6D67
:1009B00070745F00656E6400486F74656E642074C7
:1009C0006F6F20636F6C640A0053656E64204D3155
:1009D000303820746F20726573756D650A00496E3A
:1009E000736572742066696C616D656E7420616EEA
:1009F000642073656E64204D3130380A005265689A
:100A000065617420446F6E65005265686561746944
:100A10006E672E2E2E005265686561740048656110
:100A20007465722054696D656F75740053656E64EA
:100A3000204D31303820746F2068656174206E6FEE
:100A40007A7A6C650A004E6F7A7A6C652050617212
:100A50006B656400706175736564005061757365E2
:100A600000726573756D656400526573756D696EAE
:100A700067004732362043616E63656C65640047EA
:100A800032362048656174696E67204E6F7A7A6CE1
:100A900065004732362048656174696E672042659B
:100AA000640057616974696E6720666F72206865BB
:100AB000617475702E0A004669786564204C656E15
:100AC000677468205072696D6500446F6E652050D0
:100AD00072696D696E67004D616E75616C20707230
:100AE000696D696E672E2E2E004C656176696E67A2
:100AF00020473236003F537065636966696564203C
:100B0000582C5920636F6F7264696E617465206F31
:100B10007574206F6620626F756E64732E0A003FD5
:100B200028522965706561742076616C7565206E48
:100B30006F7420706C61757369626C653B206D75B4
:100B40007374206265206174206C65617374203158
:100B50002E0A003F537065636966696564206E6F95
:100B60007A7A6C652074656D7065726174757265F2
:100B7000206E6F7420706C61757369626C652E0AEB
:100B8000003F5370656369666965642066696C61DE
:100B90006D656E742073697A65206E6F7420706C59
:100BA00061757369626C652E0A003F5370656369F5
:100BB00066696564207072696D65206C656E677426
:100BC00068206E6F7420706C61757369626C652E3D
:100BD0000A003F537065636966696564206E6F7AC9
:100BE0007A6C652073697A65206E6F7420706C6111
:100BF000757369626C652E0A003F52657472616399
:100C000074696F6E204D756C7469706C69657220C3
:100C10006D757374206265207370656369666965BC
:100C2000642E0A003F5370656369666965642052EB
:100C3000657472616374696F6E204D756C74697050
:100C40006C696572206E6F7420706C617573696277
:100C50006C652E0A003F53706563696669656420A0
:100C60006C6179657220686569676874206E6F745D
:100C700020706C61757369626C652E0A0043292EC1
:100C80000A003F5370656369666965642062656444
:100C90002074656D7065726174757265206E6F7415
:100CA00020706C61757369626C65202834302D008A
:100CB000473236207374617274696E672E2E2E0A65
:100CC000004F46460A0046616465204865696768CA
:100CD000742000426564204C6576656C696E6720FF
:100CE000004661696C656420746F20656E61626C9A
:100CF0006520426564204C6576656C696E670A0004
:100D00004D65736820426564204C6576656C20648F
:100D10006174613A0A00496E76616C6964206D65A0
:100D200073682E0A00206E6F7420656E746572659C
:100D3000642E0A0050726F62696E6720506F696E90
:100D4000740025532025692F256900206F66200037
:100D50004D424C2047323920706F696E7420002953
:100D60000A004A206F7574206F662072616E676595
:100D70002028302D00290A0049206F7574206F66E5
:100D80002072616E67652028302D004732384C3064
:100D9000004D6573682070726F62696E6720646FC2
:100DA0006E65004D6573682070726F62696E6720B2
:100DB000646F6E652E0A005374617274206D6573E2
:100DC000682070726F62696E67207769746820228C
:100DD000473239205331222066697273742E0A001B
:100DE0004732395332004732384C300A4732395390
:100DF0003200686173206E6F20646174612E0A0096
:100E00004D65736820426564204C6576656C696E3B
:100E100067200053206F7574206F662072616E67C3
:100E2000652028302D35292E0A004D657368207005
:100E30006F696E74206F7574206F662072616E67C3
:100E4000650A004D34323120696E636F72726563DA
:100E50007420706172616D6574657220757361676D
:100E6000650A005741524E494E4721204C6F77206A
:100E70005A204A65726B206D6179206C656164202F
:100E8000746F20756E77616E746564207061757320
:100E900065732E0A004F4646004F4E0020204D61DC
:100EA000783A2000200020204D696E3A2000536FD0
:100EB000667420656E6473746F70733A20004D32EF
:100EC000342053256C642054256C64004739322E3D
:100ED00039204525730047312046256400473932C3
:100EE0002E39205A2573004731205A30204632309F
:100EF0003000473120582573205925732046333060
:100F00003030004D34323020532569205A2573008B
:100F10004D3130362050256920532569004D32303F
:100F20003020442573004732385230585900473931
:100F3000322E39204530205A300A47315A25730065
:100F40004D31303920532569004D3139302053253A
:100F500069004D343230205330205A300020496E21
:100F600076616C69642065787472756465722000BE
:100F700047322F47332062616420706172616D6572
:100F8000746572730A00536C6565702E2E2E004DC9
:100F900065736820706F696E74206F7574206F665A
:100FA0002072616E67650A004D302053746F7000C7
:100FB0004D312053746F7000436C69636B20746F04
:100FC00020526573756D652E2E2E004E6F204D6F6D
:100FD00076652E00456E642066696C65206C6973C9
:100FE000740A00426567696E2066696C65206C69E9
:100FF00073740A004E6F206D656469610A00526562
:1010000073756D696E6720534400286E6F206669A2
:101010006C65290043757272656E742066696C6533
:101020003A20005072696E742074696D653A200030
:101030000A53746174733A2046696C616D656E740D
:1010400020757365643A20002C204C6F6E676573C1
:1010500074206A6F623A2000546F74616C20746966
:101060006D653A200053746174733A20002C204659
:1010700061696C65643A20002C2046696E6973686A
:1010800065643A20005072696E74733A200053749C
:101090006174733A2000436F6F6C696E672E2E2E59
:1010A0000048656174696E672E2E2E004520255319
:1010B000006F6B006F666600560651064A064306CF
:1010C000350644454255473A004D313133205300EF
:1010D00042656420436F6F6C696E672E2E2E00424E
:1010E00065642048656174696E672E2E2E00343069
:1010F00030205375506552204F46462E002F2F004A
:101100004D31343520533C696E6465783E206F75EF
:1011100074206F662072616E67652028302D31293A
:101120000A00205200416363656C65726174696FE7
:101130006E3A2050004D32303620580046523A0068
:1011400020466C6F773A20004D424C2041646A750E
:101150007374205A0020643A0020693A0020703AE3
:1011600000496E76616C6964206578747275646597
:10117000720A0020643A0020693A0020703A006444
:10118000697300656E0043290A0061626C65642022
:10119000286D696E2074656D702000436F6C64204B
:1011A00065787472756465732061726520004669A4
:1011B0006C616D656E742072756E6F7574206469F4
:1011C0007374616E636520286D6D293A200046694D
:1011D0006C616D656E742072756E6F757420004F52
:1011E000666673657473204170706C696564004550
:1011F00072723A20546F6F206661722100546F6FD3
:10120000206661722066726F6D2072656665726518
:101210006E636520706F696E740A00454550524FC9
:101220004D204F4B0A002E0A002028302D31302946
:10123000002076616C7565206F7574206F66207272
:10124000616E676500416476616E6365204B3D00A9
:10125000506F7765722D6C6F7373207265636F7654
:1012600065727920004D383400446F6E65207072CD
:10127000696E74696E672066696C650A004D373760
:10128000004D3331004361703A004D4541545041A7
:10129000434B00434F4F4C45525F54454D504552D0
:1012A0004154555245004348414D4245525F5445D3
:1012B0004D504552415455524500424142595354B4
:1012C000455050494E470041524353004D4F5449F9
:1012D0004F4E5F4D4F44455300544845524D414C8D
:1012E0005F50524F54454354494F4E004C4F4E4768
:1012F0005F46494C454E414D45004155544F52457E
:10130000504F52545F53445F53544154555300530C
:10131000445F57524954450052455045415400538B
:1013200044434152440050524F4D50545F53555026
:10133000504F525400454D455247454E43595F501A
:10134000415253455200434153455F4C494748542D
:101350005F4252494748544E45535300544F474704
:101360004C455F4C494748545300534F46545741EE
:1013700052455F504F574552004255494C445F50CB
:10138000455243454E54004C4556454C494E475FE7
:1013900044415441005A5F50524F42450052554E0D
:1013A0004F5554004155544F4C4556454C005052F2
:1013B000494E545F4A4F420050524F475245535393
:1013C000004155544F5245504F52545F54454D5073
:1013D00000564F4C554D45545249430045455052D7
:1013E0004F4D0042494E4152595F46494C455F546A
:1013F00052414E534645520053455249414C5F5865
:101400004F4E5F584F4646004649524D5741524550
:101410005F4E414D453A4D61726C696E20322E30FF
:101420002E375F4457372E3320544D3344203453E6
:101430004D414E4E202841707220323520323032DC
:10144000312030303A30373A35352920534F555214
:1014500043455F434F44455F55524C3A687474703E
:10146000733A2F2F6769746875622E636F6D2F4909
:101470006E73616E6974794175746F6D6174696FB3
:101480006E2F4D61726C696E2F747265652F437299
:1014900065616C6974794477696E5F322E302050D3
:1014A000524F544F434F4C5F56455253494F4E3A5B
:1014B000312E30204D414348494E455F54595045E7
:1014C0003A343030205375506552204558545255A7
:1014D0004445525F434F554E543A31205555494487
:1014E0003A63656465326132662D343161322D3480
:1014F0003734382D396231322D63353563363266F3
:1015000033363766660A0043616E6E6F74206F7003
:10151000656E207375626469722000256973002509
:10152000696D20256973002569682025696D20256E
:10153000697300256964202569682025696D202567
:10154000697300256979202569642025696820254B
:10155000696D202569730023646566696E652044A2
:10156000454641554C545F00626564004B64200061
:101570004B6920004B702000504944204175746F26
:1015800074756E652066696E6973686564212050A4
:10159000757420746865206C617374204B702C2006
:1015A0004B6920616E64204B6420636F6E737461BD
:1015B0006E74732066726F6D2062656C6F77206940
:1015C0006E746F20436F6E66696775726174696FC0
:1015D0006E2E680A00504944204175746F74756E10
:1015E00065206661696C6564212074696D656F753D
:1015F000740A00504944204175746F74756E6520FB
:101600006661696C6564212054656D7065726174F2
:1016100075726520746F6F20686967680A00204BD7
:10162000643A2000204B693A2000204B703A200099
:1016300020436C617373696320504944200A002081
:101640004E6F206F76657273686F6F740A00205456
:10165000753A2000204B753A2000206D61783A20C1
:1016600000206D696E3A200020643A2000206269F3
:1016700061733A2000504944204175746F74756E4F
:10168000652073746172740A005049442041757476
:101690006F74756E65206661696C656421205465A0
:1016A0006D706572617475726520746F6F20686902
:1016B00067680A00504944204175746F74756E65FF
:1016C00000504944204175746F74756E65206661E1
:1016D000696C65642120426164206865617465728B
:1016E0002069640A004572723A2075746638206673
:1016F0006F6E74206E6F7420696E697469616C69B5
:101700007A65642E004572723A20757466382066D8
:101710006F6E74206E6F7420696E697469616C6994
:101720007A65642E004572723A20757466382066B8
:101730006F6E74206E6F7420696E697469616C6974
:101740007A65642E00000C0F00FE07022503BB0122
:101750007FFE08FE08FE05080806000040F0C88865
:1017600088987810050808060000C0F888888888DE
:1017700088F80505050600012030F8302005080826
:101780000600002070F820202020E005090906004E
:10179000FF2070A8A8B888887020070505070001F9
:1017A000D86C366CD80509090600FFF8A888888827
:1017B0008888A8F8050A0A0600FE20505050508874
:1017C000A8A8887003030306000340A040FFFFFFA2
:1017D000FFFFFFFFFFFFFFFFFFFFFFFFFFFFFFFF19
:1017E000FFFFFF0000000605FF010707060200805B
:1017F000808080800080030303060105A0A0A0056F
:10180000060606000050F85050F850050909060079
:10181000FF2070A8A07028A8702005070706000008
:10182000C8C8102040989805070706000040A0A0EF
:1018300040A890680103030602058080800309091F
:101840000601FF20404080808040402003090906B7
:1018500001FF80404020202040408005070706000F
:101860000020A8702070A820050505060001202092
:10187000F820200203030601FFC040800501010695
:101880000003F8020202060100C0C00507070600B7
:1018900000081010204040800507070600007088EF
:1018A00098A8C8887003070706010040C040404060
:1018B00040E0050707060000708808102040F80582
:1018C0000707060000F808103008887005070706AB
:1018D000000010305090F81010050707060000F8BF
:1018E00080F008088870050707060000304080F087
:1018F000888870050707060000F8081010202020CF
:10190000050707060000708888708888700507073B
:10191000060000708888780810600205050601003E
:10192000C0C000C0C00206060601FFC0C000C04023
:1019300080030505060101204080402005030306C1
:101940000002F800F80305050601018040204080F0
:1019500005070706000070881020200020050707F3
:101960000600007088B8A8B8807005070706000058
:10197000708888F8888888050707060000F04848BE
:10198000704848F00507070600007088808080884E
:1019900070050707060000F04848484848F005076A
:1019A00007060000F88080F08080F8050707060031
:1019B00000F88080F08080800507070600007088AE
:1019C0008080988870050707060000888888F88856
:1019D0008888030707060100E04040404040E005DA
:1019E0000707060000381010101090600507070662
:1019F00000008890A0C0A09088050707060000801E
:101A00008080808080F805070706000088D8A888B5
:101A10008888880507070600008888C8A8988888ED
:101A20000507070600007088888888887005070702
:101A3000060000F08888F080808005070706000017
:101A400070888888A89068050707060000F08888D5
:101A5000F0A090880507070600007088807008884D
:101A600070050707060000F8202020202020050729
:101A700007060000888888888888700507070600A0
:101A8000008888888850502005070706000088884D
:101A90008888A8A8500507070600008888502050AD
:101AA0008888050707060000888850202020200528
:101AB0000707060000F80810204080F8030909060F
:101AC00001FFE080808080808080E00507070600BD
:101AD00000804040201010080309090601FFE020A3
:101AE000202020202020E005030306000520508848
:101AF0000501010600FEF8030303060105804020EE
:101B000005050506000070087888780507070600B7
:101B1000008080F0888888F0050505060000708048
:101B2000808870050707060000080878888888788C
:101B30000505050600007088F0807005070706009F
:101B400000304840E04040400507070600FE70882E
:101B500088887808700507070600008080F088886C
:101B600088880307070601004000C0404040E004A9
:101B700009090601FE1000301010101090600507D2
:101B80000706000080808890E09088030707060120
:101B900000C04040404040E0050505060000D0A8D8
:101BA000A8A8A8050505060000B0C888888805050E
:101BB0000506000070888888700507070600FEF09B
:101BC000888888F080800507070600FE7888888866
:101BD000780808050505060000B0C8808080050566
:101BE0000506000078807008F00507070600002051
:101BF00020F8202020180505050600008888889810
:101C0000680505050600008888885020050505063A
:101C100000008888A8A85005050506000088502007
:101C200050880507070600FE8888885020408005F8
:101C30000505060000F8102040F80309090601FF19
:101C40002040404080404040200109090602FF80BA
:101C500080808080808080800309090601FF8040A9
:101C60004040204040408005030306000248A89001
:101C7000FF554E4C4F41442046494C414D454E5432
:101C8000004C4F41442046494C414D454E5400467E
:101C9000494C414D454E54204348414E4745004232
:101CA000656400456E636C6F7375726500256875B9
:101CB0003A25303268750025303268753A25303261
:101CC00068750020202020202020002020202000D7
:101CD0001FE02010201020101020102020102010B5
:101CE00030300840048003001FE03FF03FF03FF039
:101CF0001FE01FE03FF03FF03FF00FC00780030000
:101D00003FFFF038007030FC3020FC1020781020AD
:101D100030102C00D02E31D02F7BD02F7BD02E3105
:101D2000D02C00D020301020781020FC1030FC3057
:101D30003800703FFFF03FFFF038007031863023ED
:101D400087102787902F87D02F03D020301020783E
:101D5000102078102030102F03D02F87D0278790A5
:101D60002387103186303800703FFFF01FFFF81FC7
:101D7000FFF8041040020820020820041040082048
:101D80008010410010410008208004104000000035
:101D90001FFFF81FFFF8FFFFFF8000018E00E19F8B
:101DA00001F19381399F81F99F81F99FB9F98F28BA
:101DB000F18038018000019FFFF99174999B06A979
:101DC0009B54A99B56A99B54999FFFF9FFFFFF6E57
:101DD0006F74696669636174696F6E200063616E18
:101DE00063656C005072696E742041626F72746535
:101DF00064004469736D6973730055492041626FD3
:101E000072746564004D323520500A4D32340052F0
:101E10006573756D65005549205061757365005097
:101E2000617573696E672E2E2E00726573756D6510
:101E3000004D32340052756E6F75742044697374AE
:101E4000206D6D004C6F6164206D6D00556E6C6F80
:101E50006164206D6D0046696C2E204469612E001E
:101E60004520696E206D6D5E3300416476616E635E
:101E700065204B004D3330332055312045256920F6
:101E800053256900504944204175746F74756E651F
:101E9000202A005049442D44202A005049442D490D
:101EA000202A005049442D50202A00200820466155
:101EB0006374002008204D6178002008204D696E71
:101EC000004F6666004F6E004175746F74656D70EB
:101ED000005654726176204D696E00566D696E0031
:101EE000566D6178204500566D6178205A00566D18
:101EF0006178205900566D6178205800416D6178F5
:101F0000204500416D6178205A00416D617820596B
:101F100000416D6178205800412D54726176656CE6
:101F200000412D5265747261637400416363656C96
:101F30000056652D4A65726B00565A2D4A65726BC4
:101F40000056592D4A65726B0056582D4A65726BC2
:101F500000452073746570732F6D6D005A205374A3
:101F60006570732F6D6D00592053746570732F6DFC
:101F70006D00582053746570732F6D6D0041647649
:101F8000616E6365642053657474696E6773003FA6
:101F90000043616E63656C00496E6974004D3432B4
:101FA0003800496E697469616C697A6520454550ED
:101FB000524F4D0046696C616D656E740054656DDD
:101FC00070657261747572650053746570732F6DFE
:101FD0006D004A65726B00416363656C6572617484
:101FE000696F6E0056656C6F636974790053657430
:101FF00020486F6D65204F66667365747300436F8C
:102000006E66696775726174696F6E003F004E6538
:10201000787420506F696E7400446F6E65004E6571
:102020007874004C6576656C696E6720446F6E65E8
:1020300021004D6F7665205A004732395332004EE9
:1020400065787420506F696E74002569202F2025F3
:102050007500473239533100473239533200436CEF
:1020600069636B20746F20426567696E00486F6D0D
:10207000696E672058595A005A2056616C75650080
:10208000496E646578205900496E6465782058006F
:1020900053746F72652053657474696E6773004C76
:1020A0006F61642053657474696E6773004C657664
:1020B000656C20436F726E65727300426564205ACE
:1020C000004661646520486569676874004F66660C
:1020D000004F6E00426564204C6576656C696E67E2
:1020E0000045646974204D657368004C6576656CC5
:1020F00020426564004D6F74696F6E003F0043615C
:102100006E63656C204F626A656374004E4F0059C0
:1021100045530043616E63656C204F626A6563746A
:10212000203D004D61696E00426564004E6F7A7A11
:102130006C650046616E20537065656400436F6E88
:1021400066696775726174696F6E00526573746F4A
:1021500072652044656661756C7473004C6F6164D0
:102160002053657474696E67730053746F726520D1
:1021700053657474696E6773005072656865617445
:10218000202420436F6E6600506F776572204F7574
:1021900074616765004F6666004F6E0052756E6F22
:1021A00075742053656E736F7200416476616E635F
:1021B00065642053657474696E6773004D61696E60
:1021C000004D37303220542564004D3630302042E7
:1021D0003020542564004D373032203B2564004DBB
:1021E00037303120542564004D373032004D3730C0
:1021F00031004D363030204230004D61696E004F65
:102200006666004F6E0052756E6F75742053656E72
:10221000736F72005075726765206D6F7265004351
:102220006F6E74696E756500524553554D45204F6C
:102230005054494F4E533A005052494E5420504149
:10224000555345440020204E6F7A7A6C653A200041
:102250005061726B696E672E2E2E00000057616907
:102260007420666F720066696C616D656E742063C0
:1022700068616E676500746F2073746172740057D3
:1022800061697420666F720066696C616D656E7459
:1022900020756E6C6F616400004E6F7A7A6C6520F9
:1022A00068656174696E6700506C6561736520775D
:1022B0006169742E2E2E0000507265737320627552
:1022C00074746F6E00746F2068656174206E6F7A2D
:1022D0007A6C650000496E736572742066696C6182
:1022E0006D656E7400616E64207072657373206238
:1022F0007574746F6E00746F20636F6E74696E75A1
:1023000065005761697420666F720066696C616D63
:10231000656E74206C6F6164000050726573732089
:10232000427574746F6E00746F20726573756D659D
:10233000207072696E7400005761697420666F7254
:10234000207072696E7400746F20726573756D65AC
:102350002E2E2E00005761697420666F7200666928
:102360006C616D656E7420707572676500003E204B
:1023700000256C642E25696D00457874727564655E
:102380006420546F74616C003E20004C6F6E676572
:102390007374204A6F622054696D65003E200054BA
:1023A0006F74616C205072696E742054696D6500A1
:1023B000436F6D706C65746564003A2000507269FB
:1023C0006E7420436F756E74003A20003135300012
:1023D00035004245443A203125206265746120333E
:1023E0003935300052756E617761792057617463B9
:1023F000683A204F4E004D61782054656D7000336F
:102400003135004D696E2054656D700035004531E1
:102410003A204550434F53203130304B00505355F4
:102420000047656E657269630050726F746F636F09
:102430006C00312E3000426175640032353030302E
:102440003000437265616C69747933442052414DA8
:102450005053004D657368204C6576656C696E67F6
:102460000045787472756465727300310074696E2A
:10247000796D616368696E657333642E636F6D0097
:1024800034303020537550655200323032312D30A7
:10249000342D313800322E302E375F4457372E33EB
:1024A000004D61726C696E005072696E74657220C5
:1024B000537461747300546865726D6973746F72DC
:1024C0007300426F61726420496E666F00507269DA
:1024D0006E74657220496E666F004D61696E004DC5
:1024E000313030300053746F70205072696E740058
:1024F000526573756D65205072696E7400506F7708
:102500006572204F7574616765003F004261636BBF
:102510000053746F70005072696E742066726F6D34
:10252000204D65646961004368616E6765204D6593
:10253000646961004D32310041626F7574205072E0
:10254000696E746572004368616E67652046696CE8
:10255000616D656E7400436F6E6669677572617454
:10256000696F6E0054656D70657261747572650097
:102570004D6F74696F6E00486F737420537461728D
:102580007400526573756D65205072696E74004EEB
:102590006F204D656469610043616E63656C204F17
:1025A000626A6563740054756E650053746F7020C1
:1025B0005072696E74005061757365205072696E57
:1025C0007400496E666F2053637265656E003F004C
:1025D0005374617274205072696E740043616E634B
:1025E000656C005072696E740043616E6E6F74208A
:1025F000656E746572207375626469723A200002B8
:102600002E2E004D61696E002100486F74656E6466
:1026100020746F6F20636F6C64004261636B0050C5
:10262000726F63656564004F6666004F6E00536F9E
:10263000667420456E6473746F7073004D6F7469B7
:102640006F6E0044697361626C65205374657070CD
:10265000657273004D383400426564204C657665C0
:102660006C696E6700486F6D65205A004732385AB2
:1026700000486F6D652059004732385900486F6D2A
:102680006520580047323858004175746F20486FF4
:102690006D6500473238004D61696E0050726568A3
:1026A000656174202420456E640050726568656120
:1026B000742024204265640054656D7065726174F5
:1026C00075726500436F6F6C646F776E0050726552
:1026D0006865617420240046616E205370656564EE
:1026E000207E00426564004E6F7A7A6C65004D6111
:1026F000696E004261627973746570205A004164AA
:1027000076616E6365204B00466C6F770046616EA4
:10271000205370656564207E00426564004E6F7AC8
:102720007A6C6500426564205A00537065656400E8
:102730004D61696E00486F6D696E67204661696C16
:102740006564006F70656E005452494747455245B5
:1027500044003A200066696C616D656E74007A5FB2
:102760006D696E00795F6D696E00785F6D696E00EE
:102770005265706F7274696E6720656E6473746FF2
:1027800070207374617475730A0020746F6F206C0D
:102790006F6E6720657874727573696F6E207072E2
:1027A0006576656E7465640A0020636F6C642065ED
:1027B0007874727573696F6E2070726576656E7469
:1027C00065640A0000000000000000000000000036
:1027D0005761726E696E673A20486F6D696E672047
:1027E00042756D702044697669736F72203C2031A8
:1027F0000A000202040000CD430000C8430000C8E4
:1028000043000000410000004100000040000000C3
:1028100001000000010000800055555500000040F7
:102820000033333300AAAA2A004992240000002072
:1028300000C7711C0099991900D14517005555150D
:10284000003BB113002449120011111100000010C7
:10285000000F0F0F00E3380E0043790D00CCCC0CB5
:1028600000C3300C00E8A20B0064210B00AAAA0AE6
:1028700000703D0A009DD80900427B09009224099E
:1028800000DCD30800888808001042080000000817
:1028900000F0C107008787070075500700711C070B
:1028A000003EEB0600A1BC060069900600666606C5
:1028B00000703E06006118060017F4050074D1058B
:1028C000005BB00500B29005006272050055550529
:1028D0000078390500B81E0500050505004EEC041A
:1028E0000087D40400A1BD040090A704004992040D
:1028F00000C17D0400EE690400C75604004444048E
:10290000005C3204000821040041100400000004AF
:10291000003FF00300F8E0030026D20300C3C30326
:1029200000CCB503003AA803000A9B0300388E03CD
:1029300000C08103009F750300D0690300505E034F
:10294000001D53030034480300913D03003333035B
:102950000016290300381F030097150300300C03ED
:1029600000030303000BFA020049F10200BAE80277
:10297000005CE002002DD802002DD0020059C802F0
:1029800000B0C0020031B90200DAB10200AAAA0206
:1029900000A0A30200BC9C0200FA9502005C8F021A
:1029A00000DF88020082820200457C020027760256
:1029B0000027700200436A02007C640200D05E02BD
:1029C000003F590200C8530200FFFDFCFAF8F6F47C
:1029D000F2F0EEECEAE9E7E5E3E1E0DEDCDAD9D7B4
:1029E000D5D4D2D0CFCDCBCAC8C7C5C3C2C0BFBD56
:1029F000BCBAB9B7B6B4B3B2B0AFADACAAA9A8A6C9
:102A0000A5A4A2A1A09E9D9C9A9998979594939213
:102A1000908F8E8D8B8A8988878684838281807F40
:102A20007E7D7B7A797877767574737271706F6E4C
:102A30006D6C6B6A696867666564636261605F5E3E
:102A40005D5C5B5A59585857565554535251505023
:102A50004F4E4D4C4B4A4A494847464645444342EF
:102A60004241403F3E3E3D3C3B3B3A3938383736A9
:102A70003535343332323130302F2E2E2D2C2B2B56
:102A80002A292928272726252524232322212120F6
:102A9000201F1E1E1D1C1C1B1B1A19191818171687
:102AA00016151514131312121111100F0F0E0E0D0F
:102AB0000D0C0C0B0A0A090908080707060605058C
:102AC0000404030302020100000000CD430000C81B
:102AD000430000C8430000000000000000000000A8
:102AE0000053657474696E67732053746F72656404
:102AF00000454550524F4D20496E697469616C69BB
:102B00007A65640A003B200020204D3630332000D7
:102B100020440020204D34313220530046696C613E
:102B20006D656E742072756E6F75742073656E734B
:102B30006F723A002055004C0046696C616D656EFD
:102B400074206C6F61642F756E6C6F6164206C65AE
:102B50006E677468733A0020204D393030204B0086
:102B60004C696E65617220416476616E63653A00FE
:102B700020204D343133205300506F7765722D4C37
:102B80006F7373205265636F766572793A002044E3
:102B90000020490020204D333034205000204400D4
:102BA00020490020204D333031205000504944202E
:102BB00073657474696E67733A002046002048009C
:102BC00020204D3134352053004D617465726961A8
:102BD0006C2068656174757020706172616D6574D8
:102BE0006572733A002020473239205334205A004E
:102BF000204A00202047323920533320490020202A
:102C00004D3432302053004D657368204265642096
:102C10004C6576656C696E673A0020204D3230361F
:102C2000205800486F6D65206F66667365743A00C2
:102C300020580020530020204D32303520420041E2
:102C40006476616E6365643A20423C6D696E5F73C1
:102C500065676D656E745F74696D655F75733E2041
:102C6000533C6D696E5F66656564726174653E2094
:102C7000543C6D696E5F74726176656C5F66656504
:102C800064726174653E20583C6D61785F785F6A5C
:102C900065726B3E20593C6D61785F795F6A657241
:102CA0006B3E205A3C6D61785F7A5F6A65726B3E5D
:102CB00020453C6D61785F655F6A65726B3E002000
:102CC000540020520020204D323034205000416307
:102CD00063656C65726174696F6E2028756E6974C6
:102CE000732F7332293A20503C7072696E745F61A1
:102CF0006363656C3E20523C726574726163745FFD
:102D0000616363656C3E20543C74726176656C5FF0
:102D1000616363656C3E0020204D323031205800E5
:102D20004D6178696D756D20416363656C65726195
:102D300074696F6E2028756E6974732F7332293A27
:102D40000020204D3230332058004D6178696D7578
:102D50006D206665656472617465732028756E699F
:102D600074732F73293A0053746570732070657201
:102D700020756E69743A0020440020204D323030B6
:102D80002053002044697361626C65640A004669DF
:102D90006C616D656E742073657474696E67733AE7
:102DA0000020204D3134392043203B20556E69747A
:102DB0007320696E2043656C736975730A0020285F
:102DC0006D6D29002020473231202020203B2055E6
:102DD0006E69747320696E206D6D000000FA430007
:102DE00000C84300002041000096420000A04200BD
:102DF00000A0420000C8430000BE42E8030000EE0D
:102E0000020000640000004B00000024F4D43050A5
:102E1000C38E20C2A24017828B7011127A910D814D
:102E20006CD90AA861E108C7586607615143061EBC
:102E30004B5D05C145A7041A411104093D98037172
:102E40003931034036DB0265339102D430540280BD
:102E50002E1D02632CEE01752AC501B028A00110B9
:102E60002781018F2564012B244B01E0223401AC22
:102E7000211F018D200D01801FFC00841EED009795
:102E80001DDF00B81CD200E61BC600201BBC00647E
:102E90001AB200B219A8000A19A0006A189900D144
:102EA00017910040178B00B516840031167E00B3D1
:102EB0001579003A157300C7146F0058146A00EEB4
:102EC0001366008813630025135E00C7125B006C55
:102ED00012570015125400C111510070114F0021FA
:102EE000114B00D61049008D1047004610440002D7
:102EF000104200C00F4000800F3E00420F3C000611
:102F00000F3B00CB0E3800930E37005C0E350027C8
:102F10000E3400F30D3200C10D3100900D30006011
:102F20000D2E00320D2D00050D2C00D90C2B00AEFE
:102F30000C2900850C29005C0C2700350C27000E9D
:102F40000C2600E80B2400C40B2400A00B23007DFA
:102F50000B23005A0B2100390B2100180B2000F81D
:102F60000A1F00D90A1E00BB0A1E009D0A1D008010
:102F70000A1D00630A1C00470A1B002C0A1B0011D3
:102F80000A1A00F7091A00DD091900C4091900AB73
:102F9000091900920917007B091800630917004CF2
:102FA00009160036091600200916000A091500F551
:102FB000081500E0081400CC081400B8081400A498
:102FC000081400900813007D0812006B08130058C5
:102FD00008120046081200340811002308110012DC
:102FE00008110001081100F0071000E0071000D0E0
:102FF000071000C0071000B0070F00A107100091D4
:10300000070E0083070F0074070F0065070E0057B7
:10301000070E0049070E003B070D002E070E00208B
:10302000070D0013070D0006070D00F9060C00ED53
:10303000060D00E0060C00D4060C00C8060C00BC0F
:10304000060C00B0060C00A4060B0099060C008DBF
:10305000060B0082060B0077060B006C060B006166
:10306000060A0057060B004C060A0042060A003802
:10307000060A002E060A0024060A001A060A001094
:1030800006090007060A00FD050900F4050900EB22
:10309000050900E2050900D9050900D0050900C7A6
:1030A000050900BE050900B5050800AD050800A525
:1030B0000509009C050800940508008C050800849B
:1030C0000508007C050800740508006C050700650C
:1030D0000508005D050700560508004E0507004776
:1030E0000507004005080038050700310507002ADC
:1030F000050700230507001C050600160507000F3D
:103100000507000805060002050700FB040600F598
:10311000040700EE040600E8040600E2040700DBF2
:10312000040600D5040600CF040600C9040600C347
:10313000040600BD040600B7040600B1040500AC97
:10314000040600A6040600A00405009B04060095E2
:10315000040500900406008A04050085040500802B
:103160000406007A04050075040500700405006B70
:1031700004050066040500610405005C04050057B1
:10318000040500520405004D0405004804050043F1
:103190000405003E0404003A04050035040500302F
:1031A0000404002C04050027040400230405001E69
:1031B0000404001A04040016040500110404000DA0
:1031C000040400090405000404040000040400FCD5
:1031D000030400F8030400F4030400F0030400EC0B
:1031E000030400E8030400E4030400E0030400DC3B
:1031F000030400D8030400D4030400D0030400CC6B
:10320000030400C8030300C503030024F404D92009
:103210001BC40C5C0E9804C4095F0265077101F4BD
:1032200005F900FB04B30048048700C10369005896
:1032300003550003034500BE023A008402310053E7
:10324000022A002902250004022000E4011C00C813
:10325000011900AF011700980114008401130071D7
:103260000110006101100051010E0043010D0036F4
:10327000010B002B010B0020010B00150109000CB4
:1032800001090003010800FB000800F3000800EB3F
:10329000000700E4000600DE000600D8000600D2A9
:1032A000000600CC000500C7000500C2000500BDF7
:1032B000000400B9000400B5000400B1000400AD32
:1032C000000400A9000400A5000300A20003009F61
:1032D0000004009B00030098000300950002009387
:1032E000000300900003008D0002008B00030088A3
:1032F0000002008600020084000300810002007FBB
:103300000002007D0002007B0002007900020077CD
:1033100000010076000200740002007200010071DA
:103320000002006F0002006D0001006C0002006AE4
:1033300000010069000200670001006600010065ED
:1033400000010064000200620001006100010060F1
:103350000001005F0002005D0001005C0001005BF5
:103360000001005A000100590001005800010057F7
:1033700000010056000100550001005400010053F7
:1033800000000053000100520001005100010050F4
:103390000001004F0001004E0000004E0001004DF2
:1033A0000001004C0001004B0000004B0001004AEE
:1033B00000010049000100480000004800010047EA
:1033C00000010046000000460001004500000045E5
:1033D00000010044000100430000004300010042DE
:1033E00000000042000100410000004100010040D7
:1033F0000001003F0000003F0001003E0000003ED1
:103400000001003D0000003D0001003C0000003CC8
:103410000000003C0001003B0000003B0001003ABE
:103420000000003A000100390000003900010038B6
:1034300000000038000000380001003700000037AD
:1034400000010036000000360000003600010035A3
:103450000000003500000035000100340000003499
:10346000000000340001003300000033000000338E
:103470000001003200000032000000320001003183
:103480000000003100000031000100300000003079
:10349000000000300001002F0000002F0000002F6E
:1034A0000000002F0001002E0000002E0000002E62
:1034B0000001002D0000002D0000002D0000002D57
:1034C0000001002C0000002C0000002C0000002C4B
:1034D0000001002B0000002B0000002B0000002B3F
:1034E0000001002A0000002A0000002A0000002A33
:1034F0000001002900000029000000290000002927
:103500000000002900010028000000280000002819
:10351000000000280000002800010027000000270C
:1035200000000027000000270000002700010026FF
:1035300000000026000000260000002600000026F3
:1035400000010025000000250000002500000025E6
:1035500000000025000000250001002400000024D8
:1035600000000024000000240000002400010023CB
:1035700000000023000000230000002300000023BF
:1035800000000023000000230001002200000022B0
:1035900000000022000000220000002200000022A3
:1035A0000001002100000021000000210000002196
:1035B0000000002100000021000000210001002087
:1035C000000000200000002000000020000000207B
:1035D0000000002000000020000000200001001F6B
:1035E0000000001F0000001F0000001F0000001F5F
:1035F0000000001F0000001F0001001E0000001E50
:103600000000001E0000001E000000232C0000B877
:10361000220000561800003A0F0000B8080000B160
:10362000040000710200003E01000020436F756E2F
:103630007420583A004265640045310062656400B8
:103640002C2073797374656D2073746F707065646A
:1036500021204865617465725F49443A20004865DD
:103660006174696E67204661696C656400486561D4
:1036700074696E67206661696C6564004D31313232
:103680002053687574646F776E001000AA03F00110
:103690003A019002220130031001D00302017004AC
:1036A000F7001005ED00B005E5005006DD00F0065E
:1036B000D7009007D1003008CC00D008C7007009AF
:1036C000C300100ABE00B00ABB00500BB700F00BDD
:1036D000B300900CB000D00DAA00100FA500501040
:1036E000A00090119B00D0129600B014900090168C
:1036F0008B0070188500501A8000301C7B00B01EB3
:10370000750030216F00B023690030266400102856
:103710005F00902A5A00702C5500F02E4F00703137
:103720004800B0324500F0334100703639001037A0
:1037300037005038330090392D00D03A2700B03C84
:103740001C00503D1700F03D1100903E0900D03F95
:10375000E5FF544845524D414C2052554E4157418A
:103760005900546865726D616C2052756E617761A5
:1037700079004572723A204D415854454D50004DE4
:10378000415854454D50207472696767657265648D
:10379000004572723A204D494E54454D50004D49F6
:1037A0004E54454D502074726967676572656400B8
:1037B000202F002042403A0020403A0020573A0093
:1037C00020573A00496E76616C696420657874729E
:1037D000756465720A007C3C3E5E2B3D3F2F5B5D4D
:1037E0003B2C2A225C0043616E6E6F74206F706503
:1037F0006E207375626469722000534420496E69BB
:1038000074204661696C0053442063617264206FC8
:103810006B0A006F70656E526F6F74206661696C21
:1038200065640A00766F6C756D652E696E6974202B
:103830006661696C65640A004E6F205344206361C1
:1038400072640A0041425300504C41000A4D323428
:10385000004D3233202573002E0A006F70656E20F4
:103860006661696C65642C2046696C653A20004687
:10387000696C652073656C65637465640A00205328
:10388000697A653A200046696C65206F70656E65DF
:10389000643A2000454E4420535542524F555449F6
:1038A0004E450A002220706F7300222070617265FD
:1038B0006E743A2200535542524F5554494E45209A
:1038C00043414C4C207461726765743A2200537511
:1038D0006263616C6C204F766572666C6F77004531
:1038E00078636565646564206D6178205355425244
:1038F0004F5554494E452064657074683A002E0A4D
:103900000044656C6574696F6E206661696C6564FE
:103910002C2046696C653A200046696C6520646518
:103920006C657465643A005344207072696E746902
:103930006E67206279746520004E6F7420534420B6
:103940007072696E74696E670A002F6175746F25F5
:10395000632E670057726974696E6720746F206602
:10396000696C653A2000667265736800646F696E01
:1039700067002066696C653A20004E6F7720000270
:10398000FD55555555555FFFFFFFFFFFFFFFFFFF3B
:10399000FE00000000003FFFFFFFFFFFFFFFFFFFF3
:1039A000FD000007FFFFFFFFFFFFFFFFFFFFFFFF1F
:1039B000FE07C00555555555555FFFFFFFFFFFFF3B
:1039C000FC0A200600000000003FFFFFFFFFFFFF92
:1039D000FE141005000007FFFFFFFFFFFFFFFFFFC2
:1039E000FC28080607C00555555555555FFFFFFFD4
:1039F000FE5404040A200600000000003FFFFFFF01
:103A0000FC600406141005000007FFFFFFFFFFFF26
:103A1000FE50040428080607C00555555555555F46
:103A2000FC6004065404040A200600000000003F65
:103A3000FE54041C60040614100500000000001F62
:103A4000FC28082E50040428080607C00001F03F97
:103A5000FE1410546004065404040A200002081FD7
:103A6000FC0A206654041C60040614100005043F80
:103A7000FE07C05428082E5004042808000A021F1C
:103A8000FC00002E14105460040654040015013F7D
:103A9000FE00001C0A206654041C60040018011F6C
:103AA000FC00000607C05428082E50040014013FF3
:103AB000FE00000400002E14105460040018011FC2
:103AC000FCFFFFFE00001C0A206654041C15013F89
:103AD000FED5555400000607C05428082A0A021FC4
:103AE000FC84104600000400002E14105105043F11
:103AF000FEC41044FFFFFE00001C0A206102881F64
:103B0000FC841046D5555400000607C05101F03F13
:103B1000FE84104484104600000400002A00001FA8
:103B2000FCC41046C41044FFFFFE00001C00003F10
:103B3000FE841044841046D5555400000000001F38
:103B4000FCD5555684104484104600000000003F08
:103B5000FCFFFFFCC41046C41044FFFFFFFFFF9FA3
:103B6000FE000006841044841046D555555555BFB7
:103B7000FD555554D5555684104484104104109F6A
:103B8000FFFFFFFCFFFFFCC41046C410410411BF3F
:103B9000FFFFFFFE00000684104484104104109FC4
:103BA000FFFFFFFD555554D5555684104104109F15
:103BB000FFFFFFFFFFFFFCFFFFFCC410410411BF2C
:103BC000FFFFFFFFFFFFFE00000684104104109F6F
:103BD000FFFFFFFFFFFFFD555554D555555555BF08
:103BE000FFFFFFFFFFFFFFFFFFFCFFFFFFFFFF9F48
:103BF000FFFFFFFFFFFFFFFFFFFE00000000003F91
:103C0000FFFFFFFFFFFFFFFFFFFD55555555555FB8
:103C1000FFFFFFFFFFFFFFFFFFFFFFFFFFFFFFFFB4
:103C2000FFFFFFFFFFFFFFFFFFFFFFFFFFFFFFFFA4
:103C3000FFFFFFFFFFFFFFFFFFFFFFFFFFFFFFFF94
:103C4000FFFFFFFFFFFFFFFFFFFFFFFFFFFFFFFF84
:103C5000E02EFB7DFBFBCFC1DFBB3EC0E1FE3C1F86
:103C6000FDEE7B39F9F3CF9EDFBB3EDFDEFCDDE707
:103C7000FDEE3BBBF9EBD7BF5FBB5EDFDEFDEDF7D3
:103C8000FDEEBBD3FAEBB73FDFBB4EDFDFFFCDF37B
:103C9000FDEEDBC7FAEBBB7FC03B6EC0E3FF1DF35D
:103CA000FDEECBEFFADBBB7FDFBB66DFF8FFCDF3CA
:103CB000FDEEEBEFFB5B033F5FBB76DFFE7FEDF3DB
:103CC000FDEEF3EFFB5B79BEDFBB7ADFDE7DEDF768
:103CD000FDEEF3EFFBBAFD9EDFBB7CDFDEFDCDE743
:103CE000FDEEFBEFFBBAFDC1DFBB7EC0E0FE1C1F9B
:103CF0006D61726C696E66772E6F726700322E305E
:103D00002E375F4457372E33001FFFFFFFFFFFFFA3
:103D1000600000000001FF400000000000FF800084
:103D2000000000007F83CF00000C303F87FF800041
:103D30000C301F867980000C000F8C30C7838C30CC
:103D4000E78C30CFC7CC31F38C30DCECEC33B98C62
:103D500030D86C6C33198C30D06C0C33198C30D853
:103D60006C0C33198C30DC6C0E3B198C30CF7C071B
:103D70009F198C30C77C038F19400000000000029F
:103D8000600000000000061FFFFFFFFFFFF870014A
:103D90002C0190012701B0012201C0011D01F00199
:103DA00018011002130130020E0160020901900295
:103DB0000401C002FF000003FA004003F500800385
:103DC000F000D003EB002004E6007004E100E00402
:103DD000DC004005D700C005D2004006CD00D0066B
:103DE000C8008007C3003008BE00F008B900C00951
:103DF000B400B00AAF00B00BAA00D00CA500000EB2
:103E0000A000500F9B00C0109600501291000014AB
:103E10008C00C0158700B0178200B0197D00D01B40
:103E20007800001E730040206E0090226900F0248C
:103E3000640040275F0090295A00E02B5500102EA7
:103E4000500020304B0010324600E03341009035E6
:103E50003C001037370070383200A0392D00B03ADE
:103E60002800A03B2300603C1E00103D1900903D3F
:103E70001400103E0F00703E0A00C03E0500003FD7
:103E80000000403FFBFF803FF6FFC03FF1FF2020D6
:103E9000506C616E6E6572427566666572427974C9
:103EA00065733A20002046726565204D656D6F721E
:103EB000793A2000436F6D70696C65643A204170F7
:103EC0007220323520323032310A00204C61737456
:103ED00020557064617465643A20323032312D307F
:103EE000342D3138207C20417574686F723A20542B
:103EF000696E794D616368696E657333440A003297
:103F00002E302E375F4457372E330A004D61726CC6
:103F1000696E0020536F6674776172652052657315
:103F200065740A00205761746368646F6720526586
:103F30007365740A002042726F776E206F7574206B
:103F400052657365740A002045787465726E616C01
:103F50002052657365740A00506F77657255700A58
:103F60000073746172740A004732385859004D3139
:103F7000303031006572726F722077726974696EC9
:103F80006720746F2066696C650A00446F6E652057
:103F9000736176696E672066696C652E0A004D3222
:103FA0003900456E6473746F707300255320256368
:103FB00020256320256320256300205A3A002059DC
:103FC0003A0020583A00656E6473746F707320680D
:103FD00069743A200000000A0B02090C0D0E080754
:103FE00003040100000000000000000000000000C9
:103FF00000000000000000000000000000000000C1
:10400000001211100000000000000000000000007D
:104010000000000000000000000000004D6F766509
:104020002025736D6D004D6F766520302E316D6DDE
:10403000004D6F766520316D6D004D6F76652031D6
:10404000306D6D004D6F766520417869730045785D
:10405000747275646572004D6F7665205A004D6FFD
:1040600076652059004D6F766520580048384438F1
:104070004368616E67652046696C616D656E7400AA
:10408000556E6C6F61642046696C616D656E74007D
:104090004C6F61642046696C616D656E740050728E
:1040A000656865617420437573746F6D0050726547
:1040B000686561742024004261636B00FFFFFF4864
:1040C0006F6D65202573257325732046697273749F
:1040D0000073686F7700627574746F6E0062656755
:1040E000696E0044697361626C6552756E6F7574B8
:1040F0000050757267654D6F72650050617573652C
:104100006400436F6E74696E7565004C6F61642066
:1041100046696C616D656E74205400496E736572FA
:10412000742066696C616D656E7420616E642073C5
:10413000656E64204D3130380A00220A00556E6BDE
:104140006E6F776E20636F6D6D616E643A20220032
:104150002042002050006F6B0034303020537550E7
:1041600065522052656164792E005072696E7469DF
:104170006E672E2E2E005072696E7420506175731A
:10418000656400204500205A00205900204D393236
:1041900020580020453A00205A3A0020593A005849
:1041A0003A0020746F6F206C6F6E672065787472B0
:1041B0007573696F6E2070726576656E7465640ADA
:1041C0000020636F6C6420657874727573696F6E1C
:1041D0002070726576656E7465640A005265736559
:1041E0006E643A20006E6F74696669636174696F0A
:1041F0006E200000002200250028002B002E003138
:1042000000340002010000050108010B010000213B
:1042100000240027002A002D003000330001010097
:1042200000040107010A010505050507050808083E
:1042300008020202020A0A08080404040401010137
:10424000010101010103030303030303030407073F
:10425000070C0C0C0C0C0C0C0C02020202060606DD
:1042600006060606060B0B0B0B0B0B0B0B010210C5
:104270002020080810204010204080020102010880
:104280000402010102040810204080804020100830
:104290000402018004020180402010080402010889
:1042A00004020101020408102040800102040810E9
:1042B00020408000CA00880111241FBECFEFD1E248
:1042C000DEBFCDBF00E00CBF13E0A0E0B2E0E4E54C
:1042D000F1EC02E00BBF02C007900D92A037B107CE
:1042E000D9F729E1A0E7B3E001C01D92AA39B207CE
:1042F000E1F711E2CBE5D1E200E006C02197010928
:10430000802FFE010F94005DCA35D10780E00807B9
:10431000A9F70F94B24B0D9498600C940000FC0127
:1043200084910895FC018081089511980000000097
:104330009091020187FD9095917090930001119AE0
:1043400000000000000000001198000000009091A3
:10435000020186FD9095917090930001119A0000E2
:104360000000000000001198000000009091020180
:1043700085FD9095917090930001119A00000000C6
:10438000000000001198000000009091020184FDDF
:104390009095917090930001119A00000000000028
:1043A00000001198000000009091020183FD90959B
:1043B000917090930001119A00000000000000002D
:1043C0001198000000009091020182FD909591707B
:1043D00090930001119A0000000000000000119865
:1043E000000000009091020181FD909591709093E2
:1043F0000001119A00000000000000001198000068
:10440000000080910201817080930001119A0000E8
:10441000000000000000089590E080E00895CF9330
:10442000DF93DB01F9019C919130C1F0943080F071
:1044300094509C938830D1F480819181009771F0E1
:10444000019791838083480F591FEA01188206C0A3
:104450008C3539F49C5F9C93943041F4DF91CF917B
:1044600008958B3339F781E08C93F8CF2081318127
:10447000B9016F5F7F4F71836083420F531FEA0161
:104480008883808191818F3591056CF7E7CF0F93F9
:104490001F9381E00091811710918217209183175B
:1044A0003091841740917D1750917E1760917F174E
:1044B00070918017041715072607370708F480E066
:1044C0001F910F91089590E080E00895282F90911A
:1044D0001209833021F495FD0FC094FD0FC0892F80
:1044E00090E0B0E0A0E004C0B695A79597958795B9
:1044F0002A95D2F78170089581E0089580E00895AB
:104500001092F9088091510290915202A0915302A9
:10451000B09154028093E0069093E106A093E206E6
:10452000B093E3060895129A0895269A2E9A089554
:10453000AF92BF92CF92DF92EF92FF920F931F93B1
:10454000CF93DF936B01E9014A3009F4C1C04531D3
:1045500009F073C0DB011296ED91FC91F280C681E7
:10456000D78180910201809582708093000188E25A
:104570008A950000E9F7BF2CB29420EFB22230E117
:10458000A32EAF0C48E2E42E88EF0E9495218E2DD9
:104590008A950000E9F7BFE1BF1508F485C08F2DAB
:1045A000807780680E9495218B2D0E9495218E2D09
:1045B0008A950000E9F780E80E94952180E00E943A
:1045C00095218E2D8A950000E9F78AEF0E949521AA
:1045D0008E2D8A950000E9F78E01005F1F4F8881BC
:1045E000807F0E94952189918295807F0E949521EC
:1045F000C017D107A1F78E2D8A950000E9F7F39433
:10460000E0E1BE0EFA10C0CF80910201827080936B
:104610000001D6011296CD91DC91CE010F94123F8C
:10462000811147C2DF91CF911F910F91FF90EF90C1
:10463000DF90CF90BF90AF900895FB01028113816E
:10464000423309F4F1C108F4F5C1463409F4E2C17A
:10465000473409F4E5C14B3329F589812B81D80111
:1046600012966C91129713964C91213009F438C22E
:10467000233009F002C238EF380F582F91E043176A
:1046800008F490E041E0531708F040E031E056179D
:1046900008F430E0592F542B352309F016C2942327
:1046A00009F013C281E0BECF80EE8F0D8068807F5D
:1046B0000E9495218F2D8295807F0E9495218E2DBD
:1046C0008A950000E9F780E80E94952180E877CF7D
:1046D00080910101826080930101809102018270CA
:1046E000809300018091010181608093010180919C
:1046F0000201817080930001099A119A8091020150
:10470000809582708093000188E28A950000E9F725
:1047100088E790E0CEE9DFE0FE013197F1F70197FD
:10472000D9F788EF0E94952118E2812F8A95000021
:10473000E9F780E20E94952180E00E949521812F77
:104740008A950000E9F780E00E94952180E80E94A8
:104750009521812F8A950000E9F780E00E9495213C
:1047600080E10E949521812F8A950000E9F7CE0112
:104770000197F1F7CE010197F1F7CE010197F1F71B
:10478000CE010197F1F7CE010197F1F7CE01019724
:10479000F1F7CE010197F1F7CE010197F1F7CE01C4
:1047A0000197F1F7CE010197F1F7CE010197F1F7EB
:1047B000CE010197F1F7CE010197F1F7CE010197F4
:1047C000F1F72197F1F780E20E94952180E40E94A1
:1047D0009521812F8A950000E9F780E20E949521BA
:1047E00080E60E9495211A950000E9F710E0D0E0DC
:1047F000C8E28D2F807780680E949521812F0E94CA
:1048000095218C2F8A950000E9F780E80E94952178
:1048100080E00E9495218C2F8A950000E9F78AEFAD
:104820000E9495218C2F8A950000E9F790E211985B
:104830000000000080910201817080930001119AB4
:1048400000000000000000001198000000008091AE
:104850000201817080930001119A000000000000A5
:104860000000119800000000809102018170809387
:104870000001119A000000000000000011980000E3
:10488000000080910201817080930001119A000064
:10489000000000000000119800000000809102015B
:1048A000817080930001119A000000000000000058
:1048B0001198000000008091020181708093000136
:1048C000119A000000000000000011980000000094
:1048D00080910201817080930001119A0000000014
:1048E000000000001198000000008091020181701A
:1048F00080930001119A0000000000000000119850
:104900000000000080910201817080930001119AE3
:1049100000000000000000001198000000008091DD
:104920000201817080930001119A000000000000D4
:1049300000001198000000008091020181708093B6
:104940000001119A00000000000000001198000012
:10495000000080910201817080930001119A000093
:10496000000000000000119800000000809102018A
:10497000817080930001119A000000000000000087
:104980001198000000008091020181708093000165
:10499000119A0000000000000000119800000000C3
:1049A00080910201817080930001119A0000000043
:1049B0000000000011980000000080910201817049
:1049C00080930001119A00000000000000008C2F6D
:1049D0008A950000E9F7915009F029CF88EF0E94ED
:1049E00095218C2F8A950000E9F7DF5F105FD032A8
:1049F00009F0FFCE80E00E94952180EC0E94952175
:104A0000CA950000E9F7809102018270809300014D
:104A100081E008CED80115968C91888381E002CE82
:104A2000F80181818883FACFB901C8010F942F3F23
:104A300081E0F8CD443171F0473109F033CE18826E
:104A4000F80182818983858181508A8383818B8368
:104A500081E0E8CDD80115964C91159750E0440FB0
:104A6000551F70E060E016968D919C910F9439600F
:104A7000C8010F94283F81E0D5CD481708F412CE25
:104A8000861708F40FCEFA80E12CD12C243070F474
:104A90001DC0BE01C8010F942F3F898198819D0DD3
:104AA00098838E0D8983FF0C09F4FCCDF7FEF6CFB9
:104AB000F0CF4D8150E0440F551F70E060E08E81D3
:104AC0009F810F94396081E0ADCDFA8030E0F9012B
:104AD000E555FD4FD08029553D4FF901E080E6CFE7
:104AE00058E0580F382FCACDEF92FF920F931F93C3
:104AF000CF93DF93EC018B017A018A859B85861722
:104B0000970731F0888199810F9408411B870A87A4
:104B1000B701888199810F94B1322E813F81820F34
:104B2000932F911D9F838E8390E080E0DF91CF9142
:104B30001F910F91FF90EF9008959F92AF92BF92B7
:104B4000CF92DF92EF92FF920F931F93CF93DF9359
:104B5000EC018B01942EA52E8A859B8586179707DD
:104B600031F0888199810F9408411B870A878885D5
:104B70009985019649F5BC800A818E81080FC8800D
:104B8000D980D6015596ED91FC91C6011995B80EC4
:104B9000E92CFA2C10E0F70121917F01211127C0A7
:104BA0008E819F81810F911D9F838E8390E080E095
:104BB000DF91CF911F910F91FF90EF90DF90CF90F9
:104BC000BF90AF909F9008950E811F81692D7A2D1F
:104BD000888199810F94B132800F912F911D288582
:104BE00039852817390738F681E090E0E1CF4B2D61
:104BF000602FC6010F946041080F180FCCCFDF92D1
:104C0000EF92FF920F931F93CF93DF93EC01D62E79
:104C10001CAD0BAD7C0184E0E80EF11CE98DFA8D32
:104C2000C7011995412F480F2D2D602FC7010F94F3
:104C300060419BAD890F8BAF81E090E0DF91CF9118
:104C40001F910F91FF90EF90DF900895AB01BC0191
:104C50004093811750938217609383177093841742
:104C60008AEE98E10C94AAD1809323028032B8F5A1
:104C700090910F05891724F091E0980F90930F05FC
:104C800040910B0550910C0560910D0570910E053A
:104C9000082E04C076956795579547950A94D2F7E4
:104CA00041704093FE1087FD1DC0282F082E000C78
:104CB000330B3F938F9386E899E09F938F9386E918
:104CC00099E09F938F931F920E948BB58DB79EB7EB
:104CD00007960FB6F8949EBF0FBE8DBF0895109231
:104CE000FE10E1CF0D9418460F931F93CF93DF93DF
:104CF00000D01F92CDB7DEB79C0100EE18E090E126
:104D0000E9E4F1E1D80101900D929A95E1F7F901FA
:104D10002081318142815381F801608571858285CE
:104D200093850F94095DF801608771878287938767
:104D300080E090E0A0EAB0E489839A83AB83BC83EF
:104D4000CE0101960E946AFC0F900F900F900F9079
:104D5000DF91CF911F910F9108952F923F924F9223
:104D60005F926F927F928F929F92AF92BF92CF92FB
:104D7000DF92EF92FF921F93CF93DF93CDB7DEB711
:104D80002C970FB6F894DEBF0FBECDBF7A01190184
:104D9000DC012D913D914D915C912D833E834F839C
:104DA0005887FB0140805180628073808090491158
:104DB00090904A11A0904B11B0904C11A501940114
:104DC0006D817E818F8198850F94175681110EC059
:104DD00011E0A301920160914D1170914E118091EB
:104DE0004F11909150110F941756811110E0D1017D
:104DF0002D913D914D915C9129873A874B875C8736
:104E0000F701C080D180E280F380209109023091C7
:104E10000A0240910B0250910C02C701B6010F9497
:104E20001756882309F44EC0C0920902D0920A0294
:104E3000E0920B02F0920C02809155119091561164
:104E4000A0915711B091581140914D1150914E11B0
:104E500060914F11709150118092E0089092E1089A
:104E6000A092E208B092E3084093E4085093E5086A
:104E70006093E6087093E708C092E808D092E908CA
:104E8000E092EA08F092EB088093EC089093ED082A
:104E9000A093EE08B093EF0820E030E040E05FE33D
:104EA00060912C1170912D1180912E1190912F11E4
:104EB0000F947D5669837A838B839C83CE01019600
:104EC0000E946AFC2D813E814F8158852093E00825
:104ED0003093E1084093E2085093E3084092E408DD
:104EE0005092E5086092E6087092E708D1012D9192
:104EF0003D914D915C916091EC087091ED0880912D
:104F0000EE089091EF080F94095D6093EC087093A0
:104F1000ED088093EE089093EF0811112FC020E068
:104F200030E0A90169857A858B859C850F94175699
:104F3000811133C060E070E088EC92E469837A8389
:104F40008B839C83CE0101960E946AFC2C960FB63F
:104F5000F894DEBF0FBECDBFDF91CF911F91FF90C0
:104F6000EF90DF90CF90BF90AF909F908F907F9009
:104F70006F905F904F903F902F9008952AEF3EE7FB
:104F80004AE25FE3609130117091311180913211EA
:104F9000909133110F947D56D1CF60E070E080EA9C
:104FA00091E4CCCF8091C6049091C704009731F072
:104FB0004AE050E070E060E00D94325460E070E050
:104FC000CB01089580910B0A82FF0BC063E682E754
:104FD0009AE00E94A6B50F941C390E9471BC81E032
:104FE000089580E008958091C6049091C7040097C9
:104FF00031F04AE050E070E060E00D94045360E06E
:1050000070E0CB010895AF92BF92CF92DF92EF9202
:10501000FF920F931F93CF93DF93EC015B018A0103
:10502000FB01199587FD16C0C82ED12CF12CE12C5F
:105030002196F801C082D182E282F382CE01DF9113
:10504000CF911F910F91FF90EF90DF90CF90BF9085
:10505000AF900895982F907E903CA9F48F7190E0C6
:10506000B0E0A0E06C017D0156E0CC0CDD1CEE1C34
:10507000FF1C5A95D1F7CE010196F50119958F7352
:10508000C82A2296D6CF982F907F903E11F58F7028
:1050900090E0B0E0A0E06C017D0136E0CC0CDD1CBE
:1050A000EE1CFF1C3A95D1F7CE010196F50119953A
:1050B0008F73C82A46E0CC0CDD1CEE1CFF1C4A9501
:1050C000D1F7CE010296F50119958F73C82A239660
:1050D000B0CF982F987F903F79F5877090E0B0E03F
:1050E000A0E06C017D0186E0CC0CDD1CEE1CFF1CF9
:1050F0008A95D1F7CE010196F50119958F73C82ACB
:1051000096E0CC0CDD1CEE1CFF1C9A95D1F7CE016D
:105110000296F50119958F73C82A26E0CC0CDD1C88
:10512000EE1CFF1C2A95D1F7CE010396F5011995C7
:105130008F73C82A24967DCF982F907C903841F4A5
:10514000807C803869F42196CE01F5011995F8CF5D
:105150008E7F8D3F28F02196CE01F5011995F8CF6D
:10516000C12CD12C760165CF9CE0899F802D112424
:1051700091E0980F909310052CE0280F2093DA0807
:1051800030E02E5F3F4F409133174217130619F05E
:1051900014F080E00895209135179217D0F7662318
:1051A00041F08E5F0F9422408091DA088E5F0F9459
:1051B00022408091DA0890913317891750F320919B
:1051C000351790911005291720F310923617809308
:1051D000371781E00895CF9380910205811154C063
:1051E0001092361710923717109238171092041732
:1051F00010920317109206171092051710920817B5
:1052000081E08093071782E28093091710920E17AE
:1052100010920D17E2E2F7E120E337E18FEF81937F
:105220002E173F07E1F7C1E0C0931F172CEA31E0CA
:105230003093151720931417C09316171092171751
:105240001092181790E49093191710921A1722EEE3
:1052500031E0309331172093301726E132E030935C
:1052600002172093011797E19093261791E19093ED
:10527000271790E190932417809323178093221788
:105280000F94493FC093020581E08093030585E4B4
:1052900097E1909372168093711610927416109283
:1052A0007316CF91089520910105022E000C330B47
:1052B0008217130641F08093010565E477E18FEFD3
:1052C00096E10D9408410895CF92DF92EF92FF92FC
:1052D0000F931F93CF93DF93CDB7DEB72C970FB605
:1052E000F894DEBF0FBECDBF6F3F710581059105FC
:1052F00009F0D0F48BEF96E10E94FF25E0910317AF
:10530000F09104173196849190E02C960FB6F894A2
:10531000DEBF0FBECDBFDF91CF911F910F91FF90E8
:10532000EF90DF90CF900895F0903617E090371708
:105330002091030521110FC045E257E16E2D8F2DFD
:105340000F94CC4190E080E0F80EF0923617E09296
:1053500037179927DACFC0900317D09004172FEF93
:1053600036E13A8329832F2D30E03C832B832E2D89
:1053700030E03E832D8318861F822FEF3FEF3A8760
:1053800029871C861B860DE915E29E012F5F3F4F82
:10539000AB01BC01C6010F94EE28B6018FEF96E178
:1053A0000F9408418F819885CFCFCF93DF93FC0175
:1053B00025AD211104C021E025AF0F94493FC091D4
:1053C0000117D0910217E0913017F091311782E068
:1053D0001995E0913017F091311781E0199530E07F
:1053E00020E044E1BE018FEF96E10F94453F22E3B8
:1053F00037E147E1BE018FEF96E10F94453FE09121
:105400003017F091311780E0DF91CF911994CF924E
:10541000DF92EF92FF920F931F93CF93DF93CDB75D
:10542000DEB72C970FB6F894DEBF0FBECDBFF0905D
:105430003617E09037172091030521111DC045E074
:1054400057E16E2D8F2D0F94CC4190E080E0F80E47
:10545000F0923617E092371799272C960FB6F894EA
:10546000DEBF0FBECDBFDF91CF911F910F91FF9097
:10547000EF90DF90CF900895C0900317D09004175D
:105480002FEF36E13A8329832F2D30E03C832B83A5
:105490002E2D30E03E832D8318861F827A87698700
:1054A0001C861B860DE915E29E012F5F3F4F4FE8DA
:1054B00051E2BC01C6010F94B229B6018FEF96E10B
:1054C0000F9408418F819885C2CF6FEF7FEF0C94C6
:1054D000072ACF92DF92EF92FF920F931F93CF9301
:1054E000DF93CDB7DEB72C970FB6F894DEBF0FBEB3
:1054F000CDBFF0903617E0903717209103052111AA
:105500001DC045EE56E16E2D8F2D0F94CC4190E0DD
:1055100080E0F80EF0923617E092371799272C9614
:105520000FB6F894DEBF0FBECDBFDF91CF911F91B4
:105530000F91FF90EF90DF90CF900895C0900317E8
:10554000D09004172FEF36E13A8329832F2D30E0D6
:105550003C832B832E2D30E03E832D8318861F82C3
:105560007A8769871C861B860DE915E29E012F5FED
:105570003F4F42E951E2BC01C6010F94B229B60186
:105580008FEF96E10F9408418F819885C2CFBF922B
:10559000CF92DF92EF92FF920F931F93CF93DF93FF
:1055A0008B01F42EE90141FB662760F90E94B428C3
:1055B000882309F45AC0B12C0115110521F0C80146
:1055C0000E9442BDB82EE12C209721F0CE010E940E
:1055D0002DBFE82E80E8C82ED12CF0FE1EC085E13C
:1055E00090E08B199109B7FC93958E199109E7FC0E
:1055F000939597FD019695958795F82E30E8C32EE3
:10560000D12CFA94F7FC09C060E270E080E090E0F1
:105610000E946429C81AD90AF4CFBB2099F0C601A8
:1056200066E070E00F94D85C262F4091DC08509122
:10563000DD086091DB08C8010E9482BC96E0899F6A
:1056400060011124EE2031F0B601CE010E94692ADA
:10565000C81AD90A87E0C816D10438F060E270E0B1
:1056600080E090E00E946429F3CFDF91CF911F91F9
:105670000F91FF90EF90DF90CF90BF9008956FEF64
:105680007FEF0C94692AAF92BF92CF92DF92EF9294
:10569000FF920F931F93CF93DF935C016B010E94E6
:1056A00042BDE82EC6010E942DBFF12C03E110E09F
:1056B000081B1109C5E20E151F050CF4CFE18C2F54
:1056C00090E09C012E5F3F4F409133174217130625
:1056D00009F0CCF5099720913517281719069CF188
:1056E0004091DC085091DD086091DB08109236177C
:1056F000C093371725E1C5010E9482BCD1E0C114D7
:10570000D104B1F06AE370E080E090E00E94642987
:105710000E151F05D4F4C45F80913317C81740F0ED
:10572000209135174C2F4950550B241715067CF442
:10573000DF91CF911F910F91FF90EF90DF90CF906D
:10574000BF90AF900895D0E0DACFDD2389F3802FAA
:10575000880F080F000F00933617C093371760E2C9
:1057600070E080E090E00E946429C601DF91CF9153
:105770001F910F91FF90EF90DF90CF90BF90AF906F
:105780000C943F2B8F929F92AF92BF92CF92DF9259
:10579000EF92FF920F931F93CF93DF93CDB7DEB7B6
:1057A0002C970FB6F894DEBF0FBECDBF982F862F73
:1057B0005A017901D02E692F0E94B428882309F458
:1057C00089C0C701002391F10E9442BDC82E80907C
:1057D00003179090041780910305811145C01FEFB6
:1057E00023E12C194091DC085091DD086091DB0821
:1057F000C5010E9482BCCC2009F46CC0B6E08B9F2E
:10580000500111246AE370E080E090E00E94642976
:1058100057E0A516B10408F444C060E270E080E0EF
:1058200090E00E946429A81AB90AF2CF0E942DBF05
:10583000C82E809003179090041780910305882349
:1058400071F2FE0133968AE0DF011D928A95E9F735
:105850008FEF96E19A83898304E715E29E012F5F1B
:105860003F4F42E951E212C0FE0133968AE0DF0168
:105870001D928A95E9F78FEF96E19A83898304E771
:1058800015E29E012F5F3F4F4FE851E2B701C4017F
:105890000F94B229B4018FEF96E10F9408411F8154
:1058A0009FCF4091DA08212F30E0A6E0CA9EC001C8
:1058B00011242E5F3F4F281739070CF49C0180E814
:1058C000821B8093361740933717C701DD20A9F05C
:1058D0000E94652A2C960FB6F894DEBF0FBECDBF8E
:1058E000DF91CF911F910F91FF90EF90DF90CF90BC
:1058F000BF90AF909F908F9008950E943F2BEACF6A
:10590000EBEFF6E183AF64AFCA010C943F2B2F920B
:105910003F924F925F926F927F928F929F92AF923F
:10592000BF92CF92DF92EF92FF920F931F93CF938C
:10593000DF93D62FC72FFC0180809180A280B38097
:10594000C501B40120E831E541E050E00F945B5C13
:10595000C9016DE671E00F94D85C6B017C01C50153
:10596000B40120E13EE040E050E00F945B5CCA01EE
:10597000B90128E130E040E050E00F945B5C362E46
:10598000272E062F172F8CE3482E512C612C712CBB
:10599000C501B401A30192010F945B5CB62EA72E42
:1059A000CA01B901A30192010F945B5CCB01C11440
:1059B000D10479F1AF92BF927F936F932F923F9270
:1059C000FF92EF92DF92CF9283E495E19F938F93C2
:1059D000CF93DF930F94AE558DB79EB70E960FB64B
:1059E000F8949EBF0FBE8DBF8D2F9C2FDF91CF915E
:1059F0001F910F91FF90EF90DF90CF90BF90AF90ED
:105A00009F908F907F906F905F904F903F902F90DE
:105A10000895E114F104C9F0AF92BF927F936F93A0
:105A20002F923F92FF92EF9283E395E19F938F93A2
:105A3000CF93DF930F94AE55EDB7FEB73C960FB6FC
:105A4000F894FEBF0FBEEDBFCFCF012BB9F0AF92E0
:105A5000BF927F936F932F923F9287E295E19F933E
:105A60008F93CF93DF930F94AE558DB79EB70A9661
:105A70000FB6F8949EBF0FBE8DBFB6CF892BA9F08D
:105A8000AF92BF927F936F938FE195E19F938F9336
:105A9000CF93DF930F94AE55EDB7FEB738960FB6A0
:105AA000F894FEBF0FBEEDBF9FCFAF92BF928BE1C8
:105AB00095E19F938F93CF93DF930F94AE550F9003
:105AC0000F900F900F900F900F908ECF8F929F920C
:105AD000AF92BF92CF92DF92EF92FF920F931F93FC
:105AE000CF93DF93109200051092FF042FE32093D1
:105AF000FE041092FD041092FC041092FB0410921C
:105B0000F7041092F8041092F9041092FA049C0120
:105B1000F90190812F5F3F4F9032D1F39E34C9F449
:105B2000818190ED980F9A3020F08D3211F08B32F8
:105B300081F432969F012F5F3F4F808180538A30DE
:105B400008F47BC09F012F5F3F4F8081803209F4B2
:105B500076C0F093FF08E093FE088F010F5F1F4FA0
:105B6000C0816AE270E0C8010F945E60009731F076
:105B7000FC01319780818032E1F31182CD3429F02C
:105B8000C43519F0C73409F04BC0F80180810F5FAC
:105B90001F4F8032D1F380538A3008F041C0C09348
:105BA000FE0430E020E04AE0DF011196429FC00190
:105BB000439F900D11249C01205331098081280FAF
:105BC000311D87FD3A95818190ED980F9A30C8F18B
:105BD0003093FD042093FC048E3261F4329690E001
:105BE0004AE0DF0131968C9150ED580F5A3058F150
:105BF0009093FB04CD01DC0101964C914032D9F326
:105C0000CD3489F52E31310539F018F527313105BC
:105C100019F02C31310539F5B0930005A093FF043C
:105C2000DF91CF911F910F91FF90EF90DF90CF9078
:105C3000BF90AF909F908F900895F9017BCFF901AD
:105C400081CFFD01B1CF949F800D112490ED980F6D
:105C5000C8CF2537310538F027373105E8F2203A2B
:105C600083E03807C9F2D091FE0840E050E0BA0165
:105C700010E000E0C12CD12C7601C394FD013196D7
:105C80008C91882309F47FC08132E1F4CD34D1F4C2
:105C900020323105B9F44093F7045093F80460932F
:105CA000F9047093FA04F0930005E093FF0463E2B3
:105CB00070E0CF010F945E60009709F4B1CFFC0152
:105CC0001082AECF81548A3108F058C0DF019D9117
:105CD000903291F0A0EDA90FAA30E8F09E3271F455
:105CE000918190539A30B8F00115110519F48F0184
:105CF0000150110990E013C0FD01E8CF9D3211F071
:105D00009B3291F79181A0EDA90FAA3020F09E322D
:105D100059F79281E6CF9E2F9D1B309759F3A82FFC
:105D2000B0E04601570104C0880C991CAA1CBB1C9A
:105D30008A95D2F7482959296A297B29A352BB4F52
:105D40009C9380818154DF018A3108F497CFDF0171
:105D50008191882309F492CF90ED980F9A30B8F38F
:105D600093ED980F923098F38B3289F3CD01019621
:105D7000EC91E03209F082CFDC01F8CF011511057A
:105D800001F78D01DECF109300050093FF044093CF
:105D9000F7045093F8046093F9047093FA0440CF29
:105DA0009B01AC01485F5F4FBC016C5F7F4F0C945F
:105DB000AD260F931F93CF93DF9300D000D01F9297
:105DC0001F92CDB7DEB7FC018B0183A5811112C0F4
:105DD00081E083A784819581A681B781B0588983AA
:105DE0009A83AB83BC83BE016F5F7F4F80EE98E0E8
:105DF0000E94D02E1D821E821F82188620E030E075
:105E000040E05FE360915111709152118091531104
:105E1000909154110F94095D69837A838B839C83DD
:105E20009E012B5F3F4FAE014F5F5F4F6DE471E10D
:105E300089E491E10E94AD261D821E821F82188690
:105E400020E030E040E05FE3F80160857185828505
:105E500093850F94095D69837A838B839C83B80152
:105E60006C5F7F4F9E012B5F3F4FAE014F5F5F4FD7
:105E7000C8010E94AD2628960FB6F894DEBF0FBE6B
:105E8000CDBFDF91CF911F910F9108952F923F9237
:105E90004F925F926F927F928F929F92AF92BF923A
:105EA000CF92DF92EF92FF920F931F93CF93DF93E6
:105EB000CDB7DEB7A2970FB6F894DEBF0FBECDBF49
:105EC0008C011B015E834D834090491150904A1113
:105ED00060904B1170904C1180904D1190904E112C
:105EE000A0904F11B0905011DB018D919D910D90BC
:105EF000BC91A02D8F87988BA98BBA8B9C01AD018B
:105F0000C301B2010F94085D6B017C01D1011496AD
:105F10008D919D910D90BC91A02D8B8B9C8BAD8B09
:105F2000BE8B9C01AD01C501B4010F94085D6F8B60
:105F3000788F898F9A8FAD81BE818D919D910D90C3
:105F4000BC91A02D8F839887A987BA879C01AD014A
:105F5000C301B2010F94085D6B8F7C8F8D8F9E8F74
:105F6000AD81BE8114968D919D910D90BC91A02D17
:105F70008B879C87AD87BE879C01AD01C501B401AD
:105F80000F94085D6F8F78A389A39AA3A701960148
:105F9000C701B6010F947D566B017C012F89388DA6
:105FA000498D5A8DCA01B9010F947D569B01AC01F0
:105FB000C701B6010F94095D4B015C012F8538893B
:105FC00049895A896F81788589859A850F94085DFA
:105FD0002B013C012B893C894D895E896B857C8531
:105FE0008D859E850F94085D6B017C01A301920154
:105FF000C301B2010F947D562B013C01A70196010C
:10600000C701B6010F947D569B01AC01C301B201DB
:106010000F94095D0F94B75F6B017C012B8D3C8D54
:106020004D8D5E8DCA01B9010F947D562B013C0147
:106030002F8D38A149A15AA1CA01B9010F947D56EB
:106040009B01AC01C301B2010F94095D9B01AC013E
:10605000C501B4010F94695F1816B4F520E030E073
:10606000A901C701B6010F94695F87FF2AC0C70164
:10607000B601905820E030E040EA50E40F94695FA8
:10608000181614F5A1016D817E81C8010E94462F6A
:10609000A2960FB6F894DEBF0FBECDBFDF91CF91B1
:1060A0001F910F91FF90EF90DF90CF90BF90AF9036
:1060B0009F908F907F906F905F904F903F902F9028
:1060C0000895C701B601D6CF20E030E040E050E4AB
:1060D000C501B4010F94695F181624F4B101C80119
:1060E0000E94D92E19821A821B821C82BE016F5F08
:1060F0007F4FC1010E94D02E2DEC3CEC4CEC5CE3B8
:10610000C701B6010F947D569B01AC01F801608177
:106110007181828193810F947D5669837A838B8309
:106120009C83C8010F94E331BE016F5F7F4F8D8167
:106130009E810E94D02EACCF4F925F926F927F9241
:106140009F92AF92BF92CF92DF92EF92FF920F9306
:106150001F93CF93DF93CDB7DEB768970FB6F89450
:10616000DEBF0FBECDBFFB019080342F390D38301C
:1061700008F026C1E180022F0E0D083008F020C182
:10618000EE2DF0E0E654FB4F4080512C712C612C39
:10619000092C04C076946794579447940A94D2F7D4
:1061A00040FE0EC110E0F801E654FB4F4080512C38
:1061B000712C612CC32ED12C04C076946794579413
:1061C00047943A95D2F740FEFBC0F22E642F5C0153
:1061D000660F770B072E000C880B990B0F941E5639
:1061E0002B013C01892D94E08902F0011124E65A2B
:1061F000F84EA301920160817181828193810F9495
:10620000095D6D877E878F87988BF601EE0FFF1FE4
:10621000EE0FFF1FE65AF84EA301920160817181D3
:10622000828193810F94085D69837A838B839C8339
:106230006F2D660F770B072E000C880B990B0F94B0
:106240001E562B013C018E2D94E08902F001112491
:10625000E65CF84EA3019201608171818281938195
:106260000F94095D698B7A8B8B8B9C8B000F111FB0
:10627000000F111FF801E65CF84EA3019201608146
:106280007181828193810F94085D6D837E838F83FA
:106290009887F50180859185A285B38589879A873E
:1062A000AB87BC878D8B9E8BAF8BB88F4FE851E04F
:1062B00061E070E0CE0141960E9497D84FE851E02E
:1062C00061E070E0CE0105960E9497D849E951E05F
:1062D00061E070E0CE010D960E9497D849E951E047
:1062E00061E070E0CE0101960E9497D8C988DA88F3
:1062F000EB88FC8827E137EB41ED58EBC701B6018D
:106300000F94695F87FD5CC023E030E048EC53E404
:10631000C701B6010F94175618160CF451C0CD845E
:10632000DE84EF84F88827E137EB41ED58EBC701B5
:10633000B6010F94695F87FD43C023E030E04DEC68
:1063400053E4C701B6010F9417561816CCF1CD804F
:10635000DE80EF80F88427E137EB41ED58EBC70191
:10636000B6010F94695F87FD2BC023E030E048EC55
:1063700053E4C701B6010F94175618160CF1C980E3
:10638000DA80EB80FC8027E137EB41ED58EBC70169
:10639000B6010F94695F87FD13C023E030E04DEC38
:1063A00053E4C701B6010F94175618164CF0AE010E
:1063B0004F5F5F4FBE01635F7F4FC5010E94462F55
:1063C00068960FB6F894DEBF0FBECDBFDF91CF91B8
:1063D0001F910F91FF90EF90DF90CF90BF90AF9003
:1063E0009F907F906F905F904F9008958C389105AB
:1063F00014F08CE890E090931E0980931D090C9492
:1064000096C90E94F32797FD0CC00E94F3276F3FA7
:1064100071058105910509F034F40E94F327862F58
:10642000089580E008958FEF08958091C6049091BB
:10643000C704892B41F00E94013291E0811101C013
:1064400090E0892F089591E0FCCF0E94F327CB01C3
:1064500008950F931F93CF938091C6049091C70422
:106460000097E9F0FC018F01C1912C2F2F7D81F065
:10647000C53411F0C536B9F7F801108270E060E05C
:106480000F94A651F801C083CF911F910F910895E9
:1064900070E060E0CF911F910F910D94A65160E0E4
:1064A00070E0CB01F1CF2FEB280F2A3108F047C065
:1064B000E22FF0E08091F7049091F804A091F904A4
:1064C000B091FA0404C0B695A795979587952A953B
:1064D000D2F780FD02C081700895E352FB4FE08146
:1064E000EE2341F18091FE089091FF08E80FF92F0B
:1064F000F11D808190ED980F9A3030F08E3251F47A
:10650000818180538A3098F4F093C704E093C604E5
:1065100081E008958D3211F08B3249F4818190ED44
:10652000980F9A3088F38E3211F48281EACFF0E02E
:10653000E0E0EACF1092C7041092C604E9CF80E0F1
:1065400008950E945332882341F081E02091C604CF
:106550003091C704232B09F480E00895CF93DF9393
:10656000EB010E94A132882319F00E94F327EB016E
:10657000CE01DF91CF910895CF92DF92EF92FF92FB
:106580006A017B010E94A132882331F0FF90EF90D5
:10659000DF90CF900C942932C701B601FF90EF90A5
:1065A000DF90CF9008954F925F926F927F928F927B
:1065B0009F92AF92BF92CF92DF92EF92FF921F9382
:1065C000CF93DF9300D01F92CDB7DEB719821A8226
:1065D0001B821C82CE0101964C0189E4C82E81E108
:1065E000D82E90EEE92E98E0F92E2BEFA22E29E07E
:1065F000B22E10E088E5810F0E94A132F401819350
:106600004F01882341F00E9429322B013C018091E7
:10661000FE10882359F0F60180819181A281B38117
:10662000F70180839183A283B38314C0812F0E94DA
:106630006622882309F4D0C0F6012081318142818D
:106640005381C301B2010F94095DF7016083718327
:10665000828393831F5FF4E0CF0ED11C84E0E80EA9
:10666000F11C94E0A90EB11C133021F685E40E94C0
:10667000A1328C83882309F4B9C00E9429326B01AE
:106680007C0183E00E946622882371F020915511DD
:10669000309156114091571150915811C701B601D0
:1066A0000F94095D6B017C01C092EC08D092ED085B
:1066B000E092EE08F092EF088091D605882359F118
:1066C0008091851782FF27C08C81882321F18981E1
:1066D000811103C08A818823F1F02DEC3CEC4CE45D
:1066E0005DE3609152097091530980915409909132
:1066F00055090F94095D9B01AC0160915111709196
:10670000521180915311909154110F94695F181692
:1067100014F40F94E14240E050E0BA0186E40E9494
:10672000BC3220E030E0A9010F94695F181684F4B0
:106730000E94293220E030E040E752E40F94035EEB
:1067400060937C0270937D0280937E0290937F021F
:106750008091FF1083FD2CC08091FE10811128C014
:1067600080915A08882321F12091551130915611BA
:1067700040915711509158116091EC087091ED08BB
:106780008091EE089091EF080F94085D20916708C2
:10679000309168084091690850916A080F94095D2A
:1067A00060936708709368088093690890936A08FB
:1067B0000F900F900F900F90DF91CF911F91FF904E
:1067C000EF90DF90CF90BF90AF909F908F907F9091
:1067D0006F905F904F900895F50120813181428143
:1067E0005381C301B2010F94085D2FCF80915511E1
:1067F00090915611A0915711B09158118093EC08C7
:106800009093ED08A093EE08B093EF0855CFCF9387
:10681000DF93EB010E94A132882321F0DF91CF9119
:106820000C942532CE01DF91CF910895CF93DF9361
:10683000C82FD62F0E94A132882321F0DF91CF915B
:106840000C9415328C2F0E945332811101C08D2F70
:10685000DF91CF910895E9E4F9E082EBDF011D9229
:106860008A95E9F708958091D605811104C00E94A8
:106870002B340D941D458091851782FD0D94E142C6
:10688000089580914909882361F09091FA0989134C
:1068900008C08091851783FF04C087E899E00D94B4
:1068A000284580E00895FC01238121110C9406D530
:1068B0000895CF92DF92EF92FF920F931F93CF93A1
:1068C00090912402913009F461C0662351F0109236
:1068D000A6041092A2041092A3041092A404109291
:1068E000A504C82F0F94E338C090A204D090A3044D
:1068F000E090A404F090A5049B01AC012C193D0983
:106900004E095F0969017A01F7FC40C02091A60495
:10691000C7FD15C04C2F0C2E000C550B4C5F5F4F64
:10692000E22F022E000CFF0B4E175F077CF144EFA5
:10693000C42EDD24D394E12CF12C2C1734F438EE42
:10694000C32E33E0D32EE12CF12CC60ED71EE81E49
:10695000F91EC092A204D092A304E092A404F09283
:10696000A504022F017010E084E2809FB001819F96
:10697000700D701B112460597C4F82E390E00E94DF
:106980005E808091A6048F5F8093A604CF911F91B3
:106990000F91FF90EF90DF90CF9008950F931F938A
:1069A00001E010E020E030E0082E04C0000F111FCD
:1069B000221F331F0A94D2F740910B0550910C050A
:1069C00060910D0570910E05402B512B622B732B9E
:1069D00040930B0550930C0560930D0570930E05C5
:1069E00090912302891303C081E08093FE101F91D0
:1069F0000F9108951092D7061092D8061092D906DA
:106A00001092DA06E7EDF5E080E091E0DF019C010D
:106A10001D9221503040E1F7089590914811981748
:106A2000B1F00E946ADF80914811882341F089E427
:106A300091E10E948DDF109248110C947AF581E06B
:106A40008093481189E491E10E94BFDEF6CF08955A
:106A50004F925F926F927F928F929F92AF92BF926E
:106A6000CF92DF92EF92FF921F93CF93DF93EC01CF
:106A7000162F209113093091140940911509509156
:106A80001609688179818A819B810F941756882322
:106A900009F4AEC0B090481180E00E940D35C88066
:106AA000D980EA80FB8020E030E0A901C701B6016F
:106AB0000F94695F18161CF0C12CD12C7601C0927E
:106AC0001309D0921409E0921509F09216092DEBE2
:106AD00037E346E855EBC701B6010F94695F87FDC0
:106AE0000BC02DEB37E346E855E3C701B6010F9421
:106AF000175618160CF078C0A701960160E070E0F8
:106B000080E89FE30F94035E6093BA057093BB0522
:106B10008093BC059093BD0580EF9FEFA9E7B4EC8F
:106B20008093BE059093BF05A093C005B093C105A7
:106B3000BB2009F45DC04090491150904A1160900B
:106B40004B1170904C1180904D1190904E11A0906F
:106B50004F11B0905011C0905111D0905211E0904F
:106B60005311F090541181E00E940D35112309F466
:106B70003FC02091491130914A1140914B115091E1
:106B80004C11C301B2010F94175681111CC0209102
:106B90004D1130914E1140914F1150915011C5013E
:106BA000B4010F94175681110EC0209151113091EC
:106BB00052114091531150915411C701B6010F94D5
:106BC00017568823A9F0DF91CF911F91FF90EF9086
:106BD000DF90CF90BF90AF909F908F907F906F90FD
:106BE0005F904F900C9422FE60E070E0CB018CCF60
:106BF000DF91CF911F91FF90EF90DF90CF90BF90EA
:106C0000AF909F908F907F906F905F904F9008957E
:106C1000EF92FF920F931F93CF93DF9307ED15E051
:106C2000C8E07801D8E0F70161917191819191916B
:106C30007F0120E030E0A9010F94175681110EC0AA
:106C4000D15089F7C150005E1F4FC111EACFDF91CB
:106C5000CF911F910F91FF90EF90089581E0F7CFB2
:106C6000EFE6F0E080818260808308958091F408EF
:106C70009091F508892B79F48091F4089091F508AA
:106C8000892B49F42091F4083091F50881E0232BF9
:106C900019F480E0089581E00895CF92DF92EF9299
:106CA000FF926B017C0183E3C816D104E104F10477
:106CB00070F082E3C81AD108E108F10862E370E0DD
:106CC00080E090E00F94B0380E947CF5ECCFC701D3
:106CD000B6010F94B038FF90EF90DF90CF900C94F6
:106CE0007CF58091DA0781110AC080911109813009
:106CF00041F08091851782FB882780F9089580E014
:106D0000089581E008955F9A80916E088E7F809348
:106D10006E088A9A80916E088D7F80936E088091AC
:106D20000801809581708093060180916E088B7FA9
:106D300080936E080C9493229091851793FB88277B
:106D400080F993FF06C081E09091ED18911101C088
:106D500080E008958091DA07811110C080911109B7
:106D6000823061F00E949C36882349F0809185171B
:106D700082FB882780F991E08927089581E00895B2
:106D80000E94AA3681110DC010920B0510920C05BD
:106D900010920D0510920E0510920F058FEF0E94B4
:106DA00034260D947901E9E3FAE010821182089506
:106DB00081E008958F929F92AF92BF92CF92DF921F
:106DC000EF92FF920F93CF93DF931F92CDB7DEB771
:106DD0005C017B0149016B01C40ED51EF501808168
:106DE00091810F94355C8983002311F0F701808332
:106DF000BE016F5F7F4FC4010F94D828F5018081D9
:106E00009181019691838083FFEFEF1AFF0AEC14C2
:106E1000FD0421F780E00F90DF91CF910F91FF905B
:106E2000EF90DF90CF90BF90AF909F908F9008959C
:106E30009091C00095FFFCCF8093C6000895CF933A
:106E4000DF93EC018991882319F00E941837FACF5B
:106E50008DE00E9418378AE0DF91CF910C941837AB
:106E6000CF92DF92EF92FF92CF936B017C01C42F00
:106E70004A3069F4F7FE0BC0F094E094D094C094CB
:106E8000C11CD11CE11CF11C8DE20E9418374C2F53
:106E9000C701B601CF91FF90EF90DF90CF900D9496
:106EA0004342CF93DF93EC01FE0184912196882326
:106EB00019F00E941837F8CFDF91CF9108950F9302
:106EC0001F93CF938C01C62F85E892E10E94513722
:106ED000C8010E9451378AE30E94183780E38C0F63
:106EE0000E9418378AE0CF911F910F910C941837A8
:106EF00088E094E10E94513760E088EF93E10E94BE
:106F00005F3760E083EE93E10E945F3761E08CEDD4
:106F100093E10E945F3761E081ED93E10E945F376A
:106F200061E081EC93E10E945F3760E088EB93E1E0
:106F30000E945F3761E08EEA93E10E945F3760E074
:106F400084EA93E10E945F3761E08DE993E10E945A
:106F50005F3760E085E993E10E945F3761E087E891
:106F600093E10E945F3761E089E793E10E945F3718
:106F700060E08AE693E10E945F3760E08CE593E190
:106F80000E945F3760E086E493E10E945F3761E032
:106F900085E393E10E945F3761E086E293E10E941E
:106FA0005F3761E08FE193E10E945F3760E088E145
:106FB00093E10E945F3761E08FE093E10E945F37C9
:106FC00061E08AEF92E10E945F3761E08CEE92E12E
:106FD0000E945F3761E089ED92E10E945F3760E0D7
:106FE0008CEC92E10E945F3761E087EC92E10E94B5
:106FF0005F3761E08AEB92E10E945F3760E086EAEA
:1070000092E10E945F3760E083E992E10E945F377E
:1070100060E089E897E10E946322682F61708AE846
:1070200092E10C945F378091F704827149F480916A
:10703000F9048C7829F48091FA04837009F475C0FE
:1070400082E40E945332882351F00E94D227609339
:10705000101170931111809312119093131183E505
:107060000E945332882351F00E94293260934011CC
:1070700070934111809342119093431184E50E94D3
:107080005332882351F00E94293260934411709347
:107090004511809346119093471188E50E94533221
:1070A000882351F00E9429326093210A7093220AAA
:1070B0008093230A9093240A89E50E9453328823FF
:1070C00051F00E9429326093250A7093260A80931A
:1070D000270A9093280A8AE50E9453328823B1F048
:1070E0000E9429326093290A70932A0A80932B0AFE
:1070F00090932C0A2DEC3CEC4CEC5DE30F9417566E
:10710000181624F083E69EE00E94513785E40E9421
:107110005332882351F00E94293260932D0A7093D4
:107120002E0A80932F0A9093300A08950E941837F0
:1071300085E29DE00C9451370F931F93CF938C0100
:10714000C62F8CE999E00E945137C8010E9451373F
:10715000CC2331F08AE0CF911F910F910C94183716
:10716000CF911F910F9108950F931F93CF938C018F
:10717000C62F60E08CEA99E00E949C38C8010E940A
:107180005137CC2331F08AE0CF911F910F910C94AD
:107190001837CF911F910F91089561E084EB99E02A
:1071A0000C94B438EF92FF920F931F93CF937C010E
:1071B0008B01C42F60E08CEA99E00E949C38C701E3
:1071C0000E94513780E20E941837C8010E9451374F
:1071D000CC2319F08C2F0E9418378AE0CF911F9191
:1071E0000F91FF90EF900C941837DF92EF92FF927F
:1071F0000F931F93CF93DF93D82E7B018A01E90170
:107200000E94CD38D092F80840E0B7018DED90E4AF
:107210000E94D2380115110531F040E0B80186ED29
:1072200090E40E94D238209731F040E0BE0186ED14
:1072300090E40E94D23861E081ED90E4DF91CF913B
:107240001F910F91FF90EF90DF900C94B43861E0A4
:1072500086EA99E00C949C38AF92BF92CF92DF926D
:10726000EF92FF920F931F93CF93DF9381E799E003
:107270000E9451376091D7067091D8068091D90647
:107280009091DA0645E00F94BF0A8EE599E00E94DE
:107290005137C0E0D9E0D15021F080E20E94183788
:1072A000FACF8C2F0F94AA42CF5FC83099F78AE0AB
:1072B0000E94183707ED15E0C0E080E20E94183701
:1072C0008C2F0F94AA425801D8E080E20E94183710
:1072D000F501C080D180E280F380A7019601C7014B
:1072E000B6010F94FB5F81112CC020E030E0A901B2
:1072F000C701B6010F94695F87FD03C08BE20E944E
:10730000183745E0C701B6010F94BF0AD15080E29B
:10731000A80EB11CD111D9CF8AE00E941837CF5FD7
:107320000C5F1F4FC83049F68AE0DF91CF911F9163
:107330000F91FF90EF90DF90CF90BF90AF900C94A3
:107340001837F12C80E20E941837F3948DE3F8E0AF
:10735000FF12F9CFDBCF811107C085E99EE00E94C3
:1073600051378AE00C94183789E99EE0F8CFCF9323
:10737000DF93EB010E945137CE01DF91CF910D9445
:10738000B142CF93C62F0E9451378C2FCF910D94CD
:10739000AA42CF92DF92EF92FF926A017B010E9494
:1073A000513742E0C701B601FF90EF90DF90CF90D8
:1073B0000D94BF0ACF92DF92EF92FF926A017B0198
:1073C0000E9451374AE0C701B601FF90EF90DF906D
:1073D000CF900C9430372F923F924F925F926F92E2
:1073E0007F928F929F92AF92BF92CF92DF92EF9255
:1073F000FF920F931F93CF93DF93CDB7DEB7C654A1
:10740000D1090FB6F894DEBF0FBECDBF70E060E0CB
:1074100085E40E940734182F8F3F09F483C0882326
:10742000E9F081EC96E1CA5BDF4F0FB6F894DEBF5E
:107430000FBECDBFDF91CF911F910F91FF90EF90C5
:10744000DF90CF90BF90AF909F908F907F906F9084
:107450005F904F903F902F900C94513724EB30E089
:107460003A83298383E50E94A132882321F00E9478
:1074700025329A83898365E070E083E40E940734B3
:107480008AA760E085E50E94163425968FAF259780
:1074900060E084EB96E10E94A6B5A981BA81BD01A6
:1074A000BB0F880B990B0F941E566D837E838F83C1
:1074B00027969FAF27970F94E338688B798B8A8B39
:1074C0009B8B1F3F09F045C420E030E04CE053E4C3
:1074D0006D817E818F8127969FAD27970F94695F7D
:1074E00018160CF0AAC189E896E10E945137CA5BD0
:1074F000DF4F0FB6F894DEBF0FBECDBFDF91CF9147
:107500001F910F91FF90EF90DF90CF90BF90AF90C1
:107510009F908F907F906F905F904F903F902F90B3
:107520000D94184646E450E05A8349839BCF1FAE22
:10753000AFC12496EEADFFAD2497808383C2FBEEEE
:107540004F2E512C612C712C04C384E190E0A0E0FB
:10755000B0E08C8B9D8BAE8BBF8BE4E14E2E512C1B
:10756000612C712C04C34C8A5D8A6E8A7F8AFFC2AB
:107570002496EEADFFAD24978083D4C389819A8190
:10758000AB81BC8129A93AA94BA95CA9821B930BA9
:10759000A40BB50BB7FD59C08FAD0F94630B8AE0F8
:1075A0000E94183789819A81AB81BC818053984FA2
:1075B000AF4FBF4F89AB9AABABABBCAB9DA99111A1
:1075C00077C02EA93FA948AD59ADB101802F2696AD
:1075D0009FAD26970F94695F18160CF053C020E0FA
:1075E00030E040E050E4B101802F26969FAD269711
:1075F0000F94095D6EAB7FAB88AF99AF2CA53DA50D
:107600004EA55FA589819A81AB81BC81280F391F66
:107610004A1F5B1F2AAF3BAF4CAF5DAF20E030E0AD
:1076200040EC50E46D817E818F8127969FAD279736
:107630000F94085D9101402F26965FAD26970F9419
:107640001756881F8827881F8DAB88899989AA8932
:10765000BB89C816D906EA06FB0610F4D701C60195
:1076600029813A814B815C81281B390B4A0B5B0BCA
:10767000DA01C90181389F44A241B105A8F185ED25
:1076800095E10EC289819A81AB81BC812AAD3BAD67
:107690004CAD5DAD821B930BA40BB50B4EE556E3D1
:1076A0006DE676E3B7FDD1CF812F0E94D9D8CDCF3B
:1076B00020E030E040EF51E46D817E818F8127969C
:1076C0009FAD27970F94085D9B01AC01B101802FFE
:1076D00026969FAD26970F94175687FFB6CF42E5A3
:1076E00057E362E677E3E0CF4AA55BA5888D998DE5
:1076F000481759070CF09EC003970CF49BC088E70D
:1077000095E10E9451371F3F09F076C0A8E6B5E128
:10771000BA83A98387E595E10E94513789819A81CF
:107720000E945137488559856A857B8584E795E1B4
:107730000E94C9398AE00E94183787E595E10E94C6
:10774000513789819A810E94513749A15AA16BA171
:107750007CA180E795E10E94C9398AE00E94183730
:1077600087E595E10E94513789819A810E945137BE
:10777000B501A4018CE695E10E94C9398AE00E9416
:1077800018372596FFAD2597FF2391F12CEA35ECAC
:1077900047E25EE369A17AA18BA19CA10F947D567B
:1077A0006B017C012CEA35EC47E25EE3C501B401D4
:1077B0000F94035E288539854A855B851F3F09F54F
:1077C00020932009309321094093220950932309E3
:1077D000C0922409D0922509E0922609F092270947
:1077E000609328097093290980932A0990932B09A3
:1077F00081E0809365027BCEEBE1F0E4FA83E983DC
:1078000089CF209384163093851640938616509323
:107810008716C0928816D0928916E0928A16F09246
:107820008B1660938C1670938D1680938E169093A2
:107830008F16DECF0E94B2B980C085E796E10E9424
:1078400051370E94CCD78FE780931F0928E730E09B
:10785000A8EEB3E00F94AF5C6CA77DA78EA79FA79F
:10786000288939894A895B89260F371F481F591F84
:107870002AAF3BAF4CAF5DAF1092650281E08093C1
:10788000740232E0310F3EAF323008F450CE1FAFF9
:10789000C888D988EA88FB88C9AADAAAEBAAFCAA10
:1078A000812C912C540189A29AA2ABA2BCA28886F9
:1078B0009986AA86BB868FE790E0A0E0B0E08C8B2B
:1078C0009D8BAE8BBF8B1C8690E49A8FACE1AB8F07
:1078D000B6E4BC8F1D8E1E8E1F8E18A23FE7432E6E
:1078E000512C612C712C1DAA8EAA9FAAA8AEB9AEEC
:1078F0001EA21FA218A619A6E1E0EDA3198E188EEC
:10790000212C312C00E026961FAE2697F5E11F02B0
:10791000C00111249C012558394E22963FAF2EAF4D
:107920002297285F3F4F24963FAF2EAF24974AA55A
:10793000042E000C550B5BA74AA780917402882384
:1079400009F4B0C00F94E33869837A838B839C83F6
:107950005091F40658AB552309F48BC00E947FD890
:1079600060911B0970911C091F3F39F02296AEAD42
:10797000BFAD229714966D917C91072E000C880B59
:10798000990B0F941E561B01082F26969FAF269722
:107990002D8D3E8D4F8D58A126969FAD26970F9425
:1079A000695F18163CF42D8E3E8E0F8F2696BFAD64
:1079B0002697B8A32C853A8D4B8D5C8DB101802F15
:1079C00026969FAD26970F94175687FF07C02C86E3
:1079D0003A8E0B8F2696EFAD2697EC8FFDA1910185
:1079E000402F26965FAD26976D817E818F812796E9
:1079F0009FAD2797FF2309F45AC00F94175687FFAE
:107A000038C049815A816B817C814C195D096E09AE
:107A10007F09DB01CA0188589341A109B109B7FD6B
:107A200028C08C899D89AE89BF8984199509A609CA
:107A3000B709B595A795979587951F3F09F079CD1B
:107A400080931F094EA35FA368A779A7FD81FD8FCF
:107A50002E812E8F3F813F8F27964FAD279748A3CA
:107A600089819A81AB81BC81888B998BAA8BBB8BD6
:107A70001DA220E030E040EF51E46D817E818F81D6
:107A800027969FAD27970F94095D9101402F269669
:107A90005FAD26970F94175687FF70CD83EF95E162
:107AA0000E945137109274020E94CCD7A1CE0F943D
:107AB000695F1816F4F689819A81AB81BC812889A7
:107AC00039894A895B89821B930BA40BB50BAC01E6
:107AD000BD01485853416109710977FDCACF488DEE
:107AE000598D452B09F40DC1CEA0DFA0E8A4F9A45F
:107AF000C80ED91EEA1EFB1E2EA13FA148A559A5FE
:107B0000281B390B4A0B5B0BC301B2010F944B5C72
:107B1000A70196010F947D5C4C885D886E887F88F4
:107B2000420E531E641E751E54E145165104610435
:107B300071040CF40ACD8CEE4816510461047104F2
:107B40000CF0FDCC90E849165104610471040CF46A
:107B50000ACD4C8A5D8A6E8A7F8A2EEF30E040E043
:107B600050E0241935094609570929013A014C8981
:107B70005D896E897F898DE696E10E94DA39B301CD
:107B8000A20188E696E10E94DA394C855A8D6B8D08
:107B90007C8D81E696E10E94C9394D8D5E8D6F8D99
:107BA00078A18AE596E10E94C939A88DB98D13970D
:107BB0000CF4A7C0C301B2010F941E5620E030E0C0
:107BC00040E850E40F947D564B015C012C853A8DC2
:107BD0004B8D5C8D6D8D7E8D8F8D98A10F94085D82
:107BE0002BED3FE049E450E40F947D5620E030E077
:107BF00040E05FE30F947D569B01AC01C501B401E9
:107C00000F94035E6C877D878E879F87C701B601BF
:107C10000F941E562FE632E143E85AE30F947D5647
:107C20006B017C011E3F59F02AE939E949E15FE324
:107C3000812C912CA12C6EE3B62E1F3F59F42DEC14
:107C40003CEC4CE45EE37BEA872E7AEA972EA92C83
:107C50007EE3B72E6C857D858E859F850F947D563E
:107C6000688779878A879B879B01AC010F94095DA0
:107C7000A70196010F94035E69A37AA38BA39CA32B
:107C8000288539854A855B85C701B6010F947D56E5
:107C9000A50194010F947D564B015C014C855D85D7
:107CA0006E857F8584E596E10E94C939B701A601FA
:107CB0008EE496E10E94C9398AE00E941837BEAD71
:107CC0008FE396E1B23010F080E396E10E945137E5
:107CD000488559856A857B858AE296E10E94C93983
:107CE00049A15AA16BA17CA184E296E10E94C93905
:107CF000B501A4018EE196E10E94C9398AE00E9493
:107D000018378C899D89AE89BF89840D951DA61D64
:107D1000B71DB595A795979587951F3F09F028CC76
:107D200080931F09288D398D2F5F3F4F398F288F02
:107D30003D813C874E814A8F5F815B8F27968FAD57
:107D400027978C8FC980DA80EB80FC8098A99DA34F
:107D500090CEE12E012E000CFF08F70183E0EE0F1C
:107D6000FF1F8A95E1F7E459FD4F668177816F50D7
:107D70007109072E000C880B990B0F941E569B015E
:107D8000AC016D817E818F8127969FAD27970F94DF
:107D9000695F18160CF4A7CB85E796E10E9451376E
:107DA0000E94CCD785E18E9DF0018F9DF00D1124AE
:107DB000E558F94E8FE7808722E330E049CDCF9335
:107DC000DF93EB010E945137CE01DF91CF910D94EB
:107DD0008F2A2F923F924F925F926F927F928F9253
:107DE0009F92AF92BF92CF92DF92EF92FF920F934A
:107DF0001F93CF93DF93CDB7DEB7C058D1090FB62D
:107E0000F894DEBF0FBECDBF80EB9CE00E945137DF
:107E10000F943A4681118FC084E50E94A1328823D5
:107E200029F00E94253281110E9482D780E090E0E3
:107E3000A0E8BFE389839A83AB83BC838D839E8351
:107E4000AF83B8878DEC9CECACE4BEE389879A875E
:107E5000AB87BC8780E090E0A0E2B1E48D879E878D
:107E6000AF87B88B8CE390E09A8B898B8DEC90E098
:107E70009C8B8B8B8DEC9CECACECBEE38D8B9E8B4A
:107E8000AF8BB88F80E090E0A0EEBFE3898F9A8F30
:107E9000AB8FBC8F1BA61CA64AE959E969E97EE3B2
:107EA0008FE40E94BC326D8F7E8F8F8F98A360E02D
:107EB00083E40E94163489A360E08BE40E941634A8
:107EC0008AA389E40E94A13210E0F12CE12C8823DE
:107ED000C1F00E94013290E01816190614F481E0F6
:107EE00090E011E0180F212F2150330BC90126E03B
:107EF000289FF001299FF00D1124EC54F74FE280E8
:107F0000F38082E40E94A132882319F00E94253276
:107F10007C01E114F10459F1C70188978536910578
:107F200020F16CE870E082E89CE00E94DF3E8DE783
:107F30009CE00E945137C058DF4F0FB6F894DEBF67
:107F40000FBECDBFDF91CF911F910F91FF90EF90AA
:107F5000DF90CF90BF90AF909F908F907F906F9069
:107F60005F904F903F902F900895FA8AE98A8CE4B1
:107F70000E94A1328823E1F00E9429326B017C012A
:107F8000C986DA86EB86FC8620E030E0A9010F94F2
:107F9000695F87FD0AC020E030E040E050E4C7019F
:107FA000B6010F94175618161CF485E59CE0C1CF56
:107FB00081E50E945332882331F18091C60490916B
:107FC000C704892BE9F00E9429326B017C01CD8224
:107FD000DE82EF82F8862DEC3CEC4CE45DE30F94FE
:107FE000695F87FD0AC020E030E040E751E4C70147
:107FF000B6010F941756181634F484E29CE099CF1A
:1080000089EF9BE096CF83E50E94A1328823E9F0B7
:108010000E9429326B017C01CD8ADE8AEF8AF88EBC
:108020002DEC3CEC4CEC5DE30F94695F87FD0AC0DE
:1080300020E030E040E050E4C701B6010F9417564D
:1080400018161CF482ED9BE074CF80E50E94533239
:10805000882341F08091C6049091C704892B29F5AB
:108060008FEF8BA786E40E94A132882309F43DC0DC
:108070000E9429326B017C01C98EDA8EEB8EFC8E58
:1080800020E030E040E85FE30F94695F87FD0AC0BD
:1080900020E030E040E850E4C701B6010F941756E5
:1080A00018161CF581E89BE044CF8BA58F5F8BA74A
:1080B0000E9429326B017C01CD86DE86EF86F88A2C
:1080C00020E030E0A9010F94695F87FD0BC020E03C
:1080D00030E048EC51E4C701B6010F94175618166A
:1080E0000CF0C0CF8AEA9BE024CFC98CDA8CEB8CF1
:1080F000FC8C8D889E88AF88B88CA7019601C7013B
:10810000B6010F947D569B01AC0160E070E084E401
:1081100090E40F94035E29813A814B815C810F9436
:108120007D562B013C01A5019401C501B4010F94BA
:108130007D56A70196010F947D562CEE31E548EB54
:108140005DE30F94035E9B01AC01C301B2010F9488
:108150007D5669837A838B839C83112309F1412F98
:108160004150550B26E0249FF001259FF00D11246E
:10817000EC54F74F0081118188E40E94A1328823DA
:1081800019F00E9425328C010115110571F0C8010A
:10819000855A91098838910530F083E59BE0C9CE76
:1081A00010E000E0E9CF1C8B0B8B85E50E94533279
:1081B0008823C9F00F94E338611571058105910595
:1081C00011F00F949D518091C6049091C704892BA2
:1081D000C9F00E9429326093C2047093C304809353
:1081E000C4049093C50461E470E082E50E94073402
:1081F000E5969FAF8EAFE5971816190644F08FE10C
:108200009BE097CE60E070E088E492E4E4CF89E5FB
:108210000E94A132882309F40AC10E9429322091C8
:10822000FF093091000A4091010A5091020A0F940F
:10823000085D4B015C0188E50E94A132882309F4A6
:10824000FFC00E9429322091FB093091FC09409126
:10825000FD095091FE090F94085D6B017C01CBA2D2
:10826000DCA2EDA2FEA28FA298A6A9A6BAA627E13B
:1082700037EB41ED58EBC501B4010F94695F87FD01
:10828000E8C023E030E048EC53E4C501B4010F94AA
:10829000175618160CF4DDC027E137EB41ED58EB0B
:1082A000C701B6010F94695F87FDD3C023E030E0BA
:1082B0004DEC53E4C701B6010F94175618160CF491
:1082C000C8C084E40E94533211E081270E940D351A
:1082D00080E090E0A0EAB0E48DA79EA7AFA7B8AB7E
:1082E000CE018D960F94883150913009EC965FAF96
:1082F000EC97109230090E9419C782EA9AE00E9416
:10830000513789899A894A970CF0A6C063E68FE7AE
:108310009AE00E94A6B50F941C398B899C890E9413
:10832000ECDE41E061E080E00F945B0D882309F40E
:10833000A6C00F9418460F941C3910925511109234
:108340005611109257111092581185E591E10E9433
:1083500072F11BA5112309F4F5C020E030E040E7DD
:1083600051E46091301170913111809132119091EE
:1083700033110F94035E21966CAF7DAF8EAF9FAF2C
:1083800021971F3F09F0F9C481E08093080563E657
:1083900087ED9AE00E94A6B568E873E182E090E07C
:1083A0000E945E8080E1E9E4F1E1A0EEB8E0019096
:1083B0000D928A95E1F7CE0101960F94E331C12C1D
:1083C000D12C760180910B0A82FDB1C068E873E17F
:1083D00082E090E00E945E8020E030E040E85EE3D2
:1083E0006091EC087091ED088091EE089091EF0893
:1083F0000F94095D6093EC087093ED088093EE088C
:108400009093EF0820E030E040E85EE3C701B6015A
:108410000F94095D6B017C0120E030E84BE354E4EC
:108420000F94695F87FD73C01092080528C0809083
:108430004D1190904E11A0904F11B0905011FBCE65
:10844000C0904911D0904A11E0904B11F0904C111E
:1084500006CF85EF9AE06DCD63E682E99AE00E944F
:10846000A6B50F941C391093080589899A890E9432
:10847000F63161E081E00F94D60B811147CF6FEFA9
:1084800089EE9AE00E94A6B58CA5811112C081E008
:108490008CA78D819E81AF81B885B0588DA79EA78E
:1084A000AFA7B8ABBE01635D7F4F80EE98E00E943E
:1084B000D02E80E090E0A0EAB0E48093E8089093AA
:1084C000E908A093EA08B093EB081DA61EA61FA614
:1084D00018AABE01635D7F4F80EE98E00E94D02E07
:1084E000EC965FADEC97509330090E9419C710923B
:1084F00008058AA181111FCD10921E0910921D0935
:108500000E9496C990E080E00E94ECDE14CDCE017E
:10851000CD960E946AFC80E1E9E4F1E1A0EEB8E0CA
:1085200001900D928A95E1F70E946ADF4BCF0E947D
:1085300071BC63E68AEC9AE00E94A6B50F941C39E0
:1085400010920805EAEBF4E088E0DF011D928A95BD
:10855000E9F780E1E9E4F1E1A0EEB8E001900D92E5
:108560008A95E1F789859A85AB85BC858093E80873
:108570009093E908A093EA08B093EB081DA61EA605
:108580001FA618AABE01635D7F4F80EE98E00E948F
:10859000D02EBE01635E7F4F80EE98E00E94D02E09
:1085A00081E08093080589A1882309F43CC42091C7
:1085B000491130914A1140914B1150914C11AC9698
:1085C0002CAF3DAF4EAF5FAFAC9780914D11909106
:1085D0004E11A0914F11B0915011E0968CAF9DAF0C
:1085E000AEAFBFAFE097AAE5B7E1A196BFAFAEAF20
:1085F000A197312C212CBFEF6C96BFAF6C97EFEF9A
:10860000A496EFAFA497FFEFE396FFAFE3972FE4B5
:10861000EA962FAFEA9733ECEB963FAFEB9707E480
:1086200081E090E0A0E0B0E0022C04C0880F991F28
:10863000AA1FBB1F0A94D2F7C458DF4F88839983BF
:10864000AA83BB83CC57D040AAEBB4E0E296BFAF7D
:10865000AEAFE297EAE3F7E1A396FFAFEEAFA397E1
:1086600010E0C058DF4F2882C058D040E296AEAD2F
:10867000BFADE2978D91E296BFAFAEAFE29790E0CB
:10868000B0E0A0E0C458DF4F288139814A815B8186
:10869000CC57D04082239323A423B523892B8A2B44
:1086A0008B2B09F0E5C0A196AEADBFADA197CD90E3
:1086B000DD90ED90FC90A396AEADBFADA3972D914C
:1086C0003D914D915C91A8962CAF3DAF4EAF5FAF01
:1086D000A897A7019601AC966CAD7DAD8EAD9FAD10
:1086E000AC970F94085D2B013C01A8962CAD3DADD5
:1086F0004EAD5FADA897E0966CAD7DAD8EAD9FADF4
:10870000E0970F94085D4B015C01A3019201C30146
:10871000B2010F947D562B013C01A5019401C501C6
:10872000B4010F947D569B01AC01C301B2010F94BB
:10873000095D0F94B75F4B015C01A70196016BA126
:108740007CA18DA19EA10F94085D6B017C01A89670
:108750002CAD3DAD4EAD5FADA8976FA178A589A5B5
:108760009AA50F94085D2B013C01A7019601C70152
:10877000B6010F947D566B017C01A3019201C301E8
:10878000B2010F947D569B01AC01C701B6010F9455
:10879000095D0F94B75F20E030E040E751E40F94AB
:1087A000035EA50194010F94095D6B017C0180902B
:1087B000C2049090C304A090C404B090C50420E00B
:1087C00030E040E85FE3C501B4010F94695F18161B
:1087D000F4F4C501B4010F94755E4B015C0160E0D7
:1087E00070E0CB01181419041A041B0434F40F941C
:1087F0004E51A50194010F947D5C0F941E569B0170
:10880000AC01B601C7010F94095D6B017C01E396D1
:108810002FADE397EA963FADEA97EB964FADEB9716
:10882000502FB601C7010F94175687FF21C06C96D1
:108830001FAF6C97C058DF4FB881C058D040A49686
:10884000BFAFA497E696CFAEE697E796DFAEE79781
:10885000E896EFAEE897E996FFAEE997E396CFAEDC
:10886000E397EA96DFAEEA97EB96EFAEEB970F2D24
:108870001F5FA396EEADFFADA3973496A396FFAF0F
:10888000EEAFA397183009F0F1CEFFEF2F1A3F0A91
:10889000A1962EAD3FADA1972C5F3F4FA1963FAF64
:1088A0002EAFA19738E02316310409F0B9CE6C96AB
:1088B0004FAD6C97E42FF0E0E654FB4F208181E050
:1088C00090E0A0E0B0E0A4960FACA49704C0880F9D
:1088D000991FAA1FBB1F0A94D2F7822B8083A496EC
:1088E0005FADA49762965FAF629763964FAF639751
:1088F000E6968FADE697E7969FADE797E896AFAD22
:10890000E897E996BFADE99767968CAF9DAFAEAF9C
:10891000BFAF67975F3F09F414C24F3F09F411C21C
:1089200084E04802F0011124E65CF84E10810181D8
:108930003280238027E137EB41ED58EB612F702F18
:10894000832D922D0F94695F87FDFFC123E030E0F6
:1089500048EC53E4612F702F832D922D0F941756FE
:1089600018160CF4F2C1A4969FADA497A4E09A0245
:10897000F0011124E65AF84EC080D180E280F380E5
:1089800027E137EB41ED58EBB601C7010F94695F62
:1089900087FDDBC123E030E04DEC53E4B601C701B5
:1089A0000F94175618160CF4D0C120E030E040EABE
:1089B00050E4B601C7010F94095DA0966FAFA09770
:1089C000A2967FAFA297A5968FAFA597A9969FAFC6
:1089D000A997CB01A596AFADA597A996BFADA997CD
:1089E00021968CAF9DAFAEAFBFAF2197812F902F57
:1089F000A32DB22D25968CAF9DAFAEAFBFAF2597FF
:108A0000A496BFADA497B11150C26C96EFAD6C9710
:108A1000E11118C220E030E040EA50E4612F702FED
:108A2000832D922D0F94095DA4966FAFA497AD96F8
:108A30007FAFAD97E1968FAFE197E3969FAFE39756
:108A40006C96FFAD6C97FF2309F4F1C26C963FADB5
:108A50006C97A096CFAEA097A296DFAEA297A596F0
:108A6000EFAEA597A996FFAEA99737300CF014C2C8
:108A700022ED822E23E5922E2BE7A22E21E4B22EA8
:108A800021964CAC5DAC6EAC7FAC219725962CAD9D
:108A90003DAD4EAD5FAD25976F962CAF3DAF4EAF60
:108AA0005FAF6F97A3019201B601C7010F94085DF4
:108AB0002D966CAF7DAF8EAF9FAF2D976F962CAD7F
:108AC0003DAD4EAD5FAD6F97612F702F832D922D11
:108AD0000F94085D61966CAF7DAF8EAF9FAF6197CD
:108AE000A30192016091491170914A1180914B113B
:108AF00090914C110F94085D2B013C016F962CADA9
:108B00003DAD4EAD5FAD6F9760914D1170914E11BF
:108B100080914F11909150110F94085D6F966CAF3A
:108B20007DAF8EAF9FAF6F97A0968FADA097A296A7
:108B30009FADA297A596AFADA597A996BFADA997F2
:108B40008DA79EA7AFA7B8ABA4968FADA497AD96FF
:108B50009FADAD97E196AFADE197E396BFADE397DB
:108B600089AB9AABABABBCABC984DA84EB84FC8435
:108B7000CDAADEAAEFAAF8AE2DEC3CEC4CEC5CE3FF
:108B8000C501B4010F947D5629813A814B815C81E6
:108B90000F947D56209155113091561140915711E7
:108BA000509158110F94095D69AF7AAF8BAF9CAFAC
:108BB000A3019201C301B2010F947D562B013C0128
:108BC0006F962CAD3DAD4EAD5FAD6F97CA01B9014B
:108BD0000F947D569B01AC01C301B2010F94095D56
:108BE00020E030E040E050E40F94695F1816ACF4E8
:108BF00020E030E040E05FE3C701B6010F94095D7B
:108C000029966CAF7DAF8EAF9FAF2997BE01635C95
:108C10007F4FCE0101960E94D92E89859A85AB851A
:108C2000BC8529968CAF9DAFAEAFBFAF29976B9631
:108C30001CAE1DAE1EAE1FAE6B97BE01695A7F4FB4
:108C4000CE01CD960E94D02ECE0101960F94E33135
:108C5000A0902811B0902911C0902A11D0902B110A
:108C6000E0902411F0902511009126111091271108
:108C70009701A801B501C6010F94695F181614F099
:108C80007501860180907C0290907D02A0907E020A
:108C9000B0907F022DEC3CEC4CEC5DE3B701C801D9
:108CA0000F947D5660937C0270937D0280937E02C8
:108CB00090937F0240E0BE01675B7F4FCE018D96AF
:108CC0000F94DD3980E1E9E4F1E1A0EEB8E0019034
:108CD0000D928A95E1F780927C0290927D02A0929B
:108CE0007E02B0927F020E94E2278111C8CB20E071
:108CF0004FEFBE016F5A7F4FCE0101960E949C300C
:108D000020E041E0BE016F5A7F4FCE0101960E94E4
:108D10009C302FEF40E0BE016F5A7F4FCE0101968D
:108D20000E949C3021E040E0BE016F5A7F4FCE018F
:108D300001960E949C300E946ADF0E94E227811106
:108D40009ECB8091591180935A11E5964EAD5FAD3F
:108D5000E59741505109E5965FAF4EAFE597452B3A
:108D600009F48DCB62968FAD629787FD88CB6396B1
:108D70008FAD639787FF17CC82CB63E687EB9AE0D2
:108D80000E94A6B50F941C3980E1E9E4F1E1A0EE60
:108D9000B8E001900D928A95E1F72D853E854F85CB
:108DA00058896091EC087091ED088091EE089091DF
:108DB000EF080F94095D6093EC087093ED088093C1
:108DC000EE089093EF08CE01CD960E946AFC2D85A7
:108DD0003E854F8558896091EC087091ED0880912F
:108DE000EE089091EF080F94085D6093EC08709383
:108DF000ED088093EE089093EF088CA58111A2CB2B
:108E000081E08CA78D819E81AF81B885B0588DA7F8
:108E10009EA7AFA7B8ABBE01635D7F4F80EE98E021
:108E20000E94D02E8FCB2BA13CA14DA15EA1AC9670
:108E30002CAF3DAF4EAF5FAFAC978FA198A5A9A562
:108E4000BAA5CBCBC601D70121968CAF9DAFAEAFF3
:108E5000BFAF219720E030E040EA50E4612F702F4F
:108E6000832D922D0F94085D25966CAF7DAF8EAF4C
:108E70009FAF25976C962FAD6C9727300CF4CACD19
:108E8000A4961FAFA497AD960FAFAD97E1963FAEF6
:108E9000E197E3962FAEE39792ED892E93E5992E15
:108EA0009BEFA92E90E4B92EEBCDA4964FADA497DD
:108EB00047300CF46EC06C965FAD6C975730BCF1C8
:108EC00020E030E040EA50E4B601C7010F94085DAD
:108ED00021966CAF7DAF8EAF9FAF219720E030E041
:108EE00040EA50E4612F702F832D922D0F94085D7E
:108EF000A4966FAFA497AD967FAFAD97E1968FAF75
:108F0000E197E3969FAFE3976C969FAD6C97A09621
:108F1000CFAEA097A296DFAEA297A596EFAEA5978B
:108F2000A996FFAEA99797300CF0B6CFA1CDC60198
:108F3000D70121968CAF9DAFAEAFBFAF219720E098
:108F400030E040EA50E4612F702F832D922D0F9472
:108F5000095D25966CAF7DAF8EAF9FAF25976C9660
:108F60008FAD6C978111BACF20E030E040EA50E439
:108F7000B601C7010F94085DA0966FAFA097A296A7
:108F80007FAFA297A5968FAFA597A9969FAFA997F8
:108F900077CF6C96AFAD6C97A1112BC020E030E07D
:108FA00040E251E4A0966FADA097A2967FADA29744
:108FB000A5968FADA597A9969FADA9970F94085D2B
:108FC000A0966FAFA097A2967FAFA297A5968FAFFE
:108FD000A597A9969FAFA997A4961FAFA497AD9602
:108FE0000FAFAD97E1963FAEE197E3962FAEE397D3
:108FF0003FCD6C96BFAD6C97B73034F120E030E0D8
:1090000040E251E4A0966FADA097A2967FADA297E3
:10901000A5968FADA597A9969FADA9970F94085DCA
:1090200021966CAF7DAF8EAF9FAF2197D5CFA09625
:10903000CFAEA097A296DFAEA297A596EFAEA5976A
:10904000A996FFAEA99728CFA4961FAFA497AD9677
:109050000FAFAD97E1963FAEE197E3962FAEE39762
:1090600082ED882E83E5982E8BEFA82E81E4B82E12
:1090700007CD87E599E00C945137CF92DF92EF92BC
:10908000FF920F931F93CF93DF9388E50E94533293
:10909000D82E89E40E945332C82E8823D1F10E9431
:1090A0002532D82F89E50E945332182F8AE40E9476
:1090B0005332082F882309F455C00E942532C82F47
:1090C0008AE50E945332E82EF12C811104C081E51B
:1090D0000E945332F82EC11001C000E0802F90E0B2
:1090E000D11001C010E0810F911D019721F4E11012
:1090F00062C0F11060C00E94394883E49EE0DF91B5
:10910000CF911F910F91FF90EF90DF90CF900C9433
:109110005137D11002C0DFEFC5CF0E942932209114
:10912000FB093091FC094091FD095091FE090F9413
:10913000085D20E030E040EA51E40F94085D2BED3B
:1091400036EB4DEC51E40F94095D25EF39E44FE91E
:109150005CE30F947D560F94755ED62F683008F44B
:10916000A1CFD9CF111102C0CFEFAACF0E942932CF
:109170002091FF093091000A4091010A5091020AA2
:109180000F94085D20E030E040EA51E40F94085D60
:109190002BED36EB4DEC51E40F94095D25EF39E4EE
:1091A0004FE95CE30F947D560F94755EC62F6830CF
:1091B00008F486CFD9CFD7FD02C0C7FF05C00E94F3
:1091C00039488AE29EE09BCF0E9429329B01AC0184
:1091D000AC2FCC0FBB0B88E0D802E001112460E07B
:1091E00070E0CB01FF2069F0FE01EA0FFB1FEE0FDC
:1091F000FF1FEE0FFF1FE952FA4F608171818281DC
:109200009381CA0FDB1FCC0FDD1FCC0FDD1FC952AE
:10921000DA4F0F94095D688379838A839B83DF919A
:10922000CF911F910F91FF90EF90DF90CF90089515
:1092300081E599E00C945137CF9384E50E94A132E7
:10924000C0E08823D9F00E940132C82F1816B4F468
:109250000E9418498DE40E9418378091FC04909177
:10926000FD040F94B1426C2FCC0F770B8DE59FE07E
:109270000E94DF3E8AE00E941837CFEF8C2FCF91FB
:1092800008954F925F926F927F928F929F92AF92CA
:10929000BF92CF92DF92EF92FF92CF93DF93CDB741
:1092A000DEB72C970FB6F894DEBF0FBECDBF40904F
:1092B000FB095090FC096090FD097090FE09209117
:1092C000390230913A0240913B0250913C02C30175
:1092D000B2010F94095D69837A838B839C838090AC
:1092E000FF099090000AA090010AB090020A209114
:1092F0003D0230913E0240913F0250914002C50133
:10930000B4010F94095D6D837E838F839887C0902D
:10931000030AD090040AE090050AF090060A209112
:109320004102309142024091430250914402C701F0
:10933000B6010F94095D69877A878B879C87209196
:109340004502309146024091470250914802C301C4
:10935000B2010F94095D2B013C012091490230912B
:109360004A0240914B0250914C02C501B4010F9446
:10937000095D4B015C0120914D0230914E024091FC
:109380004F0250915002C701B6010F94095D6B0165
:109390007C010E9418498EEA9EE00E94513783E5C5
:1093A0000E945332882321F00E94153280933702A5
:1093B00080913702811151C085E99EE00E945137AA
:1093C00086EA9EE00E94513749815A816B817C81F7
:1093D00080E39CE20E94C9394D815E816F8178856E
:1093E00089E891E40E94C93949855A856B857C8555
:1093F00086E891E40E94C93984EA9EE00E945137D0
:109400008CE99EE00E945137B301A20180E39CE207
:109410000E94C939B501A40189E891E40E94C939C3
:10942000B701A60186E891E40E94C9398AE02C962A
:109430000FB6F894DEBF0FBECDBFDF91CF91FF9086
:10944000EF90DF90CF90BF90AF909F908F907F90E4
:109450006F905F904F900C94183789E99EE0AECFE3
:109460002F923F924F925F926F927F928F929F9234
:10947000AF92BF92CF92DF92EF92FF920F931F9322
:10948000CF93DF93CDB7DEB76A970FB6F894DEBF00
:109490000FBECDBF83E50E945332182F3090481184
:1094A000882319F00E941532382E409049115090AF
:1094B0004A1160904B1170904C1180914D11909118
:1094C0004E11A0914F11B09150118B8B9C8BAD8B95
:1094D000BE8B8091511190915211A0915311B09176
:1094E00054118F8B988FA98FBA8F112329F03110C7
:1094F00003C080E00E940D3586E50E945332888BC0
:109500000E940836882309F4BFC083E40E945332C6
:10951000882309F498C00E9429326B017C01A7EDD1
:10952000B5E0BF83AE83B987A887F8E0FD831D86C9
:109530001E8628EC2F8702EC1A86212C88EC8B875C
:1095400092E49C87A885B985BA8BA98B18E0E98934
:10955000FA8981909190A190B190FA8BE98B2A853C
:10956000322D4B855C85C501B4010F94175687FFDA
:1095700004C08A86292CAB86BC862D853E854F8506
:10958000502FC501B4010F94695F181624F48D861D
:109590009E86AF860B2D1150D1F6FD81F150FD83D3
:1095A00088859985809699878887F111CBCF2D85FD
:1095B0003E854F85502F6A85722D8B859C850F9433
:1095C000095D20E030E040E05FE30F947D56A701A5
:1095D00096010F94095D6B017C012DEB37E346E8A2
:1095E00055EB0F94695F87FD0AC02DEB37E346E822
:1095F00055E3C701B6010F941756181624F580E0FD
:109600000E940D3518E0AE80BF8008E0D5016D9155
:109610007D918D919D915D014D01B4E08B1A910872
:10962000A70196010F94085DF40160837183828322
:109630009383015059F711508E819F8180969F83AB
:109640008E831111E0CFA889AA2351F00E94083619
:10965000882331F080E09DE00E9451370E942C3930
:109660008AE50E945332882359F00E942932698387
:109670007A838B839C8360E0CE0101960E9428351B
:10968000832D0E940D350BC0311003C0988999239A
:1096900039F30E94184986E19DE00E94513733203A
:1096A00051F080914811811106C00E94394881EE25
:1096B0009CE00E9451370E94184983ED9CE00E9473
:1096C0005137809148110E94AB390E94184986ECAD
:1096D0009CE00E945137C0901309D0901409E0908B
:1096E0001509F090160920E030E0A901C701B60184
:1096F0000F94695F18160CF053C042E0C701B60121
:109700000F94BF0A8DE00E9418378AE00E94183734
:10971000A30192016091491170914A1180914B11FE
:1097200090914C110F94175681111FC02B893C89C1
:109730004D895E8960914D1170914E1180914F114C
:10974000909150110F94175681110FC02F89388DA9
:10975000498D5A8D60915111709152118091531120
:10976000909154110F94175681110E9422FE6A960F
:109770000FB6F894DEBF0FBECDBFDF91CF911F9122
:109780000F91FF90EF90DF90CF90BF90AF909F90A0
:109790008F907F906F905F904F903F902F900895A3
:1097A00081EC9CE00E945137B3CFCF93C82F82E069
:1097B000C11184E040E060E00E94B3870E94184934
:1097C00089EC99E0CC2311F08EED99E0CF910C94C7
:1097D0005137FF920F931F93CF93DF93EC018B01CF
:1097E000F42E0E94CCD70E94394881E399E00E9470
:1097F00051370115110511F40BE110E4209711F414
:10980000C8E2D9E00E9462BC1F930F93DF93CF930D
:1098100088E199E09F938F9381E08F930E948BB5AD
:109820000E94CA86C0910017C695C6958BEF96E137
:109830000E94D529DC2FDD0F1D2F1C0FEDB7FEB7C1
:1098400037960FB6F894FEBF0FBEEDBF83E00E94BF
:10985000532940E154E16C2F80E00E94802C10924B
:109860003617D093371789E099E00E94652A109245
:109870003617109337178CEF98E00E94652A8FEF08
:1098800096E10F94D6408111E1CF61E08FE199E03C
:109890000E949C3889EE93E030E6019729F0232F4F
:1098A0002A950000E9F7F9CFF89489EE93E038EEB5
:1098B000019729F0232F2A950000E9F7F9CF0E949C
:1098C000CCD7FF2041F00E9483360E9495229099C8
:1098D00005C0A895FCCF0E949322F7CF909B02C0B1
:1098E000A895FCCFF0E0E0E0DF91CF911F910F91C0
:1098F000FF9019945F926F927F928F929F92AF9296
:10990000BF92CF92DF92EF92FF920F931F93CF936C
:10991000DF931F92CDB7DEB77C0139018B015B016C
:10992000A40EB51ED12CC12CA016B10609F450C04E
:10993000F70180809180F80151908F015982C40114
:109940000F94355C5816B9F1652DC4010F943D5C38
:10995000FFEFCF1ADF0AC6018F779927892B21F1F4
:1099600062E070E080E090E00F94B038C4010F94A2
:10997000355C99818917F9F00E9418498BE596E0CA
:109980000E94513781E00F90DF91CF911F910F918D
:10999000FF90EF90DF90CF90BF90AF909F908F900F
:1099A0007F906F905F90089562E070E080E090E0BB
:1099B0000E944D36DBCFBE016F5F7F4FC3010F9416
:1099C000D828F70180819181019691838083ACCF63
:1099D00080E0D9CF8091591190915A112FEF3FEF2C
:1099E000981751F0E92FF0E0E75AFE4E228130E05F
:1099F0009F5F9F7790935A11C90108951F920F920C
:109A00000FB60F9211240F900FBE0F901F90189554
:109A10001F920F920FB60F9211240BB60F920F9355
:109A20001F932F933F934F935F936F937F938F93E6
:109A30009F93AF93BF93CF93DF93EF93FF93C09127
:109A4000C60000915A11D091591111E01D0F1F77D6
:109A500090918104913108F09FC0E92FF0E08827B0
:109A6000EB5CF24B8F4F0D94005D464D754D844D70
:109A7000934D9A4DCC4D9E4DCC4DA24DA64DCC4D07
:109A8000AA4DAE4DB24DB94DCC4DC44DC03229F0AA
:109A900028F5CA3011F0CD3031F5011731F0ED2F36
:109AA000F0E0E75AFE4EC283D12FD0935911FF91B7
:109AB000EF91DF91CF91BF91AF919F918F917F9166
:109AC0006F915F914F913F912F911F910F910F9047
:109AD0000BBE0F900FBE0F901F901895CD3481F0E4
:109AE00081E0CE3471F080E10CC0CA3338F4C03369
:109AF000A0F6C03291F2CD32B1F7CFCFCD3499F785
:109B000082E080938104C9CFC13359F018F4C03288
:109B100021F2E9CF88E0C433A1F38BE0C83389F3A5
:109B2000E2CF83E0EECF84E0C03359F386E0C13367
:109B300041F3D9CF85E0C833B1F6E3CF87E0C23334
:109B400091F6DFCF89E0C13371F6DBCF8AE0C03315
:109B500051F6D7CF8CE0C73331F6D3CF8DE0C63383
:109B600011F6CFCFC03209F498CF8EE0C33549F259
:109B7000BACF80ED8C0F8A3008F08FCF9FE09093A2
:109B800081048093800489CFCA3019F0CD3009F068
:109B900084CF1092810481CFCA3019F0CD3009F002
:109BA0007CCF809139178823A1F3973041F138F4A5
:109BB000953079F7109274021092FB08EACF9A3030
:109BC00011F19F3031F7909180048091F808109244
:109BD000F808823089F38430E9F08130D1F6992396
:109BE000B1F09130B1F682E08093FA088091F908E3
:109BF000882379F2109255020E948022CACF81E018
:109C00008093E906C6CF81E08093E806C2CF8093B7
:109C1000FA08BFCF81E39EE19093710880937008AA
:109C2000B8CF8EBD0DB407FEFDCF08958FEF8EBD6A
:109C30000DB407FEFDCF8EB50895909164009B7F13
:109C400090936400982F906A96959CBD80FD03C008
:109C500091E0863009F490E09DBD0895CF93DF93A5
:109C6000EB010E945137CE01DF91CF910C949ED130
:109C7000AF92BF92CF92DF92EF92FF920F931F931A
:109C8000CF93DF93CDB7DEB7E6970FB6F894DEBF7C
:109C90000FBECDBF0091FF0410910005F8010190A7
:109CA0000020E9F731976F01C01AD10AF801CF01FE
:109CB000801B910B8C159D053CF481918F32B9F777
:109CC000DF0111971C92F3CF8BE1E6EAF7E1DE01A9
:109CD0005C9601900D928A95E1F7F12CE12CEC1441
:109CE000FD040CF05DC0F801EE0DFF1D80818111B7
:109CF00003C08FEFE81AF80A5801AE0CBF1CF5013B
:109D00008081882309F44CC0FFEFEF1AFF0AF801A5
:109D1000EE0DFF1D7F01E01AF10A81918111FACF4A
:109D2000CE014C960E94AFD58BE1FE017C96DE0100
:109D3000119601900D928A95E1F7B501CE01019639
:109D40000E9410CECE0101960E9453348FE20E94F1
:109D500018378091CD1381113BC08FE593E00E94AD
:109D60009ED18091851784FF1BC019821C8221E03F
:109D7000A501BE01645E7F4FCE0101960F94E008FD
:109D8000811129C08AE00E9418370E941849B50144
:109D900087E095E10E942E4ECE0101960E94533439
:109DA0008AE00E941837CE014C960E945334E69602
:109DB0000FB6F894DEBF0FBECDBFDF91CF911F91DC
:109DC0000F91FF90EF90DF90CF90BF90AF900895EC
:109DD0008DEC93E1C4CFCE014C960E9406D58BE169
:109DE000FE013196DE015C9601900D928A95E1F7B5
:109DF000CE0101960E94533472CF2F923F924F9220
:109E00005F926F927F928F929F92AF92BF92CF920A
:109E1000DF92EF92FF920F931F93CF93DF9300D0C7
:109E200000D000D01F921F92CDB7DEB7B82E809120
:109E30004612843008F0D1C10F94E3386B017C01E5
:109E400080914612811108C08091591190915A1148
:109E5000891B8F7709F4D9C681E6A82E13C08A30F2
:109E600019F08D3009F0F6C0109241128091DF1187
:109E70009091E011FC01E552FE4E1682892BF1F41F
:109E80000E947CF580914612843008F0ECC08091ED
:109E9000591190915A11891B8F7709F4E4C00E94DF
:109EA000EA4C97FFDCCF0E94394881EA97E00E9494
:109EB00051378091591180935A11E4CF1092E011DB
:109EC0001092DF1101EE11E1F8018191803209F465
:109ED00046C08E3409F0A9C06CE977E0C8010F9440
:109EE00094554C01892B41F06EE470E0C801049652
:109EF0000F945E60009709F4C8014AE050E070E0FA
:109F000060E001960F9404532B013C018091DB111A
:109F10009091DC11A091DD11B091DE110196A11D8F
:109F2000B11D481659066A067B0629F060E089E6ED
:109F300097E0892851F16AE270E0C8010F948D60C2
:109F40009C01009729F1982F901B912C992349F09F
:109F50009150F801E90FF11D80819826F7CF8F010C
:109F6000B3CF4AE050E070E060E0C90101960F9481
:109F70000453292D30E050E040E062177307840756
:109F8000950751F060E08AE497E00F94A52D7ACF11
:109F900060E080E297E0F9CF4092DB115092DC1153
:109FA0006092DD117092DE118091B3088130E1F092
:109FB00067E470E0C8010F945E600097A9F04AE082
:109FC00050E070E060E001960F9404536430710536
:109FD0008105910548F48FE796E00E94513760E0D3
:109FE00085E796E00E94A6B5C0920009D0920109CB
:109FF000E0920209F09203098091E1118B3309F498
:10A0000041CF80914612843008F03CCF80914812B5
:10A010008A9DC001112461EE71E1875B9D4E0F9412
:10A02000696080E00F945F2D2DCF8091851780FFB0
:10A03000BBCF6EE97FE3C8010F949455009731F0D0
:10A04000FC01838180538A3008F0AECF60E086EF58
:10A0500096E09BCF2FED31E141EE51E161E472E1F9
:10A060000E940F220FCF8091851782FFB6C01A82FF
:10A07000198271E6F72EE0E1EE2EF9E6DF2E8091EF
:10A080004612843008F0A9C00E9447228111A5C061
:10A0900041E050E0BE016B5F7F4F8AEE98E10E9485
:10A0A0003ED20D8110E0019711F00FEF1FEF80916C
:10A0B000F2189091F318A091F418B091F5188093CC
:10A0C000811790938217A0938317B09384170E94EF
:10A0D00047220F3F100749F4811107C00E943948F9
:10A0E0008FEB97E00E945137CACF40914812242F3E
:10A0F00030E00A3061F00D3051F0882309F45FC080
:10A1000089819A81009719F001969A838983109228
:10A11000820489819A81F29EF001F39EF00D112450
:10A12000EA5BFD4EE80FF91F1382892B69F50E9447
:10A130007CF50E944722882309F4A1CF0E946ADFA0
:10A140008AEE98E10E9406D580917C17882391F1D0
:10A15000815080937C178D9DC001112462E0815253
:10A16000984F0F94D846E0917C1724E0E29FF001CD
:10A170001124E552F84F60817181828193810E94A0
:10A1800026260F944F447BCF1A82198281E00F94C8
:10A190005F2D8091811790918217A0918317B091C4
:10A1A00084178093421290934312A0934412B09369
:10A1B0004512BFCF0F943E44E092B30860CF4F9D4D
:10A1C000A0011124475B5D4E9E012F5F3F4F62E867
:10A1D00074E0802F0E940F2252CF0F94E3386B015E
:10A1E0007C01B11004C08091DA07882351F0C0923D
:10A1F000F008D092F108E092F208F092F308BB2444
:10A20000B3948091D8049091D904A091DA04B091CC
:10A21000DB040097A105B10551F14091F008509180
:10A22000F1086091F2087091F308840F951FA61F42
:10A23000B71FA7019601281B390B4A0B5B0BDA01EC
:10A24000C901B7FD14C00E9439486091FE087091A1
:10A25000FF088AE198E00E942E4E8AE00E9418379B
:10A2600040E070E060E090E080E00E94E94B809187
:10A27000100290911102A0911202B0911302892B49
:10A280008A2B8B2B79F09091C3168091C416981766
:10A2900009F4ACC1C092F008D092F108E092F20843
:10A2A000F092F30880919304909194049099E0C106
:10A2B00001969093940480939304809193049091D9
:10A2C00094048E3E92406CF00E94394887EF97E0EC
:10A2D0000E94513740E070E060E090E080E00E9432
:10A2E000E94B0F94E3384B015C018091FB0881112D
:10A2F00008C02091C3169091C41681E0291301C0B3
:10A3000080E020917F163091801691E089272A3ACB
:10A3100031050CF480E091E040918704509188046D
:10A320006091890470918A04452B462B472B09F4D0
:10A3300090E0981789F0882309F4A0C1D501C401E1
:10A3400080569444A24FBF4F809387049093880413
:10A35000A0938904B0938A044090551150905611EF
:10A3600060905711709058112091830430918404AB
:10A370004091850450918604C301B2010F94175691
:10A38000882319F18091870490918804A091890411
:10A39000B0918A04409283045092840460928504B0
:10A3A00070928604892B8A2B8B2B09F449C0D50126
:10A3B000C40180569444A24FBF4F8093870490936A
:10A3C0008804A0938904B0938A04809187049091B3
:10A3D0008804A0918904B0918A040097A105B10571
:10A3E00079F1881A990AAA0ABB0AB7FC29C0109207
:10A3F0008704109288041092890410928A0482EED5
:10A4000097E00E94513760E08EEC97E00E94A6B57D
:10A4100080918116909182161816190624F490E006
:10A4200080E00E94ECDE80911D0990911E091816B3
:10A43000190634F410921E0910921D090E9496C943
:10A4400080918F0490919004A0919104B091920416
:10A4500046015701881A990AAA0ABB0AD501C40104
:10A46000B7FD9CC12091C3169091C416409164021F
:10A4700080916302291306C19091390A899FC00116
:10A480001124880F892F881F990B91958D838091B6
:10A490003A0A489FC0011124880F892F881F990B01
:10A4A00091958E830F94E33869837A838B839C83A1
:10A4B00040E0BE016F5F7F4FCE0105960E94BEDF78
:10A4C0006D8170E089E00F94DA3741E0BE016F5F83
:10A4D0007F4FCE0105960E94BEDF6E8170E087E05F
:10A4E0000F94DA378091F506882309F44AC1009168
:10A4F000330210913402C8010297209181163091E5
:10A500008216281739070CF43CC18090C4168F823C
:10A51000188619861A861B868091C3169F80891516
:10A5200009F4CAC0892D90E03BE6A32EA89EF00155
:10A53000A99EF00D1124E25BF54F45895689678984
:10A54000708D452B462B472B81F4418D528D638DA9
:10A55000748D452B462B472B41F4458D568D678DC9
:10A5600070A1452B462B472BE1F12BE6B22EB89E6E
:10A570009001B99E300D1124A901425B554F1A017B
:10A58000FA0161817281838194810F94B75F4B01DD
:10A590005C01F10161A172A183A194A10F941C56E9
:10A5A0002B013C01F10165A176A187A190A50F9433
:10A5B0001C569B01AC01C301B2010F94035EA501BF
:10A5C00094010F947D564B015C01288539854A859D
:10A5D0005B850F94695F181624F488869986AA868D
:10A5E000BB868F818F5F8F708F8396CFBB2019F0D2
:10A5F0001092950457CE0F94E3380091F008109113
:10A60000F1082091F2083091F308809010029090A8
:10A610001102A0901202B0901302080D191D2A1DFC
:10A620003B1D601B710B820B930B97FDE1CF80915B
:10A630009504811137CE81E0809395045F9A8091D3
:10A640006E088E7F80936E088A9A80916E088D7F47
:10A6500080936E0880910801809581708093060137
:10A6600080916E088B7F80936E080E9493221ACE91
:10A67000181619060CF021CE01971BCE80E090E051
:10A68000DC0162CE2091C4165BE6259F9001112467
:10A69000225B354FF901EF59FF4F9081899FC0012F
:10A6A0001124880F892F881F990B91958D832E591E
:10A6B0003F4FF9018081EDCE20912D0230912E0285
:10A6C00040912F0250913002688579858A859B855B
:10A6D0000F947D564B015C01B801012E000C880BD4
:10A6E000990B0F941E569B01AC01C501B4010F9448
:10A6F000095D69837A838B839C83409131025091F9
:10A700003202B801CE0101960E9497D889809A80C2
:10A71000AB80BC8040908B0450908C0460908D0482
:10A7200070908E04A3019201C501B4010F941756D5
:10A7300087FF16C028E431EE4AE75FE3C301B201A8
:10A740000F947D5620E037ED43EA5CE30F94095DFA
:10A75000A50194010F947D5669837A838B839C8332
:10A7600069817A818B819C8160938B0470938C04C6
:10A7700080938D0490938E040F94755ECB010E949C
:10A78000ECDEF4E6CF0ED11CE11CF11CC0928F046C
:10A79000D0929004E0929104F09292040E947CF591
:10A7A0008091B308882309F4F0C180915502882371
:10A7B00009F471C08091F90881116DC00E94713651
:10A7C000811105C08091DA07882309F464C0F894E8
:10A7D000649B10C08091510290915202A09153024B
:10A7E000B09154028093E0069093E106A093E206B4
:10A7F000B093E3066091E0067091E1068091E20675
:10A800009091E306789420E030E0A9010F94175668
:10A8100087FF41C001E00093F9088091DA078111B8
:10A8200038C00E94CD380093F80840E366E878E02D
:10A830008DED90E40E94D23861E081ED90E40E94B9
:10A84000B4381091DC0460E0102784E59AE069F4E4
:10A8500084E798E00E949C3880E30E9418378AE0E1
:10A860000E94183760E087E598E00E949C3882E6F5
:10A8700098E00E94513780E30E9418378AE00E94D6
:10A880001837112331F08DE598E09093710880938B
:10A8900070080E946ADF90910901892F809581706C
:10A8A00010910802181709F45AC0209185172062E8
:10A8B000209385178093080290FD10C064EF71E02B
:10A8C00080E090E00E944D360E940FD58091851760
:10A8D00083FDBEC1112309F442C002C00E94CECD47
:10A8E000123008F46BC100E00E94EB2883E08093F3
:10A8F00080020F94E3386C597F4F8F4F9F4F6093C6
:10A9000004057093050580930605909307050023C1
:10A9100031F1123021F58091851783FF20C00F940B
:10A920009B43882379F081E00F94B74242EB50E0DB
:10A9300069E479E08BE897E10E943ED28BE897E1E9
:10A940000E9406D50E944134811144C10E942B34DB
:10A950000F941D4581E080937B170F945F450F9402
:10A96000E3386B017C0110910F021123F1F080910B
:10A97000FC088823D1F0409196045091970460918F
:10A9800098047091990446015701841A950AA60A01
:10A99000B70AB501A40177FD1AC0833009F430C1AC
:10A9A0000CF01FC181300CF024C1212F30E0A8EE43
:10A9B000B3E00F94AF5CC60ED71EE81EF91EC0921E
:10A9C0009604D0929704E0929804F09299048091B2
:10A9D0001109813009F073C00F94E3386B017C01D9
:10A9E00080919E0490919F04A091A004B091A10435
:10A9F000A7019601281B390B4A0B5B0BDA01C90131
:10AA0000B7FD3AC0D701C601805F984DAF4FBF4F29
:10AA100080939E0490939F04A093A004B093A104FC
:10AA20008090CA059090CB05A090CC05B090CD0544
:10AA30000F94B700AB01BC014093CA055093CB05FE
:10AA40006093CC057093CD0580915F08909160086C
:10AA5000A0916108B091620888199909AA09BB09F7
:10AA6000840F951FA61FB71F80935F0890936008FF
:10AA7000A0936108B093620880919A0490919B041E
:10AA8000A0919C04B0919D0446015701881A990A2F
:10AA9000AA0ABB0AD501C401B7FD11C020E8C20E45
:10AAA0002EEED21E26E3E21EF11CC0929A04D09232
:10AAB0009B04E0929C04F0929D040E946EDE0F9431
:10AAC00048050E94B2B98091D704882379F10F9488
:10AAD000E3386B017C018091D3049091D404A09160
:10AAE000D504B091D60446015701881A990AAA0ADA
:10AAF000BB0AD501C401B7FD19C02091D70430E0CD
:10AB0000A8EEB3E00F94AF5CC60ED71EE81EF91E88
:10AB1000C092D304D092D404E092D504F092D6042B
:10AB200080E00F94630B8AE00E9418378091D20472
:10AB3000882359F10F94E3386B017C018091CE0496
:10AB40009091CF04A091D004B091D104A7019601B7
:10AB5000281B390B4A0B5B0BDA01C901B7FD15C085
:10AB60002091D20430E0A8EEB3E00F94AF5CC60EA3
:10AB7000D71EE81EF91EC092CE04D092CF04E092F8
:10AB8000D004F092D1040F94BE432B960FB6F894E4
:10AB9000DEBF0FBECDBFDF91CF911F910F91FF9010
:10ABA000EF90DF90CF90BF90AF909F908F907F906D
:10ABB0006F905F904F903F902F90089560E087E9ED
:10ABC00098E00E94A6B58091120581118CCE0E945A
:10ABD000CA8689CE84EB98E09093710880937008C0
:10ABE000BECE843009F0E1CE0E9418498BEB98E08C
:10ABF00004C00E9418498AEE98E00E945137D5CED1
:10AC00000E94184983ED98E0F8CF80910009909157
:10AC10000109A0910209B0910309A7019601281B1F
:10AC2000390B4A0B5B0BDA01C901885E9340A1091D
:10AC3000B109B7FD11C989EB97E00E945137C09265
:10AC40000009D0920109E0920209F092030904C9B7
:10AC5000123028F460E085EA98E00E94A6B501E091
:10AC600043CECF93DF93C82FD62F8091FF1083FD63
:10AC700014C080914B0A811110C08091850290917F
:10AC80008602AC0141505109209181163091821603
:10AC90002417350714F40E94ECDE40E06D2F8BE0A2
:10ACA0000E94B387CC2339F040E061E080E0DF917F
:10ACB000CF910D945B0D80914B0A91E08927809391
:10ACC000740280917402882389F080917F1690919C
:10ACD00080162091811630918216821B930B97FF6C
:10ACE00003C0919581959109029744F410927402E2
:10ACF0008091FF1083FF06C0C1E01AC080E00E946F
:10AD0000FD4EDFCFC0914B0AC11112C08091850268
:10AD10009091860201972091811630918216281712
:10AD2000390754F70E94184988EB99E00E9451377F
:10AD30008C2FDF91CF910895AF92BF92CF92DF9287
:10AD4000EF92FF920F931F93CF93DF93CDB7DEB7B0
:10AD500064970FB6F894DEBF0FBECDBF0E941C49AA
:10AD6000D82E87FDB5C08AE50E94A132882309F458
:10AD7000C0C040E050E0BA018AE50E94BC327B01CD
:10AD80008C014D2D63E085E00E94B3872091511125
:10AD900030915211409153115091541160E070E084
:10ADA00088EC93E40F94085D5B016C019701A801A6
:10ADB0000F94695F181614F07501860120E030E0E9
:10ADC000A901B701C8010F94695F181624F4E12C9A
:10ADD000F12C00E010E0B701C8010F94755E072E5A
:10ADE000000C880B990B0F941E566D837E838F8306
:10ADF000988720E030E0A9010F941756882321F0AE
:10AE0000CE0105960E94742680E090E0A0EAB1E4AD
:10AE100089879A87AB87BC871D861E861F86188AFE
:10AE20008CE40E945332882309F468C00E942932BE
:10AE30006B017C0120E030E0A901C701B6010F944D
:10AE4000695F87FF04C0F7FAF094F7F8F094C98AB5
:10AE5000DA8AEB8AFC8A209181163091821624309E
:10AE6000310574F080917F1690918016821B930BB0
:10AE700097FF03C091958195910901E004970CF427
:10AE800000E063E080E00E943156811140C083E021
:10AE900080932402109211050E94CA866D817E81E2
:10AEA0008F8198858B019C01305809831A832B83ED
:10AEB0003C8320E030E0A9010F941756882321F04D
:10AEC000CE0101960E947426109211050E94CA8636
:10AED00064960FB6F894DEBF0FBECDBFDF91CF9161
:10AEE0001F910F91FF90EF90DF90CF90BF90AF90A8
:10AEF0000895E12CF12C00E211E443CFC090D2057B
:10AF0000D090D305E090D405F090D50593CF83E0A1
:10AF1000E82E22E0AE01475F5F4FBE016F5E7F4FBC
:10AF2000CE010D960F94A92FB9CF6F927F928F9279
:10AF30009F92AF92BF92CF92DF92EF92FF920F93C8
:10AF40001F93CF93DF9300D000D01F921F92CDB7F5
:10AF5000DEB75C014B013A01F22E68010091EE066A
:10AF60001092EA061092EB061092EC061092ED0693
:10AF70001092EE060F94EF38809181169091821610
:10AF80008C159D051CF4C6010E94ECDE60E080E09B
:10AF90000E94315681112FC1109211050E94CA865C
:10AFA0001C141D0444F4C6010E94ECDE40E060E085
:10AFB00080E00F945B0D40E060E088E00E94B38782
:10AFC00060E081E00E94315680E090E0A0E7B2E4CA
:10AFD00089839A83AB83BC8380E090E0A0E8B0ECE7
:10AFE0008D839E83AF83B887BE016F5F7F4FCE0195
:10AFF00005960E944AF587E00E948AF3811158C0A5
:10B000008091511190915211A0915311B09154110E
:10B010004091AE045091AF046091B0047091B104BE
:10B02000C090AA04D090AB04E090AC04F090AD04C2
:10B03000C092E008D092E108E092E208F092E308C2
:10B040004093E4085093E5086093E6087093E7089E
:10B050008093E8089093E908A093EA08B093EB087E
:10B0600080E090E0A8E4B2E489839A83AB83BC8358
:10B07000CE0101960E946AFC8091B2049091B304C3
:10B08000A091B404B091B5048093E8089093E908C6
:10B09000A093EA08B093EB0880E090E0A0EAB0E467
:10B0A00089839A83AB83BC83CE0101960E946AFC9C
:10B0B000C12CD12C80E7E82E82E4F82EC982DA82F6
:10B0C000EB82FC8280E090E0A0E8B0E48D839E8378
:10B0D000AF83B887BE016F5F7F4FCE0105960E9498
:10B0E0004AF520E030E0A9016091B6047091B70400
:10B0F0008091B8049091B9040F94175687FF0BC044
:10B10000C982DA82EB82FC82BE016F5F7F4F86EBE1
:10B1100094E00E944AF58091B6049091B704A09102
:10B12000B804B091B9048093551190935611A0932F
:10B130005711B09358118093EC089093ED08A093A9
:10B14000EE08B093EF088CEE98E00E9472F18091C7
:10B15000D60581110F94E142109211050E94CA8612
:10B1600061E081E69AE00E949C388091DA07815084
:10B170008093DA0742EF5DE169E67AE085E00F94BB
:10B18000B3308091DA07882339F00F944F448091CF
:10B19000DA0781508093DA078091A904882351F05F
:10B1A0001092A9048091A7048093390A8091A80481
:10B1B00080933A0A0E94802280911109823011F412
:10B1C0000F9479010F9418460E94CA8628960FB6EC
:10B1D000F894DEBF0FBECDBFDF91CF911F910F91CD
:10B1E000FF90EF90DF90CF90BF90AF909F908F90A7
:10B1F0007F906F900895E12C2F2DA301B401C5011C
:10B200000F94A92FCDCE4F925F926F927F92AF9203
:10B21000BF92CF92DF92EF92FF921F93CF93DF9373
:10B2200000D000D01F921F92CDB7DEB75C01E62E92
:10B23000F42E642F80E00E943156182F81111BC01C
:10B24000EE2021F0109211050E94CA86812F2896C7
:10B250000FB6F894DEBF0FBECDBFDF91CF911F9127
:10B26000FF90EF90DF90CF90BF90AF907F906F9066
:10B270005F904F900895EE2029F040E06F2D83E01D
:10B280000E94B38780E090E0A0E7B2E48D839E83C4
:10B29000AF83B88780E090E0A0E8B0EC89839A8320
:10B2A000AB83BC83BE016B5F7F4FCE0101960E94D2
:10B2B0004AF568E873E180E090E00E944D36C12CC9
:10B2C000D12C88ECE82E81E4F82ECD82DE82EF824C
:10B2D000F88680E090E0A0E8B0E489839A83AB83AD
:10B2E000BC83BE016B5F7F4FCE0101960E944AF581
:10B2F000409038115090391160903A1170903B1184
:10B30000C0923811D0923911E0923A11F0923B116B
:10B3100080E090E0A0E2B2E48D839E83AF83B887A3
:10B32000F50180819181A281B38189839A83AB8366
:10B33000BC83BE016B5F7F4FCE0101960E944AF530
:10B34000409238115092391160923A1170923B112B
:10B35000129A64E670E080E090E00E944D3676CF6D
:10B36000BF92CF92DF92EF92FF920F931F93CF93F2
:10B37000DF9300D01F92CDB7DEB77C016B018A014D
:10B38000B22E61E084E59AE00E949C3842EF5DE1D4
:10B390006BE57AE085E00F94B3309091DA0781E0B5
:10B3A000890F8093DA078091851782FF06C08B7F13
:10B3B000809385179E5F9093DA070F94B10180E127
:10B3C000E9E4F1E1AAEAB4E001900D928A95E1F78F
:10B3D0000E946ADF8091A90481110FC081E08093EF
:10B3E000A9048091390A8093A7041092390A8091A8
:10B3F0003A0A8093A80410923A0A20E030E0A901AA
:10B40000F70160817181828193810F94175688239F
:10B41000F1F080914B0A81110CC0809185029091CE
:10B420008602019720917F163091801628173907E0
:10B4300074F080E090E0A0E7B2E489839A83AB8364
:10B44000BC83BE016F5F7F4FC7010E944AF587E052
:10B450000E948AF3811103C0B6010F948D0420E08D
:10B4600030E0A901F80160817181828193810F949C
:10B470001756882329F042E06B2DC8010E9403591A
:10B48000129A64E670E080E090E00E944D3681E020
:10B490000F900F900F900F90DF91CF911F910F9110
:10B4A000FF90EF90DF90CF90BF900895CF92DF9202
:10B4B000EF92FF92CF93DF936B017C01D42FC09169
:10B4C000FC0883E08093FC0881E08093FB08C114B2
:10B4D000D104E104F10431F00F94E338C60ED71E15
:10B4E000E81EF91E8091FB08882389F0C114D1045D
:10B4F000E104F10421F48D2F0E94FD4EF3CF0F944F
:10B50000E3386C197D098E099F0997FDF4CF1092DD
:10B51000FB08C093FC08DF91CF91FF90EF90DF9084
:10B52000CF9008951F93CF93DF93D82FC62F0E94FB
:10B53000D54B61E08C2F0E9459340F94E338685347
:10B5400070458F4F9F4F6093EA067093EB06809390
:10B55000EC069093ED061092EE061091FC0883E045
:10B560008093FC0830E020E042E051E466E47AE0B9
:10B5700082E00E94F53881E08093FB088091FB080F
:10B58000882309F463C060E08C2F0E9459348091B5
:10B59000EE06882309F456C040E060E08AE00E948D
:10B5A000B3870E9418498CE29AE00E94513730E03C
:10B5B00020E046E15AE06DE17AE082E00E94F53851
:10B5C00041E060E070E0CB010E94565A30E020E09C
:10B5D00050E040E069E07AE085E00E94F5381092A2
:10B5E000EA061092EB061092EC061092ED0610920D
:10B5F000EE060F94EF3860E080E00E9431568D2F08
:10B600000E94D54B0F94E338685370458F4F9F4F7E
:10B610006093EA067093EB068093EC069093ED0638
:10B620001092EE0630E020E042E051E46DEF79E068
:10B6300082E00E94F53881E08093FB0861E08C2F66
:10B640000E94593481E00E94FD4E98CF1093FC086F
:10B65000DF91CF911F910895CF92DF92EF92FF92E9
:10B660000F931F93CF93DF93CDB7DEB7A0970FB69D
:10B67000F894DEBF0FBECDBF0E941C4987FDD1C02C
:10B68000482F61E081E00E94B38785E40E94533235
:10B69000882309F4D5C00E9429326B017C0120E087
:10B6A00030E0A9010F94695F87FF04C0F7FAF094B6
:10B6B000F7F8F094F7FAF094F7F8F094C98ADA8A78
:10B6C000EB8AFC8A8CE0EBE8F2E0DE011196019057
:10B6D0000D928A95E1F78AE50E94A132882351F004
:10B6E00040E050E0BA018AE50E94BC3269877A875F
:10B6F0008B879C8788E50E94A132882351F040E027
:10B7000050E0BA0188E50E94BC3269837A838B835A
:10B710009C8389E50E94A132882351F040E050E0EB
:10B72000BA0189E50E94BC326D837E838F8398873E
:10B7300085E50E945332882309F489C00E9429328A
:10B740006B017C0120E030E0A901C701B6010F9434
:10B75000695F87FF04C0F7FAF094F7F8F094F7FAFE
:10B76000F094F7F8F094CD8ADE8AEF8AF88E198E7D
:10B770001A8E1B8E1C8E8CE40E945332882309F48F
:10B780006FC00E9429326B017C0120E030E0A901EA
:10B79000C701B6010F94695F87FF04C0F7FAF09400
:10B7A000F7F8F094CD8EDE8EEF8EF8A262E070E0B6
:10B7B00082E40E940734F82E8091DA07811131C0AB
:10B7C00021E0AE014B5E5F4FBE016F5F7F4FCE0148
:10B7D00041960E94B059882321F16F2D81E00E948B
:10B7E000925A82E50E94A132882309F442C00E9445
:10B7F000253240E050E060EA71E44D875E876F8754
:10B80000788B2091DA07222361F08C012F2DAE0175
:10B81000435F5F4FBE01635E7F4FCE0149960E943A
:10B820009557A0960FB6F894DEBF0FBECDBFDF913F
:10B83000CF911F910F91FF90EF90DF90CF900895DF
:10B84000C12CD12C80E8E82E80E4F82E33CFC090B4
:10B85000CE05D090CF05E090D005F090D10572CF05
:10B86000C090D205D090D305E090D405F090D505D6
:10B870008CCF90E080E0BDCFCF92DF92EF92FF922D
:10B880000F931F93CF93DF93CDB7DEB76C970FB6AF
:10B89000F894DEBF0FBECDBF8CE40E9453328823E4
:10B8A00009F4C3C00E9429326B017C0120E030E022
:10B8B000A9010F94695F87FF04C0F7FAF094F7F8C5
:10B8C000F094F7FAF094F7F8F094C98EDA8EEB8ED4
:10B8D000FC8E8CE0EBE8F2E0DE01119601900D9217
:10B8E0008A95E1F788E50E94A1328823A1F040E023
:10B8F00050E0BA0188E50E94BC322091FB093091EA
:10B90000FC094091FD095091FE090F94085D69837F
:10B910007A838B839C8389E50E94A1328823A1F0DE
:10B9200040E050E0BA0189E50E94BC322091FB0959
:10B930003091FC094091FD095091FE090F94085D7A
:10B940006D837E838F8398878AE50E94A132882346
:10B9500051F040E050E0BA018AE50E94BC326987AC
:10B960007A878B879C87F0908517F2FAFF24F0F88E
:10B9700040E061E080E00E94B38760E080E50E94E3
:10B980001634E82E1D861E861F86188A8091DA07D7
:10B9900081113CC02E2DAE01435F5F4FBE016F5F32
:10B9A0007F4FCE0149960E94B059882379F180914A
:10B9B000D60581110F94E142FF2011F0EE2031F104
:10B9C00060E080E00E94925A898D9A8DAB8DBC8D8B
:10B9D000B0588D8B9E8BAF8BB88F198A1A8A1B8AB1
:10B9E0001C8A1D861E861F86188A8091DA07882386
:10B9F00069F010E000E020E0AE014B5E5F4FBE0159
:10BA00006F5E7F4FCE010D960E9495576C960FB6D4
:10BA1000F894DEBF0FBECDBFDF91CF911F910F9184
:10BA2000FF90EF90DF90CF900895C12CD12C80E84B
:10BA3000E82E80E4F82E45CF2F923F924F925F92EE
:10BA40006F927F928F929F92AF92BF92CF92DF922E
:10BA5000EF92FF920F931F93CF93DF93CDB7DEB793
:10BA6000E1970FB6F894DEBF0FBECDBF89AB209132
:10BA7000FC0828AB21E02093FC088091FE048D3463
:10BA800009F461C4843511F40C94BA71873409F057
:10BA900044C18091FC049091FD048A31910509F420
:10BAA000D5C108F03DC18430910508F030C1209126
:10BAB000B3088230910508F451C1213009F054C116
:10BAC00011E0029709F010E00E94D33219821A8225
:10BAD0001B821C821D821E821F82188682E50E94A4
:10BAE000A132882309F451C10E9429326B017C01E3
:10BAF00020E030E0A9010F941756882309F4EAC02A
:10BB00004090491150904A1160904B1170904C1127
:10BB100080914D1190914E11A0914F11B091501103
:10BB200088A799A7AAA7BBA78090E0089090E108F2
:10BB3000A090E208B090E3088091E4089091E508B5
:10BB4000A091E608B091E7088CA79DA7AEA7BFA774
:10BB5000A5019401C301B2010F94175681110DC0C4
:10BB60002CA53DA54EA55FA568A579A58AA59BA591
:10BB70000F941756882309F4ADC0A3019201C501A3
:10BB8000B4010F94085D20E030E040E05FE30F94E3
:10BB90007D566CA37DA38EA39FA328A539A54AA596
:10BBA0005BA56CA57DA58EA59FA50F94085D20E0E3
:10BBB00030E040E05FE30F947D562B013C0120E034
:10BBC00030E0A901C701B6010F941756881F8827D6
:10BBD000881F181709F4D0C080E090E0A0E8BFEB00
:10BBE00088A799A7AAA7BBA72CA13DA14EA15FA199
:10BBF000CA01B9010F947D564B015C01A30192016A
:10BC0000C301B2010F947D569B01AC01C501B40183
:10BC10000F94095D0F94B75F4B015C01AC019B0170
:10BC2000C701B6010F94085D6CA77DA78EA79FA7DB
:10BC3000A5019401C701B6010F94095D9B01AC01F8
:10BC40006CA57DA58EA59FA50F947D566B017C01EB
:10BC500020E030E0A9010F94695F87FD92C0C70121
:10BC6000B6010F94B75F6B017C01C301B20190581C
:10BC7000A50194010F94035E28A539A54AA55BA5EB
:10BC80000F947D56A70196010F947D562CA13DA1DE
:10BC90004EA15FA10F94095D69837A838B839C8396
:10BCA000A50194016CA17DA18EA19FA10F94035EBB
:10BCB00028A539A54AA55BA50F947D56A701960135
:10BCC0000F947D56A30192010F94095D6D837E83CD
:10BCD0008F83988720E030E0A90169817A818B8188
:10BCE0009C810F941756811164C020E030E0A901B7
:10BCF0006D817E818F8198850F941756811159C06F
:10BD00000E94394880E79FE00E9451372DC084305F
:10BD1000910509F461C0459739F10F949B2F24C018
:10BD20008A32910509F4EAC158F48C31910509F47D
:10BD3000A8C008F48EC04D9781F70E94CE7414C03D
:10BD40008B35910509F457C28C35910509F457C21A
:10BD50008A35910511F71092120906C0213021F49D
:10BD60000E94D3320E94B7F939A931110C94A3690A
:10BD70000F9444390C94A36980E090E0A0E8BFE3FD
:10BD80002FCFC12CD12C760170CF89E40E94A13233
:10BD9000882331F00E94293269837A838B839C83C4
:10BDA0008AE40E94A132882309F494CF0E942932A8
:10BDB0008DCF412FBE016F5F7F4F80EE98E00F94D3
:10BDC000DD390F94E3386093F0087093F1088093A5
:10BDD000F2089093F308C8CF80E50E94A132C12CED
:10BDE000D12C7601882321F00E94D2276B017C019F
:10BDF00083E50E94A132882361F00E94293220E06D
:10BE000030E04AE754E40F947D560F947C5E6B015A
:10BE10007C010E946ADF80911014811105C060E0EE
:10BE200086E89FE00E94A6B50F94E338C60ED71EA1
:10BE3000E81EF91E0F94E3386C197D098E099F09DD
:10BE400097FF92CF80E00E94FD4EF4CF0E94E93E22
:10BE50008BCF0F943A46811187CF8CE0E7E9F2E06F
:10BE6000DE01119601900D928A95E1F770E060E095
:10BE700080E50E94AE32BE016F5F7F4F0F948D044C
:10BE800073CF87E00E948AF3811106C060E08FE4DF
:10BE90000E941634811168CF0E946ADF1092380226
:10BEA000609148118CE40E941634982E80E00E9424
:10BEB0000D350F94E3386093F0087093F108809388
:10BEC000F2089093F30880917C0290917D02A091FA
:10BED0007E02B0917F028093CA049093CB04A0931A
:10BEE000CC04B093CD048091760290917702909328
:10BEF000C9048093C80484E690E09093770280930D
:10BF0000760281E080936C080E942BFF8AE50E94F4
:10BF10005332A82E88E50E945332182F89E50E94DB
:10BF20005332B82E181308C0B12EA11205C011E06B
:10BF3000BB24B394AA24A39482E50E94A13288234F
:10BF400009F4D2C00E9429326C8F7D8F8E8F9F8F13
:10BF500020E030E0A9010F941756882349F0111111
:10BF600003C0BB2009F494C0CE014C960F948831D5
:10BF7000112309F488C0BB2009F482C01092491132
:10BF800010924A1110924B1110924C1110924D11B7
:10BF900010924E1110924F11109250110E947AF58A
:10BFA000E5EFF7E2C590D590E590F490E9EFF7E280
:10BFB0004590559065907490A7019601C301B20118
:10BFC0000F94175687FF95C0A7019601C301B201D0
:10BFD0000F94035E9B01AC010F947D5620E030E08E
:10BFE00040E85FE30F94095D0F94B75F20E030E015
:10BFF00048E452E40F947D5669837A838B839C8353
:10C000008091511190915211A0915311B0915411FE
:10C010008CA39DA3AEA3BFA320E030E040EC5FE380
:10C02000C301B2010F947D562B013C0177FA709445
:10C0300077F8709420E030E040EC5FE3C701B60190
:10C040000F947D569058DE0111966D01ECA0FDA075
:10C050000EA11FA1A30192010E9473F40F94A900E5
:10C060001092491110924A1110924B1110924C11DA
:10C0700010924D1110924E1110924F1110925011BA
:10C0800080E00E94D1FCBB2019F081E00E94D1FC2D
:10C09000AA2019F082E00E94D1FC0E947AF58091DA
:10C0A0006B0880936C08892D0E940D358091CA041D
:10C0B0009091CB04A091CC04B091CD0480937C02EC
:10C0C00090937D02A0937E02B0937F028091C8047A
:10C0D0009091C904909377028093760283E08093D5
:10C0E00080020E9422FE40CE60E070E080E890E492
:10C0F0002BCFA3019201C701B6016ACF8091B3088B
:10C10000813009F031CE89E40E94A132082F10E07D
:10C11000882319F00E942532182F8AE40E94A13248
:10C12000F82E882339F00E942532011106C088308C
:10C1300068F005C080E0002349F0183028F08FE84F
:10C140009FE00E94513710CEF110F1CF90E1E9E469
:10C15000F1E1A0EEB8E001900D929A95E1F700238D
:10C1600091F0B4E01B02F0011124E65AF84E408130
:10C170005181628173814093E0085093E10860939C
:10C18000E2087093E308FF2091F024E08202F001BE
:10C190001124E65CF84E80819181A281B381809365
:10C1A000E4089093E508A093E608B093E70840E020
:10C1B00050E0BA0186E40E94BC326B017C0120E0B1
:10C1C00030E0A9010F94695F18168CF420E030E08C
:10C1D00040E752E4C701B6010F94035E69837A8396
:10C1E0008B839C83CE0101960E946AFCBDCD60E0EA
:10C1F00070E0CB01F3CF8FE080931209B5CD809131
:10C20000FB04882381F1893009F0AECD63EAA62EC4
:10C2100062E0B62E79E4C72E71E1D72EE12C00E062
:10C2200010E0D5018D915D010E94A132F82E882386
:10C2300061F0133011F4082FFE2C0E942932F60110
:10C240006083718382839383EF2C1F5FF4E0CF0EB2
:10C25000D11C143031F7EE2009F457C00E947AF552
:10C260000E9422FE81CD53EAC52E52E0D52EF12C3C
:10C27000E12C00E010E0D6018D916D010E94A13209
:10C28000382E8823D9F10E9429324B015C011330EA
:10C2900059F0F701E550F64F2081318142815381F9
:10C2A0000F94085D4B015C01F701E75BFE4E2081B6
:10C2B000318142815381C501B4010F94085D2B0186
:10C2C0003C012DEB37E346E855EB0F94695F87FDA2
:10C2D0000AC02DEB37E346E855E3C301B2010F94E2
:10C2E000175618165CF41330C1F4809255119092D1
:10C2F0005611A0925711B0925811032D1F5FB4E050
:10C30000EB0EF11C143009F0B6CF002309F4A8CFCE
:10C3100085E591E10E9472F1A3CFF701EF5CF64F42
:10C320005F01A301920160817181828193810F94E9
:10C33000095DD5016D937D938D939C931397812F08
:10C340000E946AF3DBCF8091FC049091FD04883752
:10C35000910511F40C94B46B08F077C28D349105FB
:10C3600009F421C708F0D3C08A31910509F443C606
:10C3700008F094C08431910509F489C508F071C0B2
:10C380008131910509F44AC508F044C0029708F0CC
:10C39000C4CC80E50E94A132C12CD12C7601882327
:10C3A00021F00E94D2276B017C0183E50E94A1321B
:10C3B000882361F00E94293220E030E04AE754E40B
:10C3C0000F947D560F947C5E6B017C010E946ADFA6
:10C3D0008091FF0490910005009709F419C50F940E
:10C3E000E6458091FC049091FD0460EB7FE0892B91
:10C3F00011F468EA7FE030E020E042E051E482E0BE
:10C400000E94F53840E0C701B6010E94565A0F94C9
:10C410001846AACC429709F080CC83E50E94A1324D
:10C42000882311F40C94EB6A0F94E3386093F008BE
:10C430007093F1088093F2089093F3080E942932D8
:10C4400020E030E04AE754E40F947D560F947C5E80
:10C450006093100270931102809312029093130262
:10C4600083CC8731910509F447C570F48531910576
:10C4700009F43EC5469709F050CC8091851782FD9E
:10C4800073CC0E94CECD70CC8831910509F449C59A
:10C49000499709F042CC0E943C5C66CC8F319105F3
:10C4A00009F44EC6D0F48C31910509F411C608F494
:10C4B000B5C58D31910509F413C64E9709F02DCC01
:10C4C0008091851783FF50CC0F94812F8091FF04BA
:10C4D000909100050F94B54447CC8934910509F437
:10C4E0004EC650F48032910509F401C6819709F0D7
:10C4F00014CC0E94384E38CC8B34910509F44FC6C9
:10C500008C34910509F009CC0F94B1012DCC8B36F8
:10C51000910509F434C708F00FC18435910509F479
:10C520007CCF40F58135910511F40C94CB6A90F4E1
:10C530008E34910509F0F1CB70E060E083E50E9454
:10C5400007348E34910509F033C60E9490DE0F94B3
:10C5500018460ACC8235910511F40C94E36A8335B0
:10C56000910509F0DACB809112098F7E8062809369
:10C570001209FACB8836910509F49EC608F09CC0D2
:10C580008535910511F40C942E6B8C35910509F0CD
:10C59000C4CB0E941C4987FDE7CB8091F70484FD42
:10C5A0000AC08091F90487FD06C08091FA04837067
:10C5B00011F40C945C6B23EAC22E22E0D22E30E000
:10C5C000E32E31E1F32E10E0D6018D916D010E9432
:10C5D000A132882309F466C0133011F00C94536B18
:10C5E0000E9429324B015C0120E030E040EA51E436
:10C5F0000F94175687FF4EC0A5019401609120113A
:10C600007091211180912211909123110F94035E5A
:10C610002B013C01AC019B0160912D0A70912E0A07
:10C6200080912F0A9091300A0F947D5660932D0AC5
:10C6300070932E0A80932F0A9093300AA3019201DF
:10C6400060913011709131118091321190913311BC
:10C650000F947D5660933011709331118093321195
:10C66000909333116091190A70911A0A80911B0AF4
:10C6700090911C0A0F941C56A30192010F947D56B1
:10C680000F947C5E6093190A70931A0A80931B0AB8
:10C6900090931C0A8092201190922111A092221155
:10C6A000B09223111F5FF4E0EF0EF11C143009F07B
:10C6B0008BCF0E9446DF58CB8936910509F434C6EA
:10C6C0008A36910509F029CB80E50F94BC30F82E0D
:10C6D00091E0981708F448CB81E40E9453326091AE
:10C6E000390A062F10E0811102C00FEF10E089E433
:10C6F0000E94A132882311F40C94EC710E94013243
:10C7000090E01816190614F481E090E026E0289FC6
:10C71000F001299FF00D1124EC54F74F048115818D
:10C72000EF2DF0E0E75CF54F0F3F110519F010F029
:10C730000FEF10E0008318CB8137910509F481C613
:10C7400008F068C08E36910509F427C608F059C074
:10C750008C36910509F408CB8D36910509F0DDCAB8
:10C760008091FF1083FD00CB0E941C49F82E87FDAD
:10C77000FBCA89E40E94A132882311F40C94DA7177
:10C780000E94013290E01816190614F481E090E03E
:10C7900026E0289FF001299FF00D1124EC54F74F5B
:10C7A0008081918110E00E94ECDE61E081E00F94D5
:10C7B000274A209181163091821680917F169091A0
:10C7C0008016821793070CF0A6C581EA90E19F932B
:10C7D0008F938CEA90E19F938F931F920E948BB569
:10C7E0000F900F900F900F900F9001E00F94F04971
:10C7F000002309F4B9CA40E0612F8F2D0F945B0D1F
:10C80000B3CA8F36910509F4DBC58037910509F469
:10C81000ABCA83CA8537910509F45BC758F48237E0
:10C82000910509F44EC78337910509F076CA0E9435
:10C8300078379ACA8637910509F45DC7873791051D
:10C8400009F06BCA0E9408FF8FCA8A39E1E09E078F
:10C8500009F48ACA08F03DC18D3C910511F40C948D
:10C86000BD6C08F09FC08B39910509F46DC638F591
:10C870008D37910509F40FCE58F48937910509F0E9
:10C880004CCA10926C0810926B080E942BFF6CCA65
:10C890008C38910509F4F4C58139910509F03DCA38
:10C8A00070E060E083E50E940734823008F464C7DA
:10C8B0000E94394880E091E10E94513755CA893C75
:10C8C000910509F4C5C7A8F58E3B910509F4FEC58D
:10C8D000883C910509F021CA0E941C49182F87FD48
:10C8E00043CA0091300984E40E94A132F82E8823C3
:10C8F000B9F00E9429324B015C0120E030E0A9012F
:10C900000F941756882309F4A1C724E01202F001FE
:10C910001124E45DF64F80829182A282B3820F2DB2
:10C92000602F83E50E941634809330090E9419C756
:10C930001BCA8B3C910509F4B5C78C3C910509F0E5
:10C94000ECC98091F80487FDD0C78091F9048E70FE
:10C9500009F0CBC7409134115091351160913611D7
:10C960007091371185E291E10E94C93940913811E7
:10C970005091391160913A1170913B1182E291E12D
:10C980000E94C93940913C1150913D1160913E1176
:10C9900070913F118FEB9CE20E94C9398AE00E949E
:10C9A0001837E2C98C3221E0920711F40C94DF6D44
:10C9B00008F04CC08C3D910511F40C94116D58F4A5
:10C9C0008E3C910509F4DDC7833D910509F0A5C9A9
:10C9D0000E944149C9C98D3D910511F40C94546DD3
:10C9E0008232914009F099C98AE50E94A1328823D8
:10C9F00011F40C94AB6D0E94293220E030E040E04D
:10CA000050EC0F94175687FF02C00C94CC6D0E9417
:10CA1000293220E030E040E050E40F94695F1816BE
:10CA200014F40C94D26D0E94293220911C11309183
:10CA30001D1140911E1150911F110F947D560F949E
:10CA4000755ECB010F9497390C94B16D8F32B1E0C4
:10CA50009B0711F40C940C6F78F58D32F1E09F0771
:10CA600011F40C94F56D8E32914009F056C983E5AE
:10CA70000E945332182F882369F00E9425329C01AE
:10CA8000909386028093850291E0232B09F090E039
:10CA900090934B0A80E50E945332882311F40C9442
:10CAA000EA6E2091850230918602232B11F00E94BC
:10CAB000153280934B0A58C9803331E0930711F443
:10CAC0000C94766E8039914009F027C90E946ADF84
:10CAD0004BC9883FB1E09B0711F40C946F7008F0CC
:10CAE0006DC08C3AF1E09F0711F40C94446F08F08C
:10CAF0003EC08D3931E0930711F40C949D7150F5CF
:10CB00008C39914009F009C98091F704887811F0B7
:10CB10000C94106F8091F904867011F00C94106FD2
:10CB20000E9418498EEC91E10E9451378091550284
:10CB30000E94AB39409151025091520260915302D0
:10CB4000709154028EEA91E10E94C9398AE00E94F4
:10CB500018370AC9843AE1E09E0711F40C94406F3B
:10CB6000853A914009F0D9C80E943D48FDC8853FEB
:10CB700021E0920711F40C94677068F4863EA1E0FE
:10CB80009A0711F40C94F56F843F914009F0C5C8E1
:10CB90000E9443DBE9C8863FE1E09E0711F40C9454
:10CBA0006B70873F914009F0B8C861E083E50E944F
:10CBB000163491E089270F94E90ED6C88C3623E00D
:10CBC000920709F4D1C808F0D3C08B35A2E09A07C8
:10CBD00011F40C94927068F48C30E2E09E0711F42A
:10CBE0000C9481708835924009F097C80E942C5BA4
:10CBF000BBC88D3B22E0920711F40C9412718E3B5E
:10CC0000924009F08AC80E941C49182F87FDACC8C1
:10CC10008AE50E94A132812C912C90E2A92E91E408
:10CC2000B92E882341F040E050E0BA018AE50E9425
:10CC3000BC324B015C01412F64E083E00E94B3876A
:10CC400020E030E0A901C501B4010F94695F181616
:10CC50007CF580E090E0A0EAB0E489839A83AB831E
:10CC6000BC83209151113091521140915311509138
:10CC70005411C501B4010F94095D6B017C0120E0E2
:10CC800030E048EC53E40F94175687FD06C0C12CE2
:10CC9000D12C88ECE82E83E4F82ECC8EDD8EEE8E3F
:10CCA000FF8EBE016F5F7F4FCE014C960E942BF529
:10CCB00085E50E945332882311F40C9416710E946A
:10CCC00029326B017C0120E030E0A901C701B601E7
:10CCD0000F94695F87FF04C0F7FAF094F7F8F094B7
:10CCE000F7FAF094F7F8F094C982DA82EB82FC82CA
:10CCF00044E061E0CE0101960E94035920E030E05B
:10CD0000A901C501B4010F94695F18165CF580E0B4
:10CD100090E0A0EAB0E489839A83AB83BC83A50149
:10CD20009401609151117091521180915311909121
:10CD300054110F94085D6B017C0120E030E0A901E3
:10CD40000F94695F18161CF0C12CD12C7601CC8E83
:10CD5000DD8EEE8EFF8EBE016F5F7F4FCE014C9653
:10CD60000E942BF5109211050E94CA860C94B45EA5
:10CD7000873EA3E09A0711F40C948D71C8F48438AF
:10CD8000E3E09E0711F40C942271803A934011F075
:10CD90000C948D5E2091FF043091000590918517D1
:10CDA000926090938517C9010F948F460C94B45EDE
:10CDB000883E23E0920711F40C94B671893E9340AB
:10CDC00011F00C948D5E0F945F4581110C94B45E4C
:10CDD0000E942B340F941D450F94B7006D337105DD
:10CDE0008105910520F081E892E10E9440728DE773
:10CDF00092E10E94407284EE8093090589E692E1F7
:10CE00000E94513785E692E10E9440720C94B45E14
:10CE100060E088EB9FE00E94A6B5E3CA8091F7042A
:10CE200084FD17C08091F90487FD13C08091FA0436
:10CE3000837079F460E08BEC9FE00E94A6B55F9868
:10CE40008A988091080181708093060112980C9451
:10CE5000B45E88E50E94533281115F9889E50E9493
:10CE6000533281118A988AE50E945332882329F02F
:10CE70008091080181708093060185E40E945332FD
:10CE8000882311F40C94B45E12980C94B45E8091D3
:10CE9000851783FF25C083EE9FE00E945137809164
:10CEA000851783FF17C086EA97E10E94AFD58BE113
:10CEB000E6EAF7E1DE01119601900D928A95E1F71D
:10CEC00070E060E0CE0101960F94D809CE01019682
:10CED0000E94533484ED9FE00E9451370C94B45E5D
:10CEE0000E94184984EF9FE00E9451370C94B45E71
:10CEF0000E940FD50C94B45E8091FF0490910005C0
:10CF0000FC012191222331F02032D9F7DF01119762
:10CF10001C92F7CF60E00F94D846109209050C944C
:10CF2000B45E83E50E94A132882321F00E94F3279A
:10CF30000E94262684E50E94A1328823A9F00E943F
:10CF4000F3276B017C010F945E01C092C605D0925D
:10CF5000C705E092C805F092C905CD28CE28CF2894
:10CF600019F081E0809311098091DA078823F9F0A4
:10CF700080E090E0A0EAB1E489839A83AB83BC832C
:10CF80001C8E1D8E1E8E1F8E18A219A21AA21BA205
:10CF900010E000E020E0AE014F5F5F4FBE01645E35
:10CFA0007F4FCE0180960E9495570C94B45E0E94EC
:10CFB0009C36882381F00F944F440E94C03687E846
:10CFC00099E00F94F743109242121092431210927C
:10CFD00044121092451261E08AE29EE10E949C3860
:10CFE00042EF5DE16EEF7FE085E00F94B3300F9488
:10CFF00018460C94B45E8091851783FD02C00C9492
:10D00000B45E83E50E94A132882311F40C94B45ECF
:10D010000E94F3270E9426260C94B45E83E40E94AB
:10D020005332882361F184E190E10E94513780916D
:10D03000ED188823F9F0BE016F5F7F4F8AEE98E10B
:10D040000E9475D5CE0101960E949ED1CE01019617
:10D050000F94B8458091CD13882339F080E20E9467
:10D0600018378DEC93E10E949ED18AE00E94183718
:10D070000C94B45E8AE090E10E945137F6CF83E5CC
:10D080000E94A132882301F10E940132182F8C33B3
:10D0900008F08CE38093D2040F94E3386B017C0199
:10D0A000212F30E0A8EEB3E00F94AF5CC60ED71E80
:10D0B000E81EF91EC092CE04D092CF04E092D004B4
:10D0C000F092D1040C94B45E0F94BE430C94B45E01
:10D0D0008091FF04909100050F948F460C94B45EEC
:10D0E000809185178E7F809385170C94B45E809114
:10D0F000851782FD0E946ADF8091851783FD02C03B
:10D100000C94B45E60E080E50E941634182F682FFE
:10D110008091FF04909100050F94D84683E50E940A
:10D12000A132882321F00E94F3270E9426260F9423
:10D130004F4411110C94B45E0E94C0360C94B45E3E
:10D140000F94B7006C8F7D8F8E8F9F8FBE016F5FA6
:10D150007F4FCE014C960E94872CCE0101960F94F2
:10D16000E6450E941849BE016F5F7F4F83E290E160
:10D170000E942E4E8AE00E9418370C94B45E80E51F
:10D180000E945332882311F40C94B45E0E94013241
:10D19000853608F084E6809309050C94B45E0E94FD
:10D1A000C0360C94B45E81E00F94E9000C94B45E38
:10D1B0008EE890E10E94513760915B0870915C08A5
:10D1C00085E890E10E94B73960915D0870915E0832
:10D1D00088E790E10E94B73960915B0870915C0824
:10D1E00080915D0890915E08681B790B8091110910
:10D1F000815021E030E0823010F030E020E0621B0E
:10D20000730B8DE690E10E94B7398AE00E941837CF
:10D2100085E690E10E94513780915F089091600807
:10D22000A0916108B09162088C8F9D8FAE8FBF8FE7
:10D23000BE016F5F7F4FCE014C960E94872CBE01CE
:10D240006F5F7F4F88E590E10E942E4E80916308CA
:10D2500090916408A0916508B09166088C8F9D8FAD
:10D26000AE8FBF8FBE016F5F7F4FCE014C960E9485
:10D27000872CBE016F5F7F4F88E490E10E942E4EA5
:10D2800020E030E04AE754E4609167087091680854
:10D290008091690890916A080F94035EAB01BC010C
:10D2A00080E390E10E94C9398DE60E9418378AE038
:10D2B0000E9418370C94B45E8091FF1083FF02C067
:10D2C0000C94B45E0E941C4987FF02C00C94B45EAB
:10D2D00089E40E94A132882311F40C94CF710E943A
:10D2E000013290E01816190614F481E090E026E06F
:10D2F000289FF001299FF00D1124EC54F74F8081F5
:10D3000091810E94ECDE61E080E00F94274A0F9447
:10D31000F0490C94B45E86E990E1112309F457CAF0
:10D32000012F64CA182F62CA0E941C49182F87FD5A
:10D330000AC081EB90E10E945137812F0F94630B5B
:10D340008AE00E94183788A98093FC08E1960FB6FE
:10D35000F894DEBF0FBECDBFDF91CF911F910F912B
:10D36000FF90EF90DF90CF90BF90AF909F908F9005
:10D370007F906F905F904F903F902F90089580E541
:10D380000F94BC30823010F00C94B45EE82FF0E0C3
:10D39000E75CF54F10820C94B45E8EE40E94A132DB
:10D3A000882311F40C94B45E0E94F3276093DB1180
:10D3B0007093DC118093DD119093DE110C94B45EB8
:10D3C00083E50E945332882329F083E50F94BC3013
:10D3D0008093FF100E94184982EC90E10E9451371F
:10D3E0008091FF10882351F110E000E020E080914F
:10D3F000FF1090E0B0E0A0E0002E04C0B695A79525
:10D40000979587950A94D2F780FF12C0FF24F39472
:10D41000F20E222319F08CE20E941837F801EE0F69
:10D42000FF1FE854FF4E859194910E9451372F2D94
:10D430000F5F1F4F05301105D1F617CE84EB90E139
:10D440001BCE83E50E94A132882369F00E9401323D
:10D450008D3320F480930F020C94B45E8CE38093A0
:10D460000F020C94B45E0E94184960910F0289EC7F
:10D4700090E10E94C1398AE00E9418370C94B45E92
:10D480008091FF1083FF02C00C94B45E89E40E9477
:10D49000A132882309F4ACC70E94013290E018162B
:10D4A000190614F481E090E026E0289FF001299FFE
:10D4B000F00D1124EC54F74F828193810E94F631D4
:10D4C00061E080E00F94274A0C94B45E8091FF10D5
:10D4D00083FF02C00C94B45E89E40E94A1328823C9
:10D4E00009F490C70E94013290E01816190614F44E
:10D4F00081E090E026E0289FF001299FF00D1124A3
:10D50000EC54F74F8281938110E00E94F63160E085
:10D5100081E00F94274A20911D0930911E098091C6
:10D520001B0990911C09821793071CF48FED90E161
:10D5300002C080ED90E160E00E94A6B560E0812F1E
:10D540000F94D60B0C94B45E83E50E94A13288231D
:10D5500011F40C94B45E0E940132182F8C3308F041
:10D560008CE38093D7040F94E3386B017C01212F67
:10D5700030E0A8EEB3E00F94AF5CC60ED71EE81EF5
:10D58000F91EC092D304D092D404E092D504F09254
:10D59000D6040C94B45E0E94CCD70E947BDF81E05D
:10D5A0000F94E9000E94D33668EE73E080E090E0CB
:10D5B0000E944D360E94952260E08EEE90E10E941E
:10D5C000A6B50C94B45E809112098F7D8061809322
:10D5D00012090C94B45E8091F70484FD0CC0809114
:10D5E000F90487FD08C08091FA04837021F40E9439
:10D5F0007BDF0C94B45E0E946ADF88E50E945332A0
:10D60000882331F05F9A80916E088E7F80936E0838
:10D6100089E50E945332882331F08A9A80916E08FE
:10D620008D7F80936E088AE50E945332882359F0DB
:10D6300080910801809581708093060180916E0829
:10D640008B7F80936E0885E40E945332882311F407
:10D650000C94B45E0E9493220C94B45E83E50E9405
:10D660005332882311F40C94B45E0F94E338609322
:10D67000F0087093F1088093F2089093F3080E94E9
:10D68000293220E030E04AE754E40F947D560F94AD
:10D690007C5E6093D8047093D9048093DA049093ED
:10D6A000DB040C94B45E0E942932F701648B758B05
:10D6B000868B978B0C94526381E00F94462F0C94C9
:10D6C000B45E0F94E12E85ED96E10E9499DA0C94F8
:10D6D000B45E8091FF0490910005009741F0DC0159
:10D6E0002C91222321F00F94E6450C94B45E0F9404
:10D6F00018460C94B45E0091FF041091000594E06C
:10D70000F12C40E09150F9F0F8018081282F2B7F17
:10D71000213499F421812133B1F4813411F185341C
:10D7200009F441E098012E5F3F4F89012F5F3F4F81
:10D73000F80180818032C9F3E5CF803521F4818101
:10D7400080538A3078F341110E941849FF2021F05C
:10D750008DEF90E10E945137C8010E941F370C9451
:10D76000B45EFF24F394DECF20936C0820936B0803
:10D770000E942BFF0C94B45E8C01112788E40E9458
:10D78000A1328823C1F00E9425328A3A91050CF417
:10D790004BC00E9425328D3291400CF048C00E944F
:10D7A000253226E0209FF001219FF00D1124EC543A
:10D7B000F74F9183808382E40E94A1328823A9F0ED
:10D7C0000E9425320597B4F10E9425328D389105CB
:10D7D000A4F50E94253226E0209FF001219FF00D44
:10D7E0001124EC54F74F9383828386E40E94A13284
:10D7F000882311F40C94B45E0E94253297FD20C05A
:10D800000E9425328F3F910509F0ECF40E942532E9
:10D8100026E0209FF001219FF00D1124EC54F74FDA
:10D82000958384830C94B45E8AEA90E0BACF8CE24C
:10D8300091E0B7CF85E090E0CECF8CE890E0CBCF01
:10D8400090E080E0E5CF8FEF90E0E2CF80E06CC821
:10D850000E941C4987FF02C00C94B45E03EA12E0E8
:10D8600080E0E82E81E1F82E97EAC92E92E0D92EC9
:10D87000D8018D918D010E945332882359F00E9466
:10D8800029320F947C5EF7016083718382839383D6
:10D890000E94F8DEF4E0EF0EF11CC016D10641F74D
:10D8A0000C94B45E0E941C4987FF02C00C94B45EC5
:10D8B000B3EAEB2EB2E0FB2E10E000E0D7018D9131
:10D8C0007D010E945332882349F00E942932F801D9
:10D8D000E050FF4E64A375A386A397A30C5F1F4F70
:10D8E0000031110559F70C94B45E83E50E94A13212
:10D8F000882391F00E94293260933411709335117E
:10D90000809336119093371160933C1170933D11C1
:10D9100080933E1190933F1180E50E94A1328823AD
:10D9200051F00E9429326093341170933511809325
:10D9300036119093371182E50E94A132882351F06D
:10D940000E942932609338117093391180933A11F3
:10D9500090933B1184E50E94A132882311F40C942A
:10D96000B45E0E94293260933C1170933D11809304
:10D970003E1190933F110C94B45E0E9413380C94A6
:10D98000B45EADE3EA2EA9E0FA2E10E088E5810F3F
:10D990000E945332882351F00E942932F70160839C
:10D9A000718382839383812F0E946AF31F5FF4E067
:10D9B000EF0EF11C133051F78091F90487FF02C07C
:10D9C0000C9430618091FA04837011F00C943061F2
:10D9D00040913D0950913E0960913F097091400985
:10D9E00085E391E10E94C939409141095091420972
:10D9F000609143097091440989E891E40E94C93912
:10DA00004091450950914609609147097091480934
:10DA100086E891E40E94C9398AE00E9418370C9484
:10DA2000B45E82E40E945332882341F080917602F2
:10DA300090917702909315028093140282E50E94E0
:10DA40005332882341F080911402909115029093F3
:10DA500077028093760283E50E94A132882331F019
:10DA60000E94253290937702809376028091F7048A
:10DA70009091F804A091F904B091FA04892B8A2BB3
:10DA80008B2B11F00C94B45E60917602709177024A
:10DA90008CE391E10E94DF3E85E20E9418378AE024
:10DAA0000E9418370C94B45E0E941C49082F87FF0F
:10DAB00002C00C94B45E83E50E94A132002E000CDB
:10DAC000110B7801EE0CFF1C882359F10E942532BE
:10DAD000F701EB5CFD4F91838083000F111F000F56
:10DAE000111F98012F573D4F7901BC01990F880BE9
:10DAF000990B0F941E562AE037ED43E25CE30F9436
:10DB00007D560E531A4FD8012D913D914D915C9148
:10DB10000F947D56F70160837183828393830C9405
:10DB2000B45E0E94184985E40E94183780E3800F94
:10DB30000E941837F701EB5CFD4F6081718180E432
:10DB400091E10E94DF3E85E20E9418378AE00E9440
:10DB500018370C94B45E83E50E94A13281110C94B5
:10DB6000FB648091F90487FD23C08091FA048370DF
:10DB7000F9F40E9418494091D7065091D806609157
:10DB8000D9067091DA0688E491E10E94C9398AE0E9
:10DB90000E9418370C94B45E60E070E080E090EC76
:10DBA0000C94156560E070E080E090E40C941565DD
:10DBB00082E50E9453328111DCCF0C94B45E64E0A4
:10DBC00071E083E50E94AE328C0168EE73E080E57F
:10DBD0000E94AE328938F3E19F0710F088E893E1A4
:10DBE000B8010E945E800C94B45E85E40F94BC3052
:10DBF000811174C080E50E945332882351F00E9445
:10DC000029326093841670938516809386169093BC
:10DC1000871689E40E945332882381F00E942932BA
:10DC20002CEA35EC47E25EE30F947D56609388164C
:10DC30007093891680938A1690938B1684E40E94C1
:10DC40005332882381F00E9429322CEA35EC47E2D6
:10DC50005EE30F94035E60938C1670938D16809331
:10DC60008E1690938F160E941849409184165091F9
:10DC7000851660918616709187168DE591E10E9458
:10DC8000C9392CEA35EC47E25EE360918816709161
:10DC9000891680918A1690918B160F94035EAB01C2
:10DCA000BC0189E591E10E94C9392CEA35EC47E2D3
:10DCB0005EE360918C1670918D1680918E16909116
:10DCC0008F160F947D56AB01BC0185E591E10E9452
:10DCD000C9398AE00E9418370C94B45E0E94394812
:10DCE00081E691E10E9451370C94B45E80E50E9478
:10DCF0005332882351F00E94293260932009709397
:10DD00002109809322099093230989E40E945332C8
:10DD1000882381F00E9429322CEA35EC47E25EE349
:10DD20000F947D56609324097093250980932609EA
:10DD30009093270984E40E945332882381F00E9443
:10DD400029322CEA35EC47E25EE30F94035E6093E0
:10DD500028097093290980932A0990932B090E941E
:10DD60001849409120095091210960912209709130
:10DD700023098BE791E10E94C9392CEA35EC47E28F
:10DD80005EE36091240970912509809126099091A4
:10DD900027090F94035EAB01BC0187E791E10E9464
:10DDA000C9392CEA35EC47E25EE3609128097091AD
:10DDB000290980912A0990912B090F947D56AB0176
:10DDC000BC0183E791E10E94C9398AE00E941837BB
:10DDD0000C94B45E11110C94B45E0E9418498BE946
:10DDE00091E10E94513780914B0A882391F083E89A
:10DDF00091E10E94513760918502709186028AE814
:10DE000091E10E94DF3E86E891E10E9451370C9437
:10DE1000B45E8FE791E1EDCF0E94EB390C94B45ED4
:10DE200088E40E945332882321F00E9415328093A7
:10DE3000DC0482E50E945332082F83E50E945332AE
:10DE4000182F011102C0882341F00E948022112363
:10DE500021F00E9415328093550284E40E945332CF
:10DE6000882311F40C94B45E0E942932609351020D
:10DE70007093520280935302909354020C94B45EB8
:10DE80000E94304A0C94B45E0F943A4681110C946F
:10DE9000B45E74ECC72E77E2D72E29E431E13DA3BE
:10DEA0002CA3CE0101961C017C0110E000E0F601DC
:10DEB0006591759185919491ACA1BDA18D909D9036
:10DEC000AD90BD90BDA3ACA3A50194010F94085DD6
:10DED0002B013C01F701408251826282738220E073
:10DEE00030E040EA51EC0F94695F87FD0AC020E002
:10DEF00030E040EA51E4C301B2010F9417561816FE
:10DF000084F4F801E454FF4BE4911E1654F4B7FA7C
:10DF1000B094B7F8B094D7018D929D92AD92BC9217
:10DF20001397F70181909190A190B1907F0120E02B
:10DF300030E040EA51ECC501B4010F94695F87FD00
:10DF40003FC020E030E040EA51E4C501B4010F9445
:10DF500017561816ACF10F5F1F4FF4E0CF0ED11C0F
:10DF60000330110509F0A3CF6DE3E62E69E0F62E2C
:10DF700010E0F10181919191A191B1911F01F701FF
:10DF800081939193A193B1937F01812F0E946AF3B2
:10DF90001F5F133071F70E9422FE60E08FED91E168
:10DFA0000E94A6B563E972E084E690E00E945E807C
:10DFB0006AEB72E084E690E00E945E800C94B45EAE
:10DFC0000E9439488DEF91E10E94513761E08FEE58
:10DFD00091E10E94A6B50E94CA8668E270E088ECD2
:10DFE00090E00E945E800C94B45E84E50E945332FF
:10DFF0008823A1F010920B0510920C0510920D05CC
:10E0000010920E0510920F058FEF0E94342661E0EA
:10E0100070E084E50E94073480930F0583E50E9439
:10E020005332882321F00E9425320E94342683E453
:10E030000E945332882331F080912302803210F401
:10E040000E94CE3480E50E945332882331F00E9432
:10E050002532803210F40E94CE3485E50E9453327E
:10E06000882311F40C94B45E0E942532803210F0A3
:10E070000C94B45E41E050E060E070E0082E04C013
:10E08000440F551F661F771F0A94D2F7409550958D
:10E090006095709500910B0510910C0520910D0570
:10E0A00030910E05402351236223732340930B05C7
:10E0B00050930C0560930D0570930E05909123020B
:10E0C00089130C94B45E1092FE100C94B45E0F94FD
:10E0D0002D160C94B45E0E9436FF0C94B45E20930F
:10E0E000DB060F9421161092DB06882311F40C94A2
:10E0F000B45E0E9418498BE192E10E9451370C9462
:10E10000B45E8091851782FF05C080648093851777
:10E110000C94B45E83FD02C00C94B45E0F94812F06
:10E120000C94B45E0E941C49082F87FF02C00C9417
:10E13000B45E85E50E945332882359F10E9429324A
:10E140004B015C01E02E002E000CFF0820E030E0C7
:10E15000A9010F94695F87FF04C0B7FAB094B7F8BC
:10E16000B09420E030E84BE354E4C501B4010F94CF
:10E17000695F970153E0220F331F5A95E1F722534D
:10E180003A4F1816D4F1D9018D929D92AD92BC925E
:10E1900013978CE40E945332882311F40C94B45EDC
:10E1A0000E9429326B017C01002E000C110B20E033
:10E1B00030E0A9010F94695F87FF04C0F7FAF0947B
:10E1C000F7F8F09420E030E84BE354E4C701B601DF
:10E1D0000F94695F980143E0220F331F4A95E1F7DE
:10E1E00022533A4F18169CF0D9011496CD92DD9225
:10E1F000ED92FC9217970C94B45E80E090E8ABE34C
:10E20000B4E4F90180839183A283B383C2CF80E019
:10E2100090E8ABE3B4E4F90184839583A683B783E4
:10E220000C94B45E0E949C560C94B45E28E01202DA
:10E23000F0011124E253FA4FC080D180E280F380D4
:10E240000C946366A090310AB090320AC090330AF1
:10E25000D090340A8BE40E94A132882339F10E94C5
:10E2600029327B018C0120E030E0A9010F94695F25
:10E2700087FD0AC020E030E040E251E4B701C80168
:10E280000F9417561816A4F48FE30E9418378BE4E6
:10E290000E94183781E392E10E94513789E292E1AE
:10E2A0000E94513786E292E10E9451377501860142
:10E2B0009701A801B501C6010F941756882361F094
:10E2C0000E946ADFC701D8018093310A9093320A15
:10E2D000A093330AB093340A8091F7049091F80424
:10E2E000A091F904B091FA04892B8A2B8B2B11F0A1
:10E2F0000C94B45E0E9418494091310A5091320A40
:10E300006091330A7091340A85E492E10E94C93920
:10E310008AE00E9418370C94B45E81E08093B308C1
:10E320001092651460E083E50E94163481110C940C
:10E33000B45E0F94882D0C94B45E83E50E94533232
:10E34000882341F00E9415328093D6050E94333411
:10E350000C94B45E0E94184980E592E10E94513706
:10E360008091D6050E94AB390C94B45E0E94B272C3
:10E370000C94B45E1091FC040F94E3386093F008A1
:10E380007093F1088093F2089093F308112311F42D
:10E390000C94B45E812F0E9482D70C94B45E83E506
:10E3A0000E94A132882311F40C9487690E942532BF
:10E3B0000C94816983E50E94A132182F811108C055
:10E3C00082E50E94A132082F882311F40C949269EF
:10E3D0000E9425320C94D36383E50E94A1328823E6
:10E3E00011F40C9490630E94F3278B010C949063BA
:10E3F00083E50E94A132882311F40C94B45E0E943C
:10E4000025325CC883E50E94A132182F811107C014
:10E4100082E50E94A132882311F40C94B45E0E941C
:10E42000253273C8DF92EF92FF920F931F93CF9321
:10E43000DF93EC01E090FE08F090FF088AE0D82E10
:10E440006AE070E0CE010F945E608C01009711F0DD
:10E45000FC011082CE010E94662D81E00E941C5DAD
:10E460000115110519F0E801D992EACFC701DF9132
:10E47000CF911F910F91FF90EF90DF900C94662D3C
:10E480004F925F926F927F928F929F92AF92BF92C4
:10E49000CF92DF92EF92FF920F931F93CF93DF9370
:10E4A000CDB7DEB77C014DB65EB66090FE087090C9
:10E4B000FF088DB69EB66AE070E0C7010F94525512
:10E4C0006C018C010E191F09892B21F4C7010F94CF
:10E4D00064558C01C80101962DB73EB7281B390B36
:10E4E0000FB6F8943EBF0FBE2DBF8DB79EB70196F5
:10E4F0005C01A801B7010F948555F501E00FF11FEC
:10E500001082C5010E94662D81E00E941C5DC1142D
:10E51000D10451F076019FEFE91AF90A0FB6F89489
:10E520009EBE0FBE8DBEC5CF0FB6F8949EBE0FBE69
:10E530008DBEC3010E94662D0FB6F8945EBE0FBE5D
:10E540004DBEDF91CF911F910F91FF90EF90DF9023
:10E55000CF90BF90AF909F908F907F906F905F9083
:10E560004F9008954F925F926F927F928F929F92F9
:10E57000AF92BF92CF92DF92EF92FF920F931F93D1
:10E58000CF93DF93CDB7DEB7C059D1090FB6F8945A
:10E59000DEBF0FBECDBF0E944134882369F083E502
:10E5A0000E945332882301F120E040E070E060E0F7
:10E5B00084EF96E80E946483C057DF4F0FB6F8944B
:10E5C000DEBF0FBECDBFDF91CF911F910F91FF90A6
:10E5D000EF90DF90CF90BF90AF909F908F907F9003
:10E5E0006F905F904F90089583E40E945332882388
:10E5F00019F00E94E986E0CF8090F0099090F1092F
:10E60000A090F209B090F3098091F90980FF05C04C
:10E610009091FF1098609093FF1086958170809381
:10E620004B0A82E59FE00E94407280917F099091A1
:10E6300080099E012F5F3F4F7901009799F09F93CA
:10E640008F9389E49FE09F938F933F932F930F9431
:10E65000AE55C7010E9412720F900F900F900F904D
:10E660000F900F9080917D0990917E09009799F00D
:10E670009F938F9380E49FE09F938F93FF92EF92FD
:10E680000F94AE55C7010E9412720F900F900F9019
:10E690000F900F900F906E0131E8C30ED11C609166
:10E6A0005C0970915D0980915E0990915F09860116
:10E6B00023E041E00F94E4509F938F938EE29FE01C
:10E6C0009F938F93FF92EF920F94AE55C7010E94D4
:10E6D000127286E29FE00E94407287E080936E088B
:10E6E0008093B9050F900F900F900F900F900F909F
:10E6F000809178098823F9F06091790970917A09FD
:10E7000080917B0990917C0923E041E00F94E450D3
:10E710009F938F938DE19FE09F938F93FF92EF9252
:10E720000F94AE55C7010E9412720F900F900F9078
:10E730000F900F900F90809181098823A1F01F9274
:10E740008F931F921F9280E19FE09F938F93FF9280
:10E75000EF920F94AE55C7010E9412720FB6F89453
:10E76000DEBF0FBECDBF809182098823A9F01F9222
:10E770008F931F9281E08F9380E19FE09F938F930F
:10E78000FF92EF920F94AE55C7010E9412720FB61E
:10E79000F894DEBF0FBECDBF40908309509084092E
:10E7A000609085097090860920E030E0A901C301DE
:10E7B000B2010F941756811104C08091F90982FFAC
:10E7C00020C0860121E041E0C301B2010F94E45072
:10E7D0009F938F938091F90982FB882780F91F927C
:10E7E0008F9383E09FE09F938F93FF92EF920F941C
:10E7F000AE55C7010E9412720FB6F894DEBF0FBE6D
:10E80000CDBF60914E0970914F0980915009909150
:10E8100051098E010F581F4F23E041E00F94E4503F
:10E82000782E692E60914A0970914B0980914C09AC
:10E8300090914D09860123E041E00F94E4506F92DE
:10E840007F929F938F9382EF9EE09F938F93FF928F
:10E85000EF920F94AE55C7010E9412726091520957
:10E8600070915309809154099091550923E041E03A
:10E870000F94E45087EE9EE00E944072DF92CF92A8
:10E880008DED9EE09F938F93FF92EF920F94AE5584
:10E89000C7010E94127280915B098F9380915A097F
:10E8A0008F9386ED9EE09F938F93FF92EF920F944C
:10E8B000AE55C7010E9412726091560970915709B6
:10E8C000809158099091590923E041E00F94E45058
:10E8D0009F938F938CEC9EE09F938F93FF92EF9288
:10E8E0000F94AE55C7010E9412728CE0E0E6F9E089
:10E8F000ADE3B9E001900D928A95E1F78CE0ECE68A
:10E90000F9E0A1E3B9E001900D928A95E1F780E08A
:10E910000E946AF381E00E946AF382E00E946AF337
:10E920008091F8098093120981E08093D6050E94B6
:10E93000333487E899E09F938F9381E598E39F9321
:10E940008F93FF92EF920F94AE550FB6F894DEBFFF
:10E950000FBECDBFC7010E9412728091F7098F933D
:10E960008091F6098F938091F5098F938091F40936
:10E970008F93BF92AF929F928F928EEB9EE09F9368
:10E980008F93FF92EF920F94AE55C7010E941272BF
:10E990000FB6F894DEBF0FBECDBF0ECE4F925F9282
:10E9A0006F927F928F929F92AF92BF92CF92DF929F
:10E9B000EF92FF920F931F93CF93DF9300D000D07D
:10E9C0001F921F92CDB7DEB783E50F94BC3086301F
:10E9D00028F083E19EE00E9451373FC0833009F464
:10E9E00078C1B0F4813021F1823009F450C080E068
:10E9F0009EE00E9451370E9408368823A1F0809142
:10EA000048110E94AB390E942C390E9422FE25C079
:10EA1000843009F4A4C1853051F780E00E940D359F
:10EA20000E94FA34F2CF82EF9DE00E945137EDCF81
:10EA30000E94FA3410920E0210920D0280910A0583
:10EA4000811125C08EE40E94533281111DC080EED9
:10EA50009DE0909371088093700828960FB6F89403
:10EA6000DEBF0FBECDBFDF91CF911F910F91FF9001
:10EA7000EF90DF90CF90BF90AF909F908F907F905E
:10EA80006F905F904F90089586EE9DE0E2CF809169
:10EA90000D0290910E0297FF03C087EB9DE09BCF84
:10EAA000009709F0B3C01D821E821F8218868DEC6C
:10EAB0009CECACE4BEE389839A83AB83BC83BE0148
:10EAC0006B5F7F4FCE0101960E942BF520910D02C6
:10EAD00030910E02203431050CF0C7C081E08093E4
:10EAE0003802C901019690930E0280930D02822F85
:10EAF000877887FF03C08150886F8F5FA82FE22F30
:10EB000027FF02C0E7E0E20FE595E595E595E0FF18
:10EB100002C0A7E0A81B84E0A802D0011124A65AD5
:10EB2000B84E8D909D90AD90BC9094E0E902F001BC
:10EB30001124E65CF84E40805180628073808DEC39
:10EB40009CECACE4BEE38D839E83AF83B8871982CF
:10EB50001A821B821C82CE0101966C01E12CF12CE1
:10EB600000EA10E4A3019201C501B4010E9473F40C
:10EB700019821A821B821C82B601CE0105960E9460
:10EB80002BF58092491190924A11A0924B11B092AC
:10EB90004C1140924D1150924E1160924F11709253
:10EBA000501110920A0500910D0210910E0280E49E
:10EBB000E82EF12C003411050CF47801B70180E542
:10EBC0009DE00E94DF3E60E470E08BE49DE00E94E7
:10EBD000DF3E8AE00E941837101611060CF015CFA0
:10EBE0001F9280E48F93FF92EF9284E39DE09F93C6
:10EBF0008F9382E49DE09F938F931F920E948BB529
:10EC00000FB6F894DEBF0FBECDBFFFCE8150982F58
:10EC1000977897FF03C09150986F9F5FE92F87FD0A
:10EC2000895F85958595859580FF02C0E7E0E91BA2
:10EC300028E0E202F0011124E80FF11D87FDFA95AA
:10EC4000EE0FFF1FEE0FFF1FE952FA4F8091511197
:10EC500090915211A0915311B091541180839183DE
:10EC6000A283B3831092380231CF80E090E0A0EA13
:10EC7000B0E48093511190935211A0935311B0932B
:10EC800054118CE792E00E9458F40E946ADF8FEFE3
:10EC90009FEF90930E0280930D0283EA9DE00E9405
:10ECA000513781E99DE00F94E64563E972E084E61F
:10ECB00090E00E945E806AEB72E084E690E00E9441
:10ECC0005E808BE89DE00E94407281E00E940D35DD
:10ECD00068CF89E40E94A132882371F00E94253216
:10ECE000182F883068F067E070E088E79DE00E94A8
:10ECF000DF3E85E79DE06FCE8AE40E949638ADCE78
:10ED00008AE40E94A1328823B9F30E942532082F99
:10ED1000883048F067E070E082E69DE00E94DF3EC8
:10ED20008FE59DE058CE8AE50E94A1328823A9F0A4
:10ED30000E94293228E01202F0011124E00FF11D97
:10ED400007FDFA95EE0FFF1FEE0FFF1FE952FA4F76
:10ED5000608371838283938358CE8AE5CECF8AE520
:10ED60000E94A1328823C9F30E9429326093D706FA
:10ED70007093D8068093D9069093DA0646CECF9347
:10ED8000DF93C0914712C0930C0A81E6C89FE0014F
:10ED90001124C75BDD4E8091FF1080FF05C00E94EB
:10EDA0001849CE010E941F37CE010E94662D80E0D7
:10EDB000DF91CF910C941C5D8F929F92AF92BF9286
:10EDC000CF92DF92EF92FF92CF936B017C0120E014
:10EDD00030E0A9010F94175687FFA3C06DEB77E3CE
:10EDE00086E095EBA70196010F94095D6B017C010C
:10EDF00020E030E040E251E40F947D5620E030E026
:10EE000048EC52E40F947D564B015C0120E030E069
:10EE100040E251ECC701B6010F941756181654F48E
:10EE200020E030E048EC52E4C701B6010F94695F7E
:10EE300087FD8BC020E030E0A901C701B6010F9427
:10EE4000175687FF73C060E070E080EA90ECA50180
:10EE500094010F94095D20E030E040E251E40F940A
:10EE6000035E0F94755E6B017C01F7FC64C020E1CA
:10EE700037E240E050E00F947D5CCA01B9012AE01E
:10EE800030E040E050E00F947D5C605D6093B2053F
:10EE9000C701B60128EE33E040E050E00F947D5CFE
:10EEA0009AE0892E912CA12CB12CCA01B901A5019F
:10EEB00094010F947D5C605D6093B305C701B6015A
:10EEC00024E630E040E050E00F947D5CCA01B901D7
:10EED000A50194010F947D5C605D6093B4058EE2A2
:10EEE0008093B505C701B601A50194010F947D5C1F
:10EEF000C62FCA01B901A50194010F947D5C605D24
:10EF00006093B605C05DC093B70582EB95E0CF91E5
:10EF1000FF90EF90DF90CF90BF90AF909F908F9039
:10EF200008956DEB77E386E095E35CCF60E070E0F9
:10EF300080EA90E48CCFF094E094D094C094C11C0B
:10EF4000D11CE11CF11C6DE2A1CF20E030E0A90151
:10EF5000C701B6010F94175687FF6AC060E070E0E2
:10EF600080EA90ECA50194010F94095D20E030E067
:10EF700040E251E40F94035E0F94755E4B015C0117
:10EF800020E030E0A901C701B6010F94695F87FD59
:10EF90000BC020E030E040E251E4C701B6010F941D
:10EFA000175660E287FD13C0B7FC47C0C501B40126
:10EFB00028EE33E040E050E00F947D5CCA01B901D7
:10EFC0002AE030E040E050E00F947D5C605D6093AB
:10EFD000B305C501B40124E630E040E050E00F94F1
:10EFE0007D5C8AE0C82ED12CE12CF12CCA01B9013C
:10EFF000A70196010F947D5C605D6093B4058EE27D
:10F000008093B505C501B401A70196010F947D5CFD
:10F01000C62FCA01B901A70196010F947D5C605DFE
:10F020006093B605C05DC093B70583EB95E06FCFE5
:10F0300060E070E080EA90E495CFB094A094909462
:10F040008094811C911CA11CB11C6DE2C0CF609109
:10F05000350270913602072E000C880B990B0F9425
:10F060001E562AE037ED43E25CE30F947D56209173
:10F07000C2053091C3054091C4055091C5050F9458
:10F080007D566093810270938202809383029093F5
:10F0900084020895E091DB08E23030F4F0E0E75CB0
:10F0A000F54F8091D1088083089580917A17882345
:10F0B000C1F0815080937A17E6EAF7E1882351F096
:10F0C0008150990B2BE1289FF001299FF00D11240D
:10F0D000E452F84E8BE1A1ECB7E101900D928A95D4
:10F0E000E1F720917A17211105C080918517806280
:10F0F0008093851781E090E0A0E0B0E0211103C08B
:10F1000080E090E0DC018093C9089093CA08A09346
:10F11000CB08B093CC081092CE0881E08093C80849
:10F1200083E0809380020895CF93DF93EC01CB01BD
:10F13000BA010F941E5629EC38EC48EC5EE30F94AC
:10F14000035E20E030E040E05FE30F94095D0F9440
:10F150007C5E6883DF91CF910895E091DB0886E0C3
:10F16000E802F0011124EC54F74F8091D10890E0AF
:10F17000958384830895CF93DF93EC01CB01BA018B
:10F180000F941E5620E030E0A9010F94095D0F9402
:10F190007C5E6883DF91CF9108958F929F92AF92AA
:10F1A000BF92CF92DF92EF92FF92CF936B017C01DF
:10F1B00020E030E0A9010F94175687FD9FC06DEB4A
:10F1C00077E386E095E3A70196010F94095D6B0153
:10F1D0007C0120E030E040E251E40F947D5620E0D5
:10F1E00030E048EC52E40F947D564B015C0120E086
:10F1F00030E0A901C701B6010F94175620E030E0B6
:10F2000040EA50E487FF04C020E030E040EA50ECE0
:10F21000C501B4010F94095D20E030E040E251E403
:10F220000F94035E0F94755E6B017C018BE2F7FE19
:10F2300009C0F094E094D094C094C11CD11CE11C8E
:10F24000F11C8DE28093B105C701B60120E137E2E0
:10F2500040E050E00F947D5C8AE0882E912CA12C38
:10F26000B12CCA01B901A50194010F947D5C605DC8
:10F270006093B205C701B60128EE33E040E050E0EC
:10F280000F947D5CCA01B901A50194010F947D5CC6
:10F29000605D6093B305C701B60124E630E040E04D
:10F2A00050E00F947D5CCA01B901A50194010F944F
:10F2B0007D5C605D6093B4058EE28093B505C70107
:10F2C000B601A50194010F947D5CC62FCA01B90156
:10F2D000A50194010F947D5C605D6093B605C05DEF
:10F2E000C093B70581EB95E0CF91FF90EF90DF9051
:10F2F000CF90BF90AF909F908F9008956DEB77E384
:10F3000086E095EB60CF8F929F92AF92BF92CF92A3
:10F31000DF92EF92FF92CF936B017C0120E030E00F
:10F32000A9010F94175687FDAAC06DEB77E386E01D
:10F3300095E3A70196010F94095D6B017C0120E024
:10F3400030E0A9010F94175687FF9EC0C701B60190
:10F35000905820E030E040E251E40F947D5620E0E8
:10F3600030E040E251E40F947D5620E030E040EA86
:10F3700050E40F94095D20E030E040E251E40F9446
:10F38000035E0F94755E6B017C0180E28093B10592
:10F3900060E280E1C81687E2D806E104F1048CF04F
:10F3A000C701B60120E137E240E050E00F947D5CF8
:10F3B000CA01B9012AE030E040E050E00F947D5CE2
:10F3C000605D6093B20560E288EEC81683E0D806FF
:10F3D000E104F1048CF0C701B60128EE33E040E00F
:10F3E00050E00F947D5CCA01B9012AE030E040E0B2
:10F3F00050E00F947D5C605D6093B30560E284E64D
:10F40000C816D104E104F1048CF0C701B60124E66A
:10F4100030E040E050E00F947D5CCA01B9012AE081
:10F4200030E040E050E00F947D5C605D6093B40597
:10F430008AE0882E912CA12CB12CC701B601A50120
:10F4400094010F947D5CC62FCA01B901A5019401F6
:10F450000F947D5C605D6093B5058EE28093B60588
:10F46000C05DC093B70581EB95E0CF91FF90EF9021
:10F47000DF90CF90BF90AF909F908F9008956DEBED
:10F4800077E386E095EB55CF20E030E040E251E4B1
:10F49000C701B60162CFCF93DF93EC01CB01BA0174
:10F4A0000F941E5620E030E040E251E40F94035EDA
:10F4B00020E030E0A9010F94095D688379838A8395
:10F4C0009B83DF91CF910895CF93DF93EC01CB0124
:10F4D000BA010F941E5620E030E040E251E40F9450
:10F4E000035E20E030E0A9010F94095D6883798311
:10F4F0008A839B83DF91CF9108950F941E5620E05D
:10F5000030E040E251E40F94035E20E030E0A901D6
:10F510000F94095D0C948379CF93DF93EC01CB01B9
:10F52000BA010F941E562AE037ED43E25DE30F94D3
:10F53000035E20E030E0A9010F94095D0F947C5E2A
:10F54000688379838A839B83DF91CF910895CF93DA
:10F55000DF93EC01CB01BA010F941E562AE037ED80
:10F5600043E25DE30F94035E20E030E0A9010F94D5
:10F57000095D688379838A839B83DF91CF910895A6
:10F58000CF93DF93EC01CB01BA010F941E5620E01C
:10F5900030E0A9010F94095D688379838A839B8396
:10F5A000DF91CF910895CF93DF93EC01CB01BA01A6
:10F5B0000F941E5620E030E0A9010F94095D688386
:10F5C00079838A839B83DF91CF910895CF93DF93D3
:10F5D000EC01CB01BA010F941E5620E030E048EC5C
:10F5E00052E40F94035E20E030E0A9010F94095D1E
:10F5F000688379838A839B83DF91CF910895CF932A
:10F60000DF93EC01CB01BA010F941E5620E030E0ED
:10F6100048EC52E40F94035E20E030E0A9010F941F
:10F62000095D688379838A839B83DF91CF910895F5
:10F630000F941E5620E030E048EC52E40F94035E35
:10F6400020E030E0A9010F94095D0C94CD78CF93B0
:10F65000DF93EC01CB01BA010F941E5620E030E09D
:10F66000A9010F94095D0F94755E79836883DF911A
:10F67000CF910895CF93DF93EC01CB01BA010F94A2
:10F680001E5620E030E0A9010F94095D688379835C
:10F690008A839B83DF91CF910895CF93DF93EC0111
:10F6A000CB01BA010F941E5620E030E04AE754E443
:10F6B0000F94035E20E030E0A9010F94095D688398
:10F6C00079838A839B83DF91CF9108950F941E568F
:10F6D00020E030E048EC52E40F94035E20E030E09C
:10F6E000A9010F94095D0C94DC762CEA35EC47E215
:10F6F0005EE360919F057091A0058091A1059091B6
:10F70000A2050F94035E60938C1670938D16809300
:10F710008E1690938F1608952CEA35EC47E25EE33F
:10F720006091A3057091A4058091A5059091A6050F
:10F730000F947D56609388167093891680938A166D
:10F7400090938B1608952CEA35EC47E25EE36091C6
:10F750009F057091A0058091A1059091A2050F943D
:10F76000035E60938C1670938D1680938E16909323
:10F770008F1608952CEA35EC47E25EE36091A3050D
:10F780007091A4058091A5059091A6050F947D56D2
:10F79000609388167093891680938A1690938B16BF
:10F7A00008958091D1089091D208A091D308B0918A
:10F7B000D4088093510290935202A0935302B093C5
:10F7C00054020895E0919805E63010F581E08E0F1F
:10F7D000809398054091C9085091CA086091CB0860
:10F7E0007091CC089091CE088091C70828E0E29FE4
:10F7F000F0011124E75AFA4F2091F9163091FA16C8
:10F800003183208342835383648375839683878304
:10F810000895FC01A081B1811C92A281B3818C91D9
:10F820008F5F8C930280F381E02D90818CE0989F14
:10F83000800D1124EBEFF6E113AE84AF0895CF9263
:10F84000DF92EF92FF92CF93DF9300D01F92CDB75C
:10F85000DEB76B017C0120E030E0A9010F94175660
:10F8600087FD1CC06DEB77E386E095E3A701960169
:10F870000F94095D69837A838B839C8360E2CE0158
:10F8800001960F9449020F900F900F900F90DF9107
:10F89000CF91FF90EF90DF90CF9008956DEB77E3DD
:10F8A00086E095EBE3CF0F941E5620E030E04AE768
:10F8B00054E40F94035E20E030E0A9010F94095D49
:10F8C0000C941F7CCF92DF92EF92FF926B017C0130
:10F8D00020E030E0A9010F94175687FD26C06DEB9C
:10F8E00077E386E095E3A70196010F94095D6B012C
:10F8F0007C0120E030E0A9010F94175620E030E0B1
:10F9000040E05FE387FF04C020E030E040E05FEBD1
:10F91000C701B6010F94095D0F94755ECB01FF908E
:10F92000EF90DF90CF900D940B046DEB77E386E0C2
:10F9300095EBD9CF0F941E5620E030E0A9010F942B
:10F94000095D0C94627C0F941E5620E030E0A90102
:10F950000F94095D0F94755ECB010D940B040F9409
:10F960001E5629EC38EC48EC5EE30F94035E20E071
:10F9700030E040E05FE30F94095D0F947C5E862FDA
:10F980000D9462040D94EF380D94EF386FEF809171
:10F99000D1080D940D376EE475EB82E00D94CC47E1
:10F9A00063E575EB81E00D94CC4768E575EB80E08D
:10F9B0000D94CC4769E073EB83E00D94CC47CF9274
:10F9C000DF92EF92FF92CF93DF9300D01F92CDB7DB
:10F9D000DEB76B017C0120E030E0A9010F941756DF
:10F9E00087FD1BC06DEB77E386E095E3A7019601E9
:10F9F0000F94095D69837A838B839C83CE01019682
:10FA00000F94E5020F900F900F900F90DF91CF9120
:10FA1000FF90EF90DF90CF9008956DEB77E386E055
:10FA200095EBE4CF0F941E5620E030E040E251E425
:10FA30000F94035E20E030E0A9010F94095D0C945F
:10FA4000DF7C8091C3169091C416891B8F7011F4CE
:10FA50000C94713681E0089580918002882351F0E2
:10FA600060919D0570919E0530E020E041E081E0CD
:10FA70000C94C72A089584E00D94E03583E00D943A
:10FA8000E03582E00D94E0350F941E5620E030E022
:10FA9000A9010F94095D0F947C5E862F0D9440049C
:10FAA0009091481181E089270C940D3561E081ED3A
:10FAB00098E00C9428350F94C92D0C947AF580E0C9
:10FAC00090E0A0E8B0E48093511190935211A0937C
:10FAD0005311B09354118FED92E00E9458F4E091CD
:10FAE000A80580E090E0A8E4B3E4E43009F44AC05B
:10FAF00080E090E0A0EBB1E48093491190934A112B
:10FB0000A0934B11B0934C1180934D1190934E11D3
:10FB1000A0934F11B0935011EE0FFF0BE154FD4F26
:10FB2000808191818330910549F184309105D9F12B
:10FB3000029761F480E090E0ADEBB3E4809349116B
:10FB400090934A11A0934B11B0934C1187EC92E023
:10FB50000E9458F4109251111092521110925311A8
:10FB6000109254118FED92E00E9458F48091A805F4
:10FB70008F5F8530ECF48093A805089580E090E0D5
:10FB8000ADEBB3E48093491190934A11A0934B11CC
:10FB9000B0934C1180934D1190934E11A0934F113F
:10FBA000B0935011D3CF80E090E0ADEBB3E4F2CF4F
:10FBB0001092A8050895CF93DF9300D01F92CDB780
:10FBC000DEB70F947C5E0F941C5669837A838B8317
:10FBD0009C83CE0101960F94C6010F900F900F9059
:10FBE0000F90DF91CF9108950F941E562AE037EDC4
:10FBF00043E25DE30F94035E20E030E0A9010F943F
:10FC0000095D0C94DB7DCF92DF92EF92FF92CF9350
:10FC1000DF9300D01F92CDB7DEB76B017C0120E0EF
:10FC200030E0A9010F94175687FD1BC06DEB77E3F9
:10FC300086E095E3A70196010F94095D69837A83B5
:10FC40008B839C83CE0101960F94C6010F900F9079
:10FC50000F900F90DF91CF91FF90EF90DF90CF90BA
:10FC600008956DEB77E386E095EBE4CF0F941E5695
:10FC70002AE037ED43E25DE30F94035E20E030E0DD
:10FC8000A9010F94095D0C94037E0F941E5620E089
:10FC900030E0A9010F94095D0C94037ECF92DF92AE
:10FCA000EF92FF926B017C0120E030E0A9010F94FC
:10FCB000175687FD26C06DEB77E386E095E3A70135
:10FCC00096010F94095D6B017C0120E030E0A901F1
:10FCD0000F94175620E030E040E05FE387FF04C058
:10FCE00020E030E040E05FEBC701B6010F94095D12
:10FCF0000F94755ECB01FF90EF90DF90CF900D9445
:10FD000061036DEB77E386E095EBD9CF0F941E5638
:10FD100020E030E0A9010F94095D0C944E7E0C9414
:10FD200046DF0C9446DF0C9446DF0C9446DF0C94BF
:10FD3000F8DE0C94F8DE0C94F8DE0C94F8DECF922A
:10FD4000DF92EF92FF92CF93C82F0F94E3386B01AD
:10FD50007C0124EA30E74DE75FE360912502709172
:10FD6000260280912702909128020F94175687FD52
:10FD700018C08AEF90E0A0E0B0E08C0D9D1DAE1D94
:10FD8000BF1D8093430590934405A0934505B09310
:10FD90004605C0931E02CF91FF90EF90DF90CF9069
:10FDA000089580E090E0DC01E8CFCF92DF92EF92FF
:10FDB000FF920F931F930F94E33800911405109155
:10FDC000150520911605309117056B017C01C01AAD
:10FDD000D10AE20AF30A9701860137FD11C020918A
:10FDE00013052095209313056A547C4F8F4F9F4F26
:10FDF000609314057093150580931605909317056D
:10FE000081E090911305911101C080E01F910F9145
:10FE1000FF90EF90DF90CF9008950F9418461092C6
:10FE2000FB08109274020E949C36882351F0809146
:10FE3000851782FD06C081E39EE19093710880934F
:10FE4000700861E08AE29EE10E949C380D9479017D
:10FE50004F925F926F927F928F929F92BF92CF92BA
:10FE6000DF92EF92FF920F931F93CF93DF9300D017
:10FE700000D01F921F92CDB7DEB77C016A01490105
:10FE8000FB0190818CE0989F800D1124982FF70141
:10FE90002081822F880F820F880F809336179093CE
:10FEA00037174115510571F1FA82E9827C836B8322
:10FEB000011121C0AE014B5F5F4FB401C6010E942A
:10FEC00003286C016D817E818F8198856115710594
:10FED00081059105B9F00E946429F70180818F5F47
:10FEE0008083853138F3CE0101960E94097CE2CFF0
:10FEF000B12C860129C08A01B12C26C0452846288C
:10FF00004728B1F728960FB6F894DEBF0FBECDBFD5
:10FF1000DF91CF911F910F91FF90EF90DF90CF90E5
:10FF2000BF909F908F907F906F905F904F900895BB
:10FF3000B39407C0B1102EC001151105C9F20F5FAF
:10FF40001F4F01151105A9F2AE014B5F5F4FB401C0
:10FF5000C6010E9403286C014D805E806F8078840A
:10FF60004114510461047104A9F0F0E24F165104E8
:10FF700061047104F9F2D301C2018D97A109B1099D
:10FF80000297A105B10530F04BE24416510461041B
:10FF9000710471F6F7018081482F4B0D5527551FCD
:10FFA0004631510534F0853020F0CE0101960E9493
:10FFB000097C81E0411451046104710409F480E07A
:10FFC000B80EF70180818B0D8083BB2009F496CF9A
:10FFD000BA94AE014B5F5F4FB401C8010E94032881
:10FFE0008C016D817E818F8198850E946429EDCF7F
:10FFF000EF92FF920F931F93CF93DF9300D000D027
:020000021000EC
:1000000000D01F921F92CDB7DEB77C012091CF08A0
:10001000422F022E000C550B8091D008833099F1AD
:10002000843051F18AEC91E25F932F939F938F93E9
:100030008E010F5F1F4F1F930F930F94AE55C70193
:100040000E94ECDE4FE350E0B80182E798E00F94A5
:100050007E600F900F900F900F900F900F902B9647
:100060000FB6F894DEBF0FBECDBFDF91CF911F91C9
:100070000F91FF90EF90089586ED91E227FDD4CF88
:1000800081EC91E2D1CF8FED91E2CECFE091DB0810
:1000900085E1E802F0011124E558F94E8681978147
:1000A0000C94F87FE091DB0886E0E802F00111246F
:1000B000EC54F74F808191810C94F87F0F931F933C
:1000C000CF93DF938C01EB019091E7162091E81616
:1000D000921305C00F9448050E947CF5F5CF8091DE
:1000E000E61634E0839FF0011124E751F94E1183A5
:1000F0000083D383C2839F5F9093E7168F5F281797
:1001000039F08093E616DF91CF911F910F910895FA
:100110001092E616F8CF63E972E084E690E00E9460
:100120005E806AEB72E084E690E00C945E80811160
:100130000C948B8068EB71E084E190E00C945E801D
:100140000E9443DB0C9497800F942D160C9497809B
:100150000E9436FF0C948B80CF93DF93CDB7DEB730
:1001600020E2488559856F818E810F947032DF912E
:10017000CF910895282F1092D9088091C9089091A5
:10018000CA08A091CB08B091CC08B7FF08C0109264
:10019000C9081092CA081092CB081092CC0880911E
:1001A000B005882331F08091C9088093CD08109262
:1001B000C8088091C7081816FCF4082E000C990B8B
:1001C000821B91092091CD08022E000C330B2817B9
:1001D000390794F097FF02C090E080E08093CD084B
:1001E000092E000CAA0BBB0B8093C9089093CA0878
:1001F000A093CB08B093CC088091CD086623A9F0DA
:100200009091CE08891714F48093CE082091CE08DF
:10021000022E000C330B2C5F3F4F482F082E000C92
:10022000550B241735071CF484508093CE0808958D
:100230005F926F927F928F929F92AF92BF92CF9276
:10024000DF92EF92FF920F931F93CF93DF9361E0C2
:1002500081E00E94BA80C091CE0885E0982E9C0E65
:10026000D1E094E1E92E92E2F92E882483947D2E48
:100270007C1A6C2E61942FE1C22E22E2D22E12E063
:100280001C1B33E0532E40E8A42E42E2B42EC111D1
:1002900041C0DD23D9F08091CD081816BCF0409103
:1002A000C9085091CA086091CB087091CC084F5F83
:1002B0005F4F6F4F7F4F4093C9085093CA086093B8
:1002C000CB087093CC088F5F8093CD08809180021B
:1002D000882341F030E020E041E068E272E2862DC0
:1002E0000E94C72A8091F908882309F487C0C23088
:1002F00051F48091CD08823009F445C0809180028C
:1003000081115AC0D0E0CF5F9C12C1CF83E08093AF
:10031000C70818C0C13031F79091CD08913031F045
:100320008091800281111EC0D0E0DCCF8091C60890
:100330001092C6088823A1F3C093FA088091C808D8
:10034000882371F3DF91CF911F910F91FF90EF9070
:10035000DF90CF90BF90AF909F908F907F906F90E5
:100360005F9008951F92FF92EF927F9281E091300B
:1003700009F080E08F930E94AC800F900F900F9057
:100380000F900F90D1CF8091C6081092C608882395
:1003900009F4B4CF8091550288258093550250927C
:1003A0008002A114B10411F00E9480228091C8083B
:1003B000882309F4A3CFC6CF81E09091CD08923075
:1003C00009F080E09091550223E032E2911102C0E1
:1003D0002FEF31E201E046E052E2612F0E94C22B92
:1003E00091CF8091C6081092C608882371F0C093FF
:1003F000FA088091C808882341F0A4CFC23009F0E0
:1004000082CF9091CD08923061F380918002882351
:1004100009F478CF1F92DF92CF921F9381E0923040
:1004200009F080E08F930E94AC800F900F900F90A6
:100430000F900F9067CF2F923F924F925F926F92E3
:100440007F928F929F92AF92BF92CF92DF92EF9264
:10045000FF920F931F93CF93DF934C010F9464553A
:1004600001968401080F191FC8010F946455019665
:100470006801C80ED91EF8016080C1E0611001C09A
:10048000C0E0F6013080D1E0311001C0D0E0AA24F4
:10049000A3946110A12C60E085E00E94BA80509086
:1004A000CE08752C9EE0E92EF12C252C21948A2D66
:1004B00090E001965C01AC0EB11CAD0EB11C711048
:1004C0001DC0809180028823A1F0E0912402E250B7
:1004D00068E372E2E33038F4F0E0EE0FFF1FE95119
:1004E000FD4F6081718130E020E043E0822D0E9469
:1004F000C72AD1E0611013C0D2E011C0D2E0611070
:10050000D1E0D7110CC080918002882341F030E007
:1005100020E041E0B4018D2F85190E94C72AC1E077
:10052000CD0F472C4518662079F0C7110BC080917C
:100530008002882339F030E020E041E0B801842DCA
:100540000E94C72AC2E0CD0F332071F0C7110BC043
:1005500080918002882339F030E020E041E0B6014C
:10056000842D0E94C72ACF5FF3E0AF16B1040CF4CC
:10057000CF5FC71162C080918002882309F45AC0FE
:1005800030E020E042E065E472E2842D0E94C72A58
:10059000D091110593EF9E0D909310058EEF8E0D67
:1005A0008093DA08209133172E151F0411F00CF0F8
:1005B00041C0209135179217E8F59EE390933617C6
:1005C0008093371765E470E080E090E00E94642932
:1005D00061E36D0F062E000C770B880B990B0E94C0
:1005E000642960E270E080E090E00E9464298091DC
:1005F0007F16909180160F940B040E943F2B6FE2A0
:1006000070E080E090E00E9464290E94D57E811114
:1006100009C085E08D9FF0011124E651F94F8481D6
:10062000811108C080918116909182160F940B045D
:100630000E943F2B92E090938002ECE0EE0EF11CC2
:100640007394FAE4EF16F10409F039CFCF5FC09349
:10065000C708DF91CF911F910F91FF90EF90DF902E
:10066000CF90BF90AF909F908F907F906F905F9052
:100670004F903F902F90089580E592E20C941B825A
:100680008DE592E20C941B828FE792E20C941B8220
:100690008AE193E20C941B8285ED92E20C941B821A
:1006A00082E093E20C941B8285E593E20C941B821A
:1006B00088E393E20C941B8288EB92E20C941B82F9
:1006C00089E992E20C941B828F929F92AF92BF9223
:1006D000EF92FF920F931F93CF93DF93EC018B0167
:1006E000E42EF22E8091F9169091FA168C179D0740
:1006F00009F43EC02091090527FD1092090526EB5B
:10070000C432D20709F03FC088539F4B71F40F9455
:10071000E3386E517B4F8F4F9F4F609399057093D5
:100720009A0580939B0590939C05D093FA16C093ED
:10073000F91630E020E00093C9081093CA0820930E
:10074000CB083093CC08E092CE08F092C708C8538B
:10075000DF4B21F4109212051092980582E08093ED
:10076000800281E08093C8081092AD051092A70521
:10077000DF91CF911F910F91FF90EF90BF90AF90BD
:100780009F908F9008952FEBC833D20771F6845253
:10079000964B19F0C8E3DFEBC8CF0F94E338809095
:1007A000990590909A05A0909B05B0909C056819BA
:1007B00079098A099B0997FFEDCF80916E088770B0
:1007C000873041F7C3EFD3E8B0CFCF93DF93EC018D
:1007D0000E94E27B20E040E070E060E0CE01DF912B
:1007E000CF910C94648320E040E070E060E082E10F
:1007F00092EB0E94648381E0809312051092F708C7
:100800001092F608089520E040E070E060E08AED84
:100810009CE70C94648380914B0A811114C08091F1
:10082000850290918602019720917F163091801663
:100830002817390744F420E040E070E060E08DE1E3
:100840009EEB0C9464830C94038421E020931205A6
:10085000FC0180819181A281B381809325029093D4
:100860002602A0932702B093280220E040E070E027
:1008700060E08091C4089091C5080C946483CF9384
:10088000DF9300D01F92CDB7DEB78DEC9CECACECC3
:10089000BCE389839A83AB83BC83CE0101960E941B
:1008A00025840F900F900F900F90DF91CF910895B6
:1008B000CF93DF9300D01F92CDB7DEB78DEC9CECC9
:1008C000ACECBDE389839A83AB83BC83CE010196F4
:1008D0000E9425840F900F900F900F90DF91CF9181
:1008E0000895CF93DF9300D01F92CDB7DEB780E09D
:1008F00090E0A0E8BFE389839A83AB83BC83CE01F9
:1009000001960E9425840F900F900F900F90DF9119
:10091000CF910895CF93DF9300D01F92CDB7DEB76C
:1009200080E090E0A0E2B1E489839A83AB83BC834A
:10093000CE0101960E9425840F900F900F900F908A
:10094000DF91CF9108958FEF8093D10820E040E0B0
:1009500070E060E089E399E90C94648381E080931E
:10096000120510926E081092B90520E040E070E088
:1009700060E085EE94E80E94648383E996E29093B8
:10098000710880937008089581E08093120580912A
:100990006E088770873051F010926E081092B9057A
:1009A00083E996E2909371088093700880914811D2
:1009B0008093A90580E00E940D3520E040E070E0C2
:1009C00060E086E396E80C9464838091800288233B
:1009D00041F030E020E041E06DE670E282E00E940C
:1009E000C72A8091B9058770873041F420E040E044
:1009F00070E060E088E195E80C946483089520E05D
:100A000040E070E060E08FE295E80E94648381E05E
:100A100080930A058091AA05811107C082E590E2C2
:100A20009093710880937008089588E590E2F8CF5C
:100A300080918002882341F030E020E041E06EE5C3
:100A400070E281E00E94C72A8091C6081092C60811
:100A5000882321F01092AA050C94FF8408950F9327
:100A60001F93CF93DF9300D000D000D01F92CDB75B
:100A7000DEB7809180028823F1F01F9280E48F938B
:100A80008091AA0590E001969F938F938AE490E26B
:100A90009F938F938E010F5F1F4F1F930F930F94A0
:100AA000AE55B8018FE390E20E94432B0FB6F89445
:100AB000DEBF0FBECDBF84E08093800280910A0527
:100AC000811108C020E040E070E060E085E795E833
:100AD0000E9464832A960FB6F894DEBF0FBECDBF86
:100AE000DF91CF911F910F910895CF92DF92EF92F6
:100AF000FF92CF93DF9300D01F92CDB7DEB78091E6
:100B0000C6081092C608882331F18091AA058F5F2C
:100B10008093AA058034E0F081E080930A0520E00C
:100B200040E070E060E08DE595EB0E94648389E32E
:100B300090E290937108809370080F900F900F903F
:100B40000F90DF91CF91FF90EF90DF90CF900895BD
:100B50000E94FF84F2CF6091C9087091CA08809109
:100B6000CB089091CC08611571058105910509F4B8
:100B70003EC00F941E562DEC3CEC4CEC5CE30F9405
:100B80007D56209151113091521140915311509145
:100B900054110F94095D6B017C0120E030E040E8C6
:100BA00050EC0F94175687FD53C020E030E040E82A
:100BB00050E4C701B6010F94695F18160CF44FC0DA
:100BC000C0925111D0925211E0925311F0925411EF
:100BD0008FED92E00E9458F482E0809380021092A0
:100BE000C9081092CA081092CB081092CC088091C4
:100BF0008002882309F4A1CFC0905111D0905211E6
:100C0000E0905311F090541120E030E0A901C701A9
:100C1000B6010F94175627E137EB41ED58E387FFF4
:100C200004C027E137EB41ED58EBC701B6010F9443
:100C3000095D69837A838B839C836BE2CE01019685
:100C40000F944902BC0182E390E20E94432B75CFCE
:100C5000C12CD12C90E8E92E90ECF92EB1CFC12C0B
:100C6000D12C80E8E82E80E4F82EAACF8091800273
:100C7000882341F030E020E041E06DE670E282E060
:100C80000E94C72A8091B9058770873079F4109245
:100C9000A80520E040E070E060E08FEE9EEB0E944F
:100CA000648381E08093A7050C945F7D08952F9263
:100CB0003F924F925F926F927F928F929F92AF92EC
:100CC000BF92CF92DF92EF92FF920F931F93CF9339
:100CD000DF9300D000D0CDB7DEB71C017A836983E3
:100CE0002B833C834D835E832701380181E0809311
:100CF000C8080E94E27B83E08093800230929705CF
:100D00002092960589819A81909395058093940508
:100D10008B819C81AD81BE818093900590939105DC
:100D2000A0939205B093930540928C0550928D0547
:100D300060928E0570928F05F12CE12CC092C9084B
:100D4000D092CA08E092CB08F092CC08B092FA1682
:100D5000A092F91690928B0580928A058C8D8093D3
:100D6000890526960FB6F894DEBF0FBECDBFDF9182
:100D7000CF911F910F91FF90EF90DF90CF90BF9098
:100D8000AF909F908F907F906F905F904F903F902B
:100D90002F90089520E040E070E060E088E39FEB52
:100DA0000C9464830E94D3360E94CCD70C94CA86DC
:100DB00084E099E00F9457440E94CA860D94184627
:100DC0000E94CA868FED94E2909371088093700818
:100DD00008950E942B340F941D4581E080937B176A
:100DE0000F945F450C94CA866F927F928F929F9268
:100DF000AF92BF92CF92DF92EF92FF920F931F9329
:100E0000CF93DF9381E08093120561E00E94BA8066
:100E1000C091CE0885E0882E8C0ED1E009EE16E850
:100E200095EEE92E94E2F92E82E0982E9C1A20EE9F
:100E3000C22E26E8D22E30EFA32E34E2B32E7D2E22
:100E40007C1A6C2E6194C11130C0DD23D9F08091E1
:100E5000CD081816BCF04091C9085091CA0860919D
:100E6000CB087091CC084F5F5F4F6F4F7F4F40931F
:100E7000C9085093CA086093CB087093CC088F5F61
:100E80008093CD0880918002882341F030E020E0FB
:100E900041E06DEF74E2862D0E94C72ACF5F8C126D
:100EA000D2CF83E08093C70823C0C13081F5809101
:100EB000CD08813089F080918002882309F444C0F4
:100EC000DF92CF92BF92AF927F9281E09091CD0856
:100ED000913089F180E02FC08091C6081092C60839
:100EE000882349F30E94E0868091C808882319F37B
:100EF000DF91CF911F910F91FF90EF90DF90CF90F6
:100F0000BF90AF909F908F907F906F900895C23068
:100F100029F68091CD088230C9F080918002882323
:100F200099F01F930F93FF92EF929F9281E090911F
:100F3000CD08923079F68F930E94AC800F900F907D
:100F40000F900F900F900F90D0E0A8CF8091C6081F
:100F50001092C608882309F30E94E9868091C80888
:100F60008823D9F2C5CF6111609324024093110503
:100F70008C3008F03AC0E82F880FFF0B8827EC531D
:100F8000F8478F4F0D94005DF787D087DB87FA878E
:100F9000DE87E187E487F087E787F587EA87ED87D3
:100FA00080E493E821E02093120520E040E070E027
:100FB00060E00C94648388E493E8F4CF8CE493E8D5
:100FC000F1CF80E593E8EECF84E593E8EBCF88E5B9
:100FD00093E8E8CF8CE593E8E5CF80E693E8E2CFAD
:100FE0001092FA0888E191E8DDCF0C94CA868CE370
:100FF00093E8D8CF84E493E8D5CFCF930E9436FF0F
:101000000E9443DBC82F882319F080E00F94E90E7B
:101010008C2F0E949780CF910C94CA860F931F93B8
:10102000CF93DF93CDB7DEB76E970FB6F894DEBFE0
:101030000FBECDBF282F082E000C330B90911F023E
:10104000409120028F3F39F0F901EE0FFF1FEF5D55
:10105000FD4F908141814F939F933F938F9384E7FE
:101060009EE19F938F938E010F5F1F4F1F930F93EE
:101070000F94AE554FE350E0B80182E798E00F942B
:101080007E600E94CA860FB6F894DEBF0FBECDBF49
:101090006E960FB6F894DEBF0FBECDBFDF91CF9135
:1010A0001F910F9108958FEF0C940E888091DB08AB
:1010B0000C940E88E0919805EE2389F0E150E093BE
:1010C000980588E0E89FF0011124E75AFA4F628101
:1010D000738127814681808191810C9464830C9473
:1010E000CA862F923F924F925F926F927F928F9219
:1010F0009F92AF92BF92CF92DF92EF92FF920F93A7
:101100001F93CF93DF9300D01F92CDB7DEB761E07E
:1011100081E00E94BA802091CE082B832C83822FFD
:101120008B5F898389E0821B8A8388E0782E721A1C
:1011300087E0682E621A86E0582E521A85E0482E03
:10114000421A84E0382E321A222E21942B8121114A
:101150005BC08091CD08882399F18091800288231B
:1011600059F081E09091CD08911180E024E040E3B6
:1011700057E2622D0F9470328091390A8093D10822
:101180008B81853009F0A1C01092DB088091CD08D9
:10119000853009F45CC180918002882309F436C24D
:1011A00011E08091CD08853009F010E08091D108E0
:1011B0000F94620400E09C014DE057E2642D82C070
:1011C0008091C6081092C608882339F20E945A8876
:1011D0008091C808882309F4C0CF0F900F900F901A
:1011E0000F90DF91CF911F910F91FF90EF90DF90C3
:1011F000CF90BF90AF909F908F907F906F905F90B7
:101200004F903F902F9008958B818130B9F5809158
:10121000CD088130E1F080918002882309F4ACCFC1
:1012200011E08091CD08813009F010E080917602C4
:10123000909177020F940B0461E02C81621B00E017
:101240009C014AE257E2812F0E94C22B95CF8091E8
:10125000C6081092C6088823F1F210E000E027EEDD
:1012600033E04AE050E066E772E08AE297E20F94EA
:101270005D348091C808882371F2AFCF8B818230B2
:1012800009F087C18091CD08823009F44EC0809169
:1012900080028823D1F011E08091CD08823009F0DE
:1012A00010E06091D7067091D8068091D906909190
:1012B000DA060E941F7C62E02C81621B00E09C0128
:1012C00044E257E2812F0E94C22B80913A0A809318
:1012D000D1089B81963009F0E4C081E08093DB085F
:1012E0008091CD08863009F4C7C0809180028823A0
:1012F00091F011E08091CD08863009F010E08091E6
:10130000D1080F94620400E09C014DE057E2652D86
:10131000812F0E94C22B9B819F5F9B832981291370
:1013200015CF8AE08093C70858CF8091C6081092E5
:10133000C608882309F4ABCF20E030E04AE754E444
:101340006091D7067091D8068091D9069091DA06FF
:101350000F947D5620E030E0A9010F94095D20E054
:1013600030E04AE754E40F94095D0F947C5E1F92CD
:10137000912C812C80ECA82E81EBB82E6B0110ED06
:10138000E12E17E0F12E00E010E028E13CEF4FEFF6
:101390005FEF67ED76E084E297E20E9457860F9058
:1013A0008091C808882309F472CF17CF8091CD08A7
:1013B0008330C9F080918002882309F486CF11E040
:1013C0008091CD08833009F010E0809181169091D2
:1013D00082160F940B0463E02C81621B00E09C01D9
:1013E0004DE157E230CF8091C6081092C60888239D
:1013F00009F30F94E53204EC1CE72CE231E050E0F5
:1014000040E061E876E18DE197E20F945D348091F0
:10141000C808882379F2E1CE8091C6081092C608E8
:10142000882309F4C2C00F94E53206E919EC2CE8D0
:1014300030E050E040E06DE179E089E197E20F941F
:101440005D348091C808882309F4AFC0C6CE80916E
:10145000C6081092C608882309F49DCE0F94E53281
:101460006AE478E78DE097E20F949C358091C80894
:10147000882309F490CEB1CE8091C6081092C60898
:10148000882309F432CF0F94E5326AE478E78DE0DF
:1014900097E20F949C358091C808882309F425CFE2
:1014A0009CCE2B81273091F58091CD088730B9F003
:1014B00080918002882309F42ECF11E08091CD081D
:1014C000873009F010E080913502909136020F9438
:1014D0000B0400E09C0148E057E2662D19CF809193
:1014E000C6081092C608882319F307E218E727EE0A
:1014F00033E04AE050E065E372E088E097E20F9461
:101500005D348091C808882399F267CE8B8188303A
:1015100009F062C08091CD088830D9F080918002B6
:10152000882309F4F8CE11E08091CD08883009F0C5
:1015300010E06091310A7091320A8091330A9091E3
:10154000340A0E94DC7600E09C014EEF56E2672DE3
:10155000DFCE8091C6081092C6088823F9F261E3B5
:101560007AE08EEF96E20F9456358091C808882372
:10157000A9F233CE8091C6081092C6088823A1F143
:1015800083EF93E80E94E5838091C808882361F186
:1015900024CE8B81833009F409CF843009F0ECCD5F
:1015A0008091CD08843009F437CF80918002882360
:1015B00009F48BCE11E08091CD08843009F010E061
:1015C00080911D0990911E090F940B0400E09C016D
:1015D00049E157E2632D37CE9B81993009F09BCECC
:1015E0008091CD08893031F280918002882309F4FE
:1015F00092CE81E09091CD08993009F080E023E00F
:1016000043EF56E26A810F94703285CE80913A0A98
:101610008093D10880CE5F926F927F928F929F923B
:10162000AF92BF92CF92DF92EF92FF920F931F93F0
:10163000CF93DF93FF24F3948091811690918216CB
:10164000892B09F4F12C61E081E00E94BA80C091FD
:10165000CE088C2E95E0992E9C0EAA24A39484E0AB
:10166000E82EEC1A83E0D82EDC1A82E0C82ECC1AC1
:101670007A2C7C1A6C2E619487E0B82EBC1AC111AA
:10168000B8C08091CD08882309F495C0809180026C
:10169000882359F081E09091CD08911180E024E0F9
:1016A0004EEE56E2662D0F94703280913A0A809386
:1016B000D108C430E9F4A092DB088091CD088430D1
:1016C00009F445C180918002882391F0D1E0809196
:1016D000CD08843009F0D0E08091D1080F946204E5
:1016E00000E09C0147ED56E26E2D8D2F0E94C22B2B
:1016F00010E000E0D5E05C2E58180093D108CD131F
:101700001FC0F801EE0FFF1FE459FF4B8591949124
:101710009093DD088093DC088091CD088C1709F444
:101720002BC180918002882359F081E09091CD08EF
:101730009D1380E023E04DEC56E2652D0F9470324E
:101740008D2F0F5F1F4FD6E08630B9F680911D09AF
:1017500090911E09892B19F4FF2009F42DC1C7307F
:1017600009F58091CD08873009F417C18091800276
:101770008823C1F082ED96E89F938F9384EC96E2E4
:101780009F938F93BF9281E09091CD08973009F09D
:1017900080E08F930E94AC800F900F900F900F907D
:1017A0000F900F9088E0FF24F394CF5FC91167CFAB
:1017B0008093C7080EC08091C6081092C60888237F
:1017C00009F464CF0E945A888091C808882309F4DC
:1017D0005DCFDF91CF911F910F91FF90EF90DF9040
:1017E000CF90BF90AF909F908F907F906F905F90C1
:1017F0000895C13009F05FC08091CD08813009F4AF
:101800003FC080918002882309F44FCFD1E08091BE
:10181000CD08813009F0D0E0809181169091821638
:101820000F940B0400E09C0147EE56E2672D8D2FCC
:101830000E94C22B8091390A8093D108C33009F0ED
:1018400034CF1092DB088091CD08833009F46AC050
:1018500080918002882309F44BCFD1E08091CD089C
:10186000833009F0D0E08091D1080F94620400E049
:101870009C0147ED56E26D2D8D2F0E94C22B15CF96
:101880008091C6081092C608882309F4BACF0F9435
:10189000E53202EC1CE72CE231E050E040E061E888
:1018A00076E187EE96E20F945D348091C808882334
:1018B00009F4A7CF8ECFC23009F0BCCF8091CD08FC
:1018C0008230B9F080918002882309F4EECED1E015
:1018D0008091CD08823009F0D0E080911D0990916F
:1018E0001E090F940B0400E09C0143EE56E26C2DA0
:1018F0009ECF8091C6081092C608882319F30F94D2
:10190000E53206E919EC2CE830E050E040E06DE10A
:1019100079E083EE96E20F945D348091C8088823C5
:1019200089F257CF8091C6081092C608882309F41F
:101930008FCF0F94E5326AE478E787ED96E20F9453
:101940009C358091C808882309F482CF42CF8091CA
:10195000C6081092C608882309F4B4CE0F94E53265
:101960006AE478E787ED96E20F949C358091C80889
:10197000882309F4A7CE2DCF8091C6081092C608FF
:10198000882309F4CECE8EED9CE80E94E5838091F9
:10199000C808882309F4C5CE1CCF8091C6081092D0
:1019A000C608882309F4E2CE0E94D2868091C80836
:1019B000882309F4DBCE0DCF87E0F7CE4F925F92FC
:1019C0006F927F928F929F92AF92BF92CF92DF924F
:1019D000EF92FF920F931F93CF93DF930091D10863
:1019E00061E081E00E94BA80C091CE0810E0000F53
:1019F000111F04591F4B95E0592E5C0E2AEAE22E66
:101A000026E2F22ED3E0DC1B36ECC32E3CE7D32ECD
:101A10004CE9A42E46E2B42E82E0782E7C1A5DECCE
:101A2000852E56E2952E81E0682E6C1A4C2E41943C
:101A3000C11137C08091CD088823B1F08091800218
:101A4000882359F081E09091CD08911180E024E045
:101A500048EB56E2642D0F947032CF5F5C12E8CFF2
:101A600084E08093C7080CC08091C6081092C60815
:101A7000882321F30E945A888091C8088823F1F2B4
:101A8000DF91CF911F910F91FF90EF90DF90CF905A
:101A9000BF90AF909F908F907F906F905F904F908E
:101AA0000895C13059F5F801859194919093DD081E
:101AB0008093DC088091CD08813081F08091800294
:101AC000882359F21F929F928F926F9281E090919A
:101AD000CD08913009F474C080E072C08091C608CE
:101AE0001092C608882351F38091D108682F0F9473
:101AF0000D378091C808882309F3C2CFC23009F09E
:101B000042C0F801859194919093DD088093DC08A0
:101B10008091CD088230D1F080918002882309F431
:101B20009CCFDF92CF92BF92AF927F9281E0909153
:101B3000CD08923009F080E08F930E94AC800F9026
:101B40000F900F900F900F900F9087CF8091C60845
:101B50001092C608882301F30E94C67C8091C808B1
:101B60008823D1F28DCF8091C6081092C6088823B1
:101B7000C1F06091D1088FEF0F940D378091C808A4
:101B8000882379F07DCFC33009F067CFF8018591C4
:101B900094919093DD088093DC088091CD08833088
:101BA00011F380918002882309F457CF1F92FF928E
:101BB000EF92DF9381E09091CD08933009F08CCFC4
:101BC0008F930E94AC800F900F900F900F900F900A
:101BD00044CF9F92AF92BF92CF92DF92EF92FF924B
:101BE0000F931F93CF93DF9361E081E00E94BA804F
:101BF000C091CE08CC2E85E0982E9C0E94E5A92E9F
:101C000096E2B92ED7E0DC1B16E01C1B05E00C1B8E
